:100000000C94CC0C0C94FD0C0C94FD0C0C94FD0C7D
:100010000C94FD0C0C941C510C946E570C9466704F
:100020000C94FD0C0C94FD0C0C94FD0C0C94FD0C2C
:100030000C94FD0C0C94FD0C0C94FD0C0C94FD0C1C
:100040000C94FD0C0C947C600C94A0500C94FD0C52
:100050000C94FD0C0C94FD0C0C94FD0C0C94746E23
:100060000C94FD0C0C94404C0C94174C0C94FD0C0F
:100070000C94FD0C0C94FD0C0C94FD0C0C94FD0CDC
:100080000C94CF7E0C94FD0C0C94FD0C0C94FD0C88
:100090000C94EE4B0C94C54B0C94FD0C0C94FD0C85
:1000A0000C94FD0C0C94FD0C0C94FD0C0C94FD0CAC
:1000B0000C94FD0C0C9497680C94FD0C0C94FD0CA6
:1000C0000C94FD0C0C94FD0C0C94FD0C0C949C4BAE
:1000D0000C94734B0C94FD0C0C944A4B0C94214BD8
:1000E0000C94FD0C761353132F139313EB13B213CD
:1000F000E213D1139B147E145A14ED14B814B814DF
:10010000DC14C514E0170E1845187C1857198E1901
:10011000BC19EA19B11AB11AB11AB11AB11AB11A45
:10012000B11AB11AB11AB11AB11AB11AB11AB11A77
:10013000B11AB11AB11AB11AB11AB11AB11AB11A67
:10014000B11AB11AB11AB11AB11AB11AB11AB31857
:10015000EA182219181A461A7E1AB01CB61CBC1CC2
:10016000C21CC81CCE1CD41CDA1CE01CE61CEC1CF7
:10017000F21C041D0A1D101D161D1C1D221D281D0C
:100180002E1D341D3A1D401D461D4C1D521D581D6F
:100190005E1D641D701D7C1D821D881D8E1DA61D8B
:1001A000AC1DB21DB81DBE1DC41D7E1E841E8A1E40
:1001B000961E9C1EA21EAE1EB41EBA1EC01EC61ED9
:1001C000CC1EDE1EE41E0E1F141F1A1F201F381F18
:1001D0003E1F441F4A1F621F681F6E1F741F781F37
:1001E0007C1F801F861F8A1F8E1F921F961F9A1FBB
:1001F0009E1FA41FAA1FB01FB61FBC1FC21FC81F6F
:10020000CE1F941DCA1DD01DD61DDC1DE21DE81D8C
:10021000261F2C1F321F501F561F5C1FD41FDA1FB2
:10022000E01FD21ED81EEE1DF41DFA1D001E061E74
:100230000C1E901EA81E761DF81CFE1C9A1DA01DEB
:10024000E61FEC1FF21F6A1DEA1EF01EF61EFC1EC2
:10025000021F081F121E181E1E1E241E2A1E301EDC
:10026000361E3C1E421E481E4E1E541E5A1E601E46
:10027000661E6C1E721E781E8B338B33A5338B3338
:10028000B233CB33E63301341A481D480C481048CA
:1002900016485448214825482B482F4833483948A8
:1002A0003D484148544847484B484F48AA4DAF4DF8
:1002B000B44DBE4DC84D414ED24DDA4DE24DEC4DE0
:1002C000F64D004E0F4E194E414E234E2D4E374ED9
:1002D000C468CD68D568E968FB680D6918690F7452
:1002E000437478749874CD74027512753C76867573
:1002F0009075C475F9750776468A5D8A748A8B8A0B
:10030000A28AB98AD08AE78AFF8A1E8B358B4C8BEA
:100310006B8B818B212000464143544F5259205210
:10032000455345542120003400330032004E6F6E97
:10033000650053746F70706564004E65757472610A
:100340006C205475726E004D6F76696E6720526531
:100350007665727365004D6F76696E6720466F72C1
:1003600077617264004272616B696E670054414E3E
:100370004B20524553544F52454400250048656177
:100380006C7468204C6576656C3A20005645484987
:10039000434C452052455041495220434F4D504C0B
:1003A0004554450054414E4B2044455354524F59F7
:1003B00045440025004865616C7468204C6576658D
:1003C0006C3A2000290056454849434C4520524587
:1003D0005041495220535441525445442028005220
:1003E0004550414952204F5045524154494F4E20AB
:1003F00043414E43454C4C45440029004D41434840
:10040000494E452047554E20484954212028005246
:100410004550414952204F5045524154494F4E207A
:1004200043414E43454C4C454400290043414E4E08
:100430004F4E20484954212028005475727265742B
:1004400020726F746174696F6E206973206E6F74AF
:10045000206F66207479706520536572766F2E2048
:100460004E6F20736574757020617661696C61628E
:100470006C652E0054757272657420656C657661CA
:1004800074696F6E206973206E6F74206F662074BC
:1004900079706520536572766F2E204E6F207365DC
:1004A00074757020617661696C61626C652E0054B0
:1004B0006F70204C65667400546F702043656E74D5
:1004C000657200546F70205269676874004D6964EA
:1004D000646C65204C656674004D6964646C6520CD
:1004E00043656E746572004D6964646C6520526981
:1004F00067687400426F74746F6D204C6566740099
:10050000426F74746F6D2043656E74657200426F44
:1005100074746F6D205269676874004649524D5774
:100520004152452056455253494F4E3A20006942A8
:10053000757300534275730050504D004E6F6E65D9
:1005400020446574656374656400417A696D7574EF
:10055000682020202000456C65766174696F6E20EC
:1005600020005475726E2020202020202000546826
:10057000726F74746C6520202000537469636B2063
:100580002020202020204D696E2020202043656EF1
:100590007465722020204D61782020202044656100
:1005A0006462616E642020526576657273656400D2
:1005B000524144494F20494E464F202D20004E4F76
:1005C000542044455445435445440049474E4F52F6
:1005D000454400416E616C6F6700446967697461EE
:1005E0006C00417578204368616E2E2020204D6993
:1005F0006E20202020204D6178202020202054795A
:100600007065004368616E6E656C73207574696C0B
:10061000697A65643A20004368616E6E656C732088
:1006200064657465637465643A20002028446973C6
:1006300061626C656429002028456E61626C6564A6
:1006400029004D656368616E6963616C2072656342
:100650006F696C00416972736F6674004D65636801
:10066000616E6963616C2042617272656C3A200050
:1006700020284D31290020284D32290020284229E8
:100680000042617272656C20456C65766174696FB9
:100690006E3A20200020284D30290020284D312995
:1006A00000202841290054757272657420526F74BD
:1006B0006174696F6E3A202020004472697665206B
:1006C0004D6F746F72733A202020202020004D4F10
:1006D000544F522054595045530054616E6B20289A
:1006E00054616D69796120444D44290054616E6BF9
:1006F0002028444B4C4D2047656172626F78290079
:100700004361720048616C66747261636B0054618E
:100710006E6B00554E4B4E4F574E00596573004E51
:100720006F002900252C20446563656C6572617437
:10073000696F6E20666163746F72200020284B69B8
:10074000636B6261636B2073706565642000547233
:1007500061636B205265636F696C20456E61626CEA
:1007600065643A202020004E2F4120666F7220766B
:10077000656869636C652074797065005475726E84
:10078000204D6F64653A202020202020202020204A
:1007900020202020004E2F4120666F722076656851
:1007A00069636C65207479706500596573202854FD
:1007B000616D69796129002500202D20004E657545
:1007C0007472616C205475726E20416C6C6F776529
:1007D000643A2020200020736563005472616E73B8
:1007E0006D697373696F6E2044656C61793A20207E
:1007F000202020002073656300456E67696E6520C8
:1008000050617573652054696D653A202020202061
:100810002000207365630053686966742054696D15
:10082000653A202020202020202020202020200089
:100830004175746F6D61746963004D616E75616CB3
:10084000005472616E736D697373696F6E205479B1
:1008500070653A2020202020200025005965732053
:100860002D2000526576657273652053706565644E
:10087000204C696D697465643A2020002500596533
:1008800073202D2000466F7277617264205370656B
:100890006564204C696D697465643A202000206DA0
:1008A00073290025207468726F74746C6520666FFC
:1008B0007220002028004D6F746F72204E7564679F
:1008C0006520456E61626C65643A20202020002915
:1008D000004E6F6E65004E6F6E65002C2050726585
:1008E0007365743A20002900202841646A75737486
:1008F000656420746F200020284C6576656C3A2072
:1009000000446563656C2052616D7020456E6162C4
:100910006C65643A20202020200029004E6F6E650F
:10092000004E6F6E65002C205072657365743A201E
:10093000002900202841646A757374656420746F0F
:10094000200020284C6576656C3A20004163636581
:100950006C2052616D7020456E61626C65643A2056
:1009600020202020004163746976652044726976F6
:10097000696E672050726F66696C653A2000566533
:100980006869636C6520547970653A2020202020C6
:100990002020202020200044524956452053455411
:1009A00054494E47530020736563005265636F6975
:1009B0006C2064656C61793A202020202020202062
:1009C00020202020202020202020200025005965E4
:1009D00073202D200042617272656C20456C657633
:1009E0006174696F6E205370656564204C696D6930
:1009F0007465643A20002500596573202D20005449
:100A0000757272657420526F746174696F6E2053D1
:100A100070656564204C696D697465643A202000D6
:100A20005455525245542053455454494E4753004F
:100A3000556E6B6E6F776E004865617679004D6517
:100A40006469756D004C6967687400437573746FF1
:100A50006D00556E6B6E6F776E004E6F6E65004F5A
:100A600070656E2050616E7A65720054616D6979AF
:100A70006120537065630020736563207265636F46
:100A8000766572792900207365632072656C6F61E9
:100A9000642C2000204D4720686974732C200020AE
:100AA00063616E6E6F6E20686974732C200028007D
:100AB00057656967687420436C6173733A2020201E
:100AC00020200044616D6167652050726F66696C1B
:100AD000653A202020005965732028004163636532
:100AE0007074204D472044616D6167653A2000595C
:100AF000657320280053656E64204D4720495220BD
:100B0000436F64653A2020004E2F410052657061AA
:100B1000697265642062793A202020202020004EEE
:100B20002F41004869742050726F746F636F6C209E
:100B3000323A20202000290020285465616D2000D1
:100B4000466972652050726F746F636F6C3A202033
:100B5000202000466972652050726F746F636F6C5D
:100B60003A2020202000497320526570616972206C
:100B700054616E6B3F202020004952202620546192
:100B80006E6B20426174746C696E67204469736196
:100B9000626C656400424154544C4520494E464FB6
:100BA00000554E4B4E4F574E0042656E6564696E60
:100BB0006920544253204D6963726F004265696534
:100BC000722055534D2D52432D3200546169676593
:100BD0006E20536F756E642043617264004F7065C0
:100BE0006E2050616E7A657220536F756E6420437B
:100BF0006172640042656E6564696E692054425397
:100C0000204D696E6900536F756E64206361726474
:100C10003A2000534F554E44204341524400486906
:100C20006C6C205068797369637320456E61626CE7
:100C300065643A202020202020202020004261727C
:100C400072656C2053746162696C697A6174696F52
:100C50006E20456E61626C65643A200053656E7368
:100C60006F722064657465637465643A2020202087
:100C7000202020202020202020205965730053654B
:100C80006E736F72206E6F74206465746563746533
:100C9000642100494E45525449414C204D45415331
:100CA0005552454D454E5420554E495400556E6B96
:100CB0006E6F776E0042617272656C20456C65766E
:100CC0006174696F6E20436F6D6D616E6400547561
:100CD0007272657420526F746174696F6E20436F15
:100CE0006D6D616E64005374656572696E67204353
:100CF0006F6D6D616E640056656869636C65205345
:100D00007065656400456E67696E65205370656542
:100D100064005468726F74746C6520436F6D6D610C
:100D20006E64005370656564206465637265617309
:100D300065732062656C6F77200053706565642071
:100D4000696E637265617365732061626F76652099
:100D50000043616E6E6F6E2052656C6F61646564F6
:100D60000056656869636C652044657374726F79B9
:100D700065640043616E6E6F6E2048697400427254
:100D8000616B6573204170706C69656400566172B7
:100D90006961626C6500290020286F662000506F31
:100DA000732000417578204368616E6E656C200089
:100DB0005661726961626C65004F6E004F66660035
:100DC0004200410045787465726E616C20496E7016
:100DD00075742000070809090B0C0C0B0C0C5475DA
:100DE0007272657420537469636B202D2000467500
:100DF0006E6374696F6E202300202D3E20002073E7
:100E0000656300547572726574206D6F76656D65EB
:100E10006E742064656C61793A2020004E6F6E65B7
:100E20000059657300547572726574207374696338
:100E30006B2066756E6374696F6E733A2000465559
:100E40004E4354494F4E2054524947474552530050
:100E500076206375746F666629002028004C56431F
:100E600020456E61626C65643A20202020202000BD
:100E70007600566F6C746167653A20202020202030
:100E80002020202000596573004E6F004261747469
:100E90006572792044657465637465643A20004224
:100EA0004154544552590053657269616C20332096
:100EB000547820426175643A2020004175782053AF
:100EC000657269616C20426175643A202020004D92
:100ED0006F746F722053657269616C204261756432
:100EE0003A20005553422053657269616C2042617B
:100EF00075643A2020200042415544205241544517
:100F00005300524144494F204641494C53414645C4
:100F100000526164696F205265616479202D200060
:100F200052657665727365643A2020004D617820C1
:100F300050756C73653A20004D696E2050756C7366
:100F4000653A2000456E642056616C7565730045F6
:100F50006E64205265636F696C20536572766F20F2
:100F6000536574757000456E6420526F74617469C6
:100F70006F6E20536572766F2053657475700045EF
:100F80006E6420456C65766174696F6E205365727E
:100F9000766F20536574757000536572766F207597
:100FA0006E2D726576657273656400536572766F37
:100FB000207265766572736564005265766572733A
:100FC00065643A2020004D61782050756C73653A55
:100FD00020004D696E2050756C73653A2000537483
:100FE0006172742056616C75657300494E56414CB0
:100FF000494420534552564F2E204E4F20534554BE
:1010000055502E005365747570205265636F696C7E
:1010100020536572766F0053657475702054757235
:1010200072657420526F746174696F6E2050616EC6
:1010300020536572766F0053657475702054757215
:1010400072657420456C65766174696F6E205061BD
:101050006E20536572766F00557365722046756E0B
:101060006374696F6E203100557365722046756E2A
:101070006374696F6E203200466F7277617264200C
:1010800047656172004E65757472616C20476561D9
:101090007200526576657273652047656172005310
:1010A000657420416363656C2052616D70204C65EE
:1010B00076656C3A200053657420446563656C2046
:1010C00052616D70204C6576656C3A2000536574F2
:1010D0002042617272656C2053656E736974697623
:1010E0006974793A20005365742048696C6C205308
:1010F000656E73697469766974793A2000416E612E
:101100006C6F6720557365722046756E6374696FE6
:101110006E2031202D2000416E616C6F6720557369
:1011200065722046756E6374696F6E2032202D20C3
:10113000002D00202D20002000545255450046412E
:101140004C534500250057616974696E6720666FCE
:101150007220726164696F2E2E2E2000456E6769C1
:101160006E65204175746F2053687574646F776E77
:1011700000456E67616765205472616E736D6973B7
:1011800073696F6E00446973656E676167652054AB
:1011900072616E736D697373696F6E00536574204D
:1011A0005475726E204D6F64653A2031005365743A
:1011B000205475726E204D6F64653A20320053657D
:1011C00074205475726E204D6F64653A203300456B
:1011D0006E61626C65204E65757472616C20547529
:1011E000726E730044697361626C65204E6575743C
:1011F00072616C205475726E730042617272656C1C
:101200002053746162696C697A6174696F6E3A2007
:101210005475726E6564204F4E0042617272656C47
:101220002053746162696C697A6174696F6E3A20E7
:101230005475726E6564204F46460048696C6C2098
:10124000506879736963733A205475726E656420CF
:101250004F4E0048696C6C20506879736963733A2B
:10126000205475726E6564204F464600494F2050E9
:101270006F72742041204F7574707574202D204F4B
:101280006E00494F20506F72742041204F7574706A
:101290007574202D204F666600494F20506F727480
:1012A0002042204F7574707574202D204F6E0049B8
:1012B0004F20506F72742042204F757470757420E7
:1012C0002D204F6666004C56432045786974202DCA
:1012D00020566F6C7461676520526573746F726518
:1012E00064007629004C5643207468726573686FF9
:1012F0006C642072656163686564212028004C6914
:101300006768742031204F6E004C69676874203123
:10131000204F6666004C696768742032204F6E006B
:101320004C696768742032204F666600326E642014
:101330004D472053746F7000326E64204D47205328
:10134000746172740052756E6E696E67204C6967C5
:10135000687473204F6E0052756E6E696E67204C14
:101360006967687473204F666600417578204F7511
:1013700074707574204F6E00417578204F757470CD
:101380007574204F66660053746F70205265766FD7
:101390006C76696E6720417578204C6967687400C7
:1013A00053746F7020417578204F75747075742078
:1013B000426C696E6B696E6700417578204F757479
:1013C000707574205072657365742044696D0053A4
:1013D0007461727420417578204F75747075742033
:1013E000426C696E6B696E67000000210024002763
:1013F000002A002D00300033000101000004010725
:10140000010A0100002200250028002B002E0031D7
:1014100000340002010000050108010B010000205A
:10142000002300260029002C002F003200000100BC
:10143000000301060109010505050507050808085F
:1014400008020202020A0A08080404040401010155
:10145000010101010103030303030303030407075D
:10146000070C0C0C0C0C0C0C0C02020202060606FB
:1014700006060606060B0B0B0B0B0B0B0B010210E3
:10148000202008081020401020408002010201089E
:10149000040201010204081020408080402010084E
:1014A00004020180040201804020100804020108A7
:1014B0000402010102040810204080010204081007
:1014C00020408000000A0B02090C0D0E08070304DF
:1014D000010000000000000000000000000000000B
:1014E00000000000000000000000000000000012EA
:1014F00011100000000000000000000000000000CB
:10150000000000000000000000556E6B6E6F776EEB
:101510000044657461636865642F4E4100526563E1
:101520006F696C20536572766F0050616E20536551
:1015300072766F00536572766F2F455343004F6E7E
:10154000626F617264204D6F746F722044726976AD
:101550006572004F70656E2050616E7A657220531F
:10156000636F75742053657269616C204553430045
:101570005361626572746F6F74682053657269613C
:101580006C00506F6C6F6C752053657269616C00F4
:10159000536572766F203100536572766F2032008A
:1015A000536572766F203300536572766F20340076
:1015B000536572766F203500536572766F20360062
:1015C000536572766F203700536572766F2038004E
:1015D000401F7017D007A00FA00FDC05D007C4096B
:1015E00010278813983A10276C023A026C023A02CC
:1015F0006C023A026C02B036384A5C121C255C124E
:101600005C121C255C12BC7FC7F2C07887A5B7C5E9
:10161000A00F8813B80B401FB80BB80B7017401FF2
:101620005374617274205265766F6C76696E6720B0
:10163000417578204C6967687400536F6E79005269
:10164000435441204D616368696E652047756E00A3
:10165000436C61726B204D616368696E65204775EC
:101660006E005243544120526570616972004942D4
:10167000552052657061697200436C61726B205233
:101680006570616972004F70656E50616E7A657247
:1016900000567354616E6B00464F56005461696783
:1016A000656E0048656E67204C6F6E670054616D13
:1016B00069796120312F33350054616D697961207A
:1016C000322D53686F740054616D69796100556EF5
:1016D0006B6E6F776E003A2000426974200047619C
:1016E000703A2000466972652043616E6E6F6E002D
:1016F0004669726520526570616972205369676E30
:10170000616C00416972736F6674202D204D616EAB
:1017100075616C2054726967676572004D65636816
:10172000616E6963616C205265636F696C202D2066
:101730004D616E75616C2054726967676572005304
:101740006572766F205265636F696C202D204D6144
:101750006E75616C205472696767657200486967CD
:101760006820496E74656E7369747920466C617384
:101770006820556E6974202D204D616E75616C2056
:1017800054726967676572004D47205374617274C3
:10179000004D472053746F7000417578204F757469
:1017A00070757420466C61736865640041757820BB
:1017B0004F757470757420496E7665727365204636
:1017C0006C61736865640053746F70204175782094
:1017D0004F757470757420426C696E6B696E67002A
:1017E00053746F70205265766F6C76696E67204116
:1017F0007578204C6967687400536D6F6B65722053
:10180000656E61626C656400536D6F6B6572206418
:10181000697361626C65640053657420766F6C75E2
:101820006D653A2000202D2053746172742052653A
:1018300070656174696E6700202D2053746F7000AD
:101840005573657220536F756E6420004169727321
:101850006F6674202D20456E61626C6564004D6575
:101860006368616E6963616C205265636F696C20A7
:101870002D20456E61626C656400416972736F660C
:1018800074202D2044697361626C6564004D65634A
:1018900068616E6963616C205265636F696C202DAD
:1018A0002044697361626C656400436F6D6D7320E1
:1018B0006368616E67656420746F2055534200430E
:1018C0006F6D6D73206368616E67656420746F204F
:1018D00053657269616C20310044726976696E6784
:1018E0002050726F66696C652073657420746F2078
:1018F00023005475726E20456E67696E65204F6EC9
:10190000004D616E75616C207472616E736D6973E8
:1019100073696F6E202D2070757420696E206E655E
:10192000757472616C2067656172206265666F72A2
:1019300065207374617274696E6720656E67696E85
:101940006521005475726E20456E67696E65204F83
:101950006666002900202D2041646A7573746564F1
:1019600020746F2000202853656E7369746976694E
:10197000747920002900202D2041646A75737465F4
:101980006420746F2000202853656E736974697633
:101990006974792000009EA311241FBECFEFD1E20D
:1019A000DEBFCDBF00E00CBF15E0A0E0B2E0E7EB8A
:1019B000F7E801E00BBF02C007900D92AC3EB10703
:1019C000D9F723E1ACEEB5E001C01D92AD30B2070E
:1019D000E1F71CE0CCECDCE000E006C02197010957
:1019E000802FFE010E949AAECB3CD10780E0080711
:1019F000A9F70E94F3910C945AB40C9400002F9212
:101A00003F924F925F926F927F928F929F92AF928E
:101A1000BF92CF92DF92EF92FF920F931F93CF93DB
:101A2000DF93CDB7DEB7AB970FB6F894DEBF0FBE2E
:101A3000CDBF87EC91E00E94E5B36637794181051F
:101A4000910519F00E94687B08C04BEC51E060E002
:101A500070E08FE89EE00E94CDB340E052EC61E080
:101A600070E08CEC98E00E94E56640913610509151
:101A7000371060913810709139108FE298E00E9411
:101A8000E56640913A1050913B1060913C10709186
:101A90003D1082E997E00E94E56640913E1050912A
:101AA0003F10609140107091411085EF96E00E94C8
:101AB000E5668EE29DE09093EF058093EE058FEE54
:101AC0009AE09093ED058093EC058CEC98E0909370
:101AD00008138093071310928A0D1092330D109201
:101AE000300D1092320D1092310D11E010937812DA
:101AF0000E94D28F8091551080939806109297067D
:101B00001092800082E0809381008FE286BB109269
:101B10006F0010928500109284009BE29093A000C9
:101B200099E09093A10089BB109272001092A500D9
:101B30001092A4001092A9001092A8001092AB007D
:101B40001092AA001092AD001092AC0099EA909306
:101B50002001109321018ABB10927300109225017D
:101B600010922401109229011092280110922B0149
:101B700010922A0110922D0110922C0180912C0FAD
:101B800090912D0F8093280690932906813071F44F
:101B900061E08FE30E94474D80912906882319F068
:101BA0000E9445420FC00E942E420CC0809129061F
:101BB000882311F062E001C060E08FE30E94474D8E
:101BC0000E940B4580912E0F90912F0F80932F062E
:101BD00090933006813071F461E08EE30E94474DAE
:101BE00080913006882319F00E9416420FC00E948F
:101BF000FF410CC080913006882311F062E001C0E3
:101C000060E08EE30E94474D0E94D84460E085E486
:101C10000E94474D62E08CE30E94474D62E08BE3F7
:101C20000E94474D62E080E40E94474D62E081E4FB
:101C30000E94474D62E082E40E94474D62E081E2EB
:101C40000E94474D62E084E40E94474D61E089E3D1
:101C50000E94474D61E08AE30E94474D0E94073889
:101C60000E948E4361E085E30E94474D61E085E07C
:101C70000E94474D61E070E085E00E94834D61E085
:101C800084E00E94474D61E087E00E94474D61E09B
:101C900089E20E94184D61E089E20E94474D6A9AEC
:101CA00060E085E30E94184D60E085E00E94184DD9
:101CB00060E084E00E94184D60E087E00E94184DCB
:101CC000729861E088E00E94474D80E090E09C01BE
:101CD0002157314FF901ED55FF4F40814F3629F41F
:101CE000329720813181232B31F403968837910577
:101CF00071F760E001C061E088E00E94184D61E08A
:101D00008BE20E94474D60E08BE20E94184D0E94DA
:101D10008E430E9431778091DF0A813009F06CC0D8
:101D20008091E20A9091E30AA091E40AB091E50A59
:101D30004091E60A5091E70A6091E80A7091E90A39
:101D4000841B950BA60BB70B84379E40A105B105EC
:101D500000F30E94687B80919506909196060E9400
:101D6000FE4A80919506909196060E94FE4A0E9436
:101D70002A4167E173E080919506909196060E9452
:101D8000A04901E010E00E940B380E948E436EEEE5
:101D900072E080E090E00E94694E64E173E080911F
:101DA0009506909196060E94A0490E9407380E94CD
:101DB0008A430530110531F064EF71E080E090E076
:101DC0000E94694E0F5F1F4F06301105E1F68091AA
:101DD0009506909196060E94FE4A0E942A418091A3
:101DE0009506909196060E94FE4A809195069091E4
:101DF00096060E94FE4A02C081118BCF80916F002F
:101E0000826080936F00809184009091850080565D
:101E1000904F909389008093880081E080935B0DC0
:101E200080935E0D8093610D8093640D8093700D9F
:101E30008093730D9091E40F9150953040F0809312
:101E4000E40F61E070E085E591E00E949776909163
:101E5000E40F2DEF290F8091A80F233008F012C254
:101E60008A3079F03CF4883009F45DC0893009F497
:101E7000C1C1B7C18B3009F49EC08C3009F4E0C0F9
:101E8000B0C183E290E00E94B4AFFC0188E090E032
:101E9000938382838824839499249A94958284825C
:101EA000AA24AA94B12CB782A68211861086108E1D
:101EB00003E8702E718E82E9C82E87E0D82ED38E6B
:101EC000C28E9AE6E92E92E0F92EF182E0820AE3D0
:101ED00010E111A300A312A2F0938706E0938606F7
:101EE000CF010E94965983E290E00E94B4AFFC01BA
:101EF00089E090E09383828395828482B782A68270
:101F000011861086108E718ED38EC28EF182E08281
:101F100011A300A312A2F0938506E0938406CF01DB
:101F20000E94965929C380E290E00E94B4AFFC0160
:101F300088E090E0938382838824839499249A9400
:101F400095828482AA24AA94B12CB782A682118693
:101F50001086108E7AE0D72ED18EA2E9EA2EA7E065
:101F6000FA2EF38EE28E02E512E011830083F093E5
:101F70008706E0938606CF010E94FF5880E290E03A
:101F80000E94B4AFFC0189E090E093838283958244
:101F90008482B782A68211861086108ED18EF38E2F
:101FA000E28E11830083F0938506E0938406CF01CF
:101FB0000E94FF58E1C289E190E00E94B4AFFC01A9
:101FC00088E090E093838283CC24C394DD24DA9468
:101FD000D582C482EE24EA94F12CF782E68211863F
:101FE0001086108E06E412E011830083F0938706BA
:101FF000E0938606CF010E949B581092700D80914D
:10200000E40F843009F0B8C289E190E00E94B4AFD7
:10201000FC0189E090E093838283D582C482F782B9
:10202000E68211861086108E11830083F093850658
:10203000E0938406CF010E949B581092730D9CC2BE
:10204000943009F063C089E190E00E94B4AF8C0144
:10205000BEE98B2EB5E09B2EDC0111969C928E92F0
:1020600087E090E013969C938E931297AA24A394F2
:10207000BB24BA941596BC92AE921497CC24CA9401
:10208000D12C1796DC92CE92169719961C921E921E
:10209000189758961C92C8010E944B612EEFE22EB1
:1020A00023E0F22EF801F182E0821093870600937C
:1020B0008606C8010E94478310925B0D89E190E07B
:1020C0000E94B4AF8C01DC0111969C928E9286E046
:1020D00090E013969C938E9312971596BC92AE92B5
:1020E00014971796DC92CE92169719961C921E9210
:1020F000189758961C92C8010E944B61F801F18212
:10210000E082109385060093840665C085E0809385
:10211000E40F89E190E00E94B4AF8C017EE9872E44
:1021200075E0972EDC0111969C928E9287E090E0EC
:1021300013969C938E931297AA24A394BB24BA94CB
:102140001596BC92AE921497CC24CA94D12C1796B3
:10215000DC92CE92169719961C921E92189758965A
:102160001C92C8010E944B61AEEFEA2EA3E0FA2E4A
:10217000F801F182E0821093850600938406C8017D
:102180000E94478310925B0D89E190E00E94B4AFFA
:102190008C01DC0111969C928E9286E090E0139661
:1021A0009C938E9312971596BC92AE9214971796A5
:1021B000DC92CE92169719961C921E9218975896FA
:1021C0001C92C8010E944B61F801F182E0821093D9
:1021D000870600938606C8010E94478310925E0D11
:1021E000CBC189E08093A80F69E070E089E191E0BC
:1021F0000E94977680E290E00E94B4AFFC0188E0F4
:1022000090E0938382838824839499249A9495827E
:102210008482AA24AA94B12CB782A6821186108641
:10222000108E50E8D52ED18E62E9E62E67E0F62EAC
:10223000F38EE28E0EE512E011830083F0938706A1
:10224000E0938606CF010E94415980E290E00E940F
:10225000B4AFFC0189E090E093838283958284820D
:10226000B782A68211861086108ED18EF38EE28EF2
:1022700011830083F0938506E0938406CF010E94CA
:1022800041597AC18A3009F470C03CF4883009F4AD
:10229000B6C0893009F419C10FC18B3009F4D2C01E
:1022A0008C3009F009C189E190E00E94B4AF8C0143
:1022B0008EE9882E85E0982ED80111969C928E92F8
:1022C00087E090E013969C938E931297AA24A39490
:1022D000BB24BA941596BC92AE921497CC24CA949F
:1022E000D12C1796DC92CE92169719961C921E92BC
:1022F000189758961C92C8010E944B613EEFE32E3E
:1023000033E0F32EF801F182E08210938906009306
:10231000880689E190E00E94B4AF8C01DC0111963F
:102320009C928E9286E090E013969C938E931297E7
:102330001596BC92AE9214971796DC92CE92169791
:1023400019961C921E92189758961C92C8010E94CA
:102350004B61F801F182E08210938B0600938A06AC
:1023600010925B0D10925E0DF1C083E290E00E942E
:10237000B4AFFC017090F00F88E090E0938382830B
:102380008824839499249A9495828482AA24AA9476
:10239000B12CB782A68211861086108E83E8682E33
:1023A000618E92E9C92E97E0D92ED38EC28E2AE68D
:1023B000E22E22E0F22EF182E0820AE310E111A384
:1023C00000A372A2F0938906E093880683E290E06E
:1023D0000E94B4AFFC0189E090E0938382839582F0
:1023E0008482B782A68211861086108E618ED38E6B
:1023F000C28EF182E08211A300A372A2A3C080E288
:1024000090E00E94B4AFFC0188E090E09383828367
:102410008824839499249A9495828482AA24AA94E5
:10242000B12CB782A68211861086108EAAE0DA2E11
:10243000D18EB2E9EB2EB7E0FB2EF38EE28E02E5F1
:1024400012E065C089E190E00E94B4AFFC0188E031
:1024500090E093838283CC24C394DD24DA94D582E4
:10246000C482EE24EA94F12CF782E682118610866B
:10247000108E06E412E011830083F0938906E09346
:10248000880689E190E00E94B4AFFC0189E090E009
:1024900093838283D582C482F782E6821186108676
:1024A000108E11830083F0938B06E0938A061092BE
:1024B000700D1092730D4AC089E08093A80F69E0F7
:1024C00070E089E191E00E94977680E290E00E94BE
:1024D000B4AFFC0188E090E09383828388248394E6
:1024E00099249A9495828482AA24AA94B12CB782C2
:1024F000A68211861086108EB0E8DB2ED18E12E9EE
:10250000E12E17E0F12EF38EE28E0EE512E011833C
:102510000083F0938906E093880680E290E00E94B1
:10252000B4AFFC0189E090E093838283958284823A
:10253000B782A68211861086108ED18EF38EE28E1F
:1025400011830083F0938B06E0938A0680918A06BC
:1025500090918B06DC01ED91FC910280F381E02DDE
:1025600019958091880690918906DC01ED91FC9186
:102570000280F381E02D19958091E40F833039F0CA
:10258000823009F059C08091A80F8C3059F189E14F
:1025900090E00E94B4AF8C018EE995E0F801918340
:1025A000808386E090E09383828381E09FEF958330
:1025B00084838FEF90E09783868311861086108E38
:1025C000C8010E944B618EEF93E0D8018D939C93DC
:1025D0001093820600938106C8010E9447831092DF
:1025E0005E0D2AC089E190E00E94B4AF8C018EE9B3
:1025F00095E0F8019183808384E090E09383828367
:1026000081E09FEF958384838FEF90E097838683AB
:1026100011861086108EC8010E944B618EEF93E0E8
:10262000D8018D939C931093820600938106C80174
:102630000E9447831092640DE091A90F8E2FEE0F38
:10264000990BAA0BBB0BFC013897E830F10508F099
:10265000B9C08827EE58FF4F8F4F0C949AAE83E293
:1026600090E00E94B4AFFC0188E090E09383828305
:1026700081E09FEF958384838FEF90E0978386833B
:1026800011861086108E84E8818F82E997E0938FFF
:10269000828F8AE692E0918380838AE390E191A31E
:1026A00080A312A21EC080E290E00E94B4AFFC01A1
:1026B00088E090E09383828381E09FEF9583848319
:1026C0008FEF90E09783868311861086108E87E8BF
:1026D000818F82E997E0938F828F8EE592E09183DC
:1026E0008083F0939006E0938F069CC080E290E098
:1026F0000E94B4AFFC0188E090E09383828381E084
:102700009FEF958384838FEF90E097838683118674
:102710001086108E8DE0818F82E997E0938F828FF3
:1027200082E592E0DCCF89E190E00E94B4AFFC0149
:1027300088E090E09383828381E09FEF9583848398
:102740008FEF90E09783868311861086108E86E443
:1027500092E091838083F0939006E0938F0610922D
:10276000700D60C08CE190E00E94B4AF8C018EE9E6
:1027700095E0F8019183808385E090E093838283E4
:1027800081E09FEF958384838FEF90E0978386832A
:1027900011861086108EC8010E944B6182E995E077
:1027A00038C089E190E00E94B4AFFC01138212822C
:1027B000158214821782168211861086108E82E28C
:1027C00092E08DCF8CE08093A90F6CE070E08AE1FD
:1027D00091E00E94977689E190E00E94B4AF8C016D
:1027E0008EE995E0F8019183808385E090E0938302
:1027F000828381E09FEF958384838FEF90E09783BE
:10280000868311861086108EC8010E944B618EEF60
:1028100093E0D8018D939C931093900600938F06BC
:102820001092610D80918F0690919006DC01ED91E0
:10283000FC910280F381E02D19958091B10F8436CF
:1028400058F4853608F084E664E6681B80918F06AC
:10285000909190060E941E5A8091A90F8C50823050
:10286000A8F46091B20F7091B30F85E00E94965F5B
:102870006091B40F7091B50F85E00E947B5F8091ED
:10288000B60FE0918F06F0919006808F2091AA0FED
:10289000822F022E000C990BAA0BBB0BFC01389760
:1028A000E830F10508F088C08827E658FF4F8F4FC1
:1028B0000C949AAE83E290E00E94B4AFFC0189E0F0
:1028C00090E09383828381E09FEF958384838FEFF1
:1028D00090E09783868311861086108E84E8818F1E
:1028E00082E997E0938F828F8AE692E091838083DA
:1028F0008AE390E191A380A312A259C080E290E004
:102900000E94B4AFFC0189E090E09383828381E070
:102910009FEF958384838FEF90E097838683118662
:102920001086108E87E8818F82E997E0938F828FDF
:102930008EE592E03AC080E290E00E94B4AFFC01E4
:1029400089E090E09383828381E09FEF9583848385
:102950008FEF90E09783868311861086108E8DE02E
:10296000818F82E997E0938F828F82E592E01DC08C
:102970008091E40F823011F00C94FB218091A80F1C
:102980008C3011F00C94FB211FC089E190E00E9473
:10299000B4AFFC0113821282158214821782168250
:1029A00011861086108E82E292E091838083F093EC
:1029B0009406E093930660C08091E40F823061F545
:1029C0008091A80F8C3041F58BE08093AA0F6BE0CB
:1029D00070E08BE191E00E94977689E190E00E949F
:1029E000B4AFFC0189E090E09383828381E09FEFA4
:1029F000958384838FEF90E097838683118610867A
:102A0000108E86E492E091838083F0939406E093A5
:102A100093061092730D30C08CE08093AA0F6CE087
:102A200070E08BE191E00E94977689E190E00E944E
:102A3000B4AF8C018EE995E0F8019183808384E046
:102A400090E09383828381E09FEF958384838FEF6F
:102A500090E09783868311861086108EC8010E94AD
:102A60004B618EEF93E0D8018D939C931093940665
:102A7000009393061092640D8091930690919406B2
:102A8000DC01ED91FC910280F381E02D199580919C
:102A9000B00F843658F4853608F084E664E6681B87
:102AA00080919306909194060E941E5A8091AA0FDD
:102AB0008C50823000F56091AB0F7091AC0F84E0C8
:102AC0000E94965F6091AD0F7091AE0F84E00E94FE
:102AD0007B5F8091AF0FE0919306F0919406808F19
:102AE0008091AA0F8D3039F48091AF0FE091400DA5
:102AF000F091410D808F8EE190E00E94B4AF8C0187
:102B0000D090BB0FA090BF0FB090C00F8090BD0FB2
:102B10009090BE0F8EE995E0F8019183808383E069
:102B200090E09383828381E09FEF95838483EE24FA
:102B3000EA94F12CF782E68211861086108EC80185
:102B40000E944B618AE392E0D80111969C938E9388
:102B50005A969C928E9259975C96BC92AE925B97D5
:102B60005D96DC9210936D1200936C126091C10F10
:102B70007091C20F83E00E94965F6091C30F7091C5
:102B8000C40F83E00E947B5F8091BB0FE0916C12C9
:102B9000F0916D12808F8091BB0F0E9462768091C0
:102BA0006C1290916D12DC01ED91FC910280F38129
:102BB000E02D19958091C50F882339F185E290E0C9
:102BC0000E94B4AFFC018091CA0F9091CB0F20916D
:102BD000C80F3091C90F4091C60F5091C70F68E0E0
:102BE00070E07383628315821482F782E682118615
:102BF0001086108E6EE272E071836083528F418F77
:102C0000348F238F968F858F22C085E290E00E94BB
:102C1000B4AFFC018091C80F9091C90F2091C60FED
:102C20003091C70F48E050E05383428315821482ED
:102C3000F782E68211861086108E4EE252E05183B2
:102C40004083328F218F948F838FF68EE58EF093A1
:102C50000D06E0930C0680910C0690910D060E94E3
:102C600043848091700D8823F9F089E190E00E94FF
:102C7000B4AFFC0188E090E09383828315821482D4
:102C80008FEF93E0978386838FEF91E09187808722
:102C9000108E86E492E091838083F0936F0DE09331
:102CA0006E0DCF010E949B588091730D8823F9F01F
:102CB00089E190E00E94B4AFFC0189E090E0938349
:102CC0008283158214828FEF93E0978386838FEF40
:102CD00091E091878087108E86E492E091838083D3
:102CE000F093720DE093710DCF010E949B5880EF1D
:102CF0009AE09093DB0D8093DA0D1091F30F209101
:102D0000F20F8091E10F9091E30F3091E40F309337
:102D1000F0059093F3058093F40530E0AFEFB0E059
:102D20000E944BB424E630E040E050E00E94FDB346
:102D30002093E112612F70E080E090E00E94B8B231
:102D400023EC34E64AEA5AE30E9419B32AE939E946
:102D500049E55FE30E94AFAE6093DB127093DC1233
:102D60008093DD129093DE121092950010929400E1
:102D7000109290008CE08093910084EF90E090930B
:102D800099008093980011E018BB82E08093710055
:102D9000809100020E946D8F809195069091960619
:102DA000209198064091DD0F5091DE0F5093421212
:102DB000409341122093F7129093F6128093F512EC
:102DC0001092F505109343128091FA0F853040F070
:102DD0001092FA0F60E070E08BE691E00E94977627
:102DE0001091FA0F123009F441C0F0F4112309F4E4
:102DF00063C0113009F058C08CE090E00E94B4AF7D
:102E00002AE333E0FC013183208322E937E0338772
:102E1000228790939206809391061093670D1093EA
:102E20006A0D10936D0D67C0133009F45EC0143045
:102E3000D9F585E090E00E94B4AF8C012CE933E035
:102E4000FC0121933193CF0141E060EF7AE00E94D1
:102E50002D6886E792E0D8018D939C93109392069B
:102E60000093910681E08093670D41C086E090E079
:102E70000E94B4AF28ED32E0DC012D933C93909397
:102E80009206809391068FB7F8942CED35E030933D
:102E90007D1120937C11109282118FBF81E080936D
:102EA000670D80936A0D25C01092FA0F60E070E004
:102EB0008BE691E00E94977685E090E00E94B4AFA7
:102EC0008C012CE933E0FC0121933193CF0140E0E8
:102ED00060EF7AE00E942D6886E792E0D8018D933A
:102EE0009C9310939206009391061092670D109296
:102EF0006A0D10926D0D8091910690919206DC0101
:102F0000ED91FC910190F081E02D199580915B0D80
:102F100081111FC080915E0D81111BC08091610DD8
:102F2000811117C08091640D811113C08091670DCC
:102F300081110FC080916A0D81110BC080916D0DC0
:102F4000811107C081E00E94CE8F882309F419C344
:102F500011C3A12CB12C812C1DA2412C512C612C10
:102F6000712C912C0EE915E0EE24EA94A3E0FA2EE0
:102F7000CC24CA94DD24D39482E9282E85E0382E0F
:102F8000C5018157914FFC01ED55FF4FE081EE23C4
:102F900009F4E7C2DC01AF55BF4F8D919C91892B9D
:102FA00009F4DFC28E2F90E0FC01F797EB32F105B8
:102FB00008F0D7C28827EE57FF4F8F4F0C949AAE78
:102FC00080915B0D882309F4CCC29110CAC289E1BB
:102FD00090E00E94B4AF9C01FC011183008387E064
:102FE00090E09383828315821482F782E682D186F1
:102FF000C086108EC9012AA73BA70E944B612AA553
:103000003BA5EEEFF3E0D901ED93FC9330934C0D2B
:1030100020934B0DC9010E9447837DC180915E0DB5
:10302000882309F49EC271109CC289E190E00E943D
:10303000B4AF9C01DC0111961C930E93E6E0F0E026
:103040001396FC93EE93129715961C921E9214976A
:103050001796FC92EE9216971996DC92CE921897DC
:1030600058961C922AA73BA70E944B612AA53BA514
:10307000EEEFF3E0D901ED93FC9330934E0D2093E6
:103080004D0DC9010E94478374C18091610D882351
:1030900009F467C2611065C289E190E00E94B4AF93
:1030A0009C01DC0111961C930E93E5E0F0E0139671
:1030B000FC93EE93129715961C921E9214971796F6
:1030C000FC92EE9216971996DC92CE92189758962B
:1030D0001C922AA73BA70E944B612AA53BA5EEEFB5
:1030E000F3E0D901ED93FC933093500D20934F0DF5
:1030F000C9010E9447836BC18091640D882309F444
:1031000030C251102EC289E190E00E94B4AF9C0100
:10311000DC0111961C930E93E4E0F0E01396FC930F
:10312000EE93129715961C921E9214971796FC9286
:10313000EE9216971996DC92CE92189758961C929A
:103140002AA73BA70E944B612AA53BA5EEEFF3E01F
:10315000D901ED93FC933093520D2093510DC90189
:103160000E94478362C18091670D882309F4F9C1E9
:103170004110F7C189E190E00E94B4AF9C01DC01ED
:1031800011961C930E93E2E0F0E01396FC93EE93FD
:10319000129715961C921E9214971796FC92EE9217
:1031A00016971996DC92CE92189758961C922AA7D9
:1031B0003BA70E944B612AA53BA5EEEFF3E0D901A6
:1031C000ED93FC933093540D2093530DC9010E944D
:1031D000478359C180916A0D882309F4C2C12DA18A
:1031E0002111BFC189E190E00E94B4AF9C01DC01D4
:1031F00011961C930E93E1E0F0E01396FC93EE938E
:10320000129715961C921E9214971796FC92EE92A6
:1032100016971996DC92CE92189758961C922AA768
:103220003BA70E944B612AA53BA5EEEFF3E0D90135
:10323000ED93FC933093560D2093550DC9010E94D8
:10324000478359C180916D0D882309F48AC181108B
:1032500088C189E190E00E94B4AF9C01DC01119625
:103260001C930E9313961C921E92129715961C9205
:103270001E9214971796FC92EE9216971996DC926E
:10328000CE92189758961C922AA73BA70E944B6192
:103290002AA53BA58EEF93E0F901918380833093BB
:1032A000580D2093570DC9010E94478358C1809142
:1032B0005B0D882309F455C1911053C18CE190E056
:1032C0000E94B4AF9C01DC0111961C930E93E7E0C1
:1032D000F0E01396FC93EE93129715961C921E92B3
:1032E00014971796FC92EE9216971996DC92CE924E
:1032F000189758961C922AA73BA70E944B612AA5B3
:103300003BA5D9012D923C9230935A0D2093590D33
:10331000C9010E94BE839924939423C180915E0DBC
:10332000882309F41EC171101CC18CE190E00E9439
:10333000B4AF9C01FC011183008386E090E093838D
:10334000828315821482F782E682D186C086108E2F
:10335000C9012AA73BA70E944B612AA53BA5D90119
:103360002D923C9230935D0D20935C0DC9010E941B
:10337000BE8377247394F5C08091610D882309F48E
:10338000F0C06110EEC08CE190E00E94B4AF9C01EF
:10339000FC011183008385E090E093838283158292
:1033A0001482F782E682D186C086108EC9012AA7D0
:1033B0003BA70E944B612AA53BA5D9012D923C92C7
:1033C0003093600D20935F0DC9010E94BE83662477
:1033D0006394C7C08091640D882309F4C2C0511062
:1033E000C0C08CE190E00E94B4AF9C01FC0111834D
:1033F000008384E090E09383828315821482F782B5
:10340000E682D186C086108EC9012AA73BA70E94FA
:103410004B612AA53BA5D9012D923C923093630DB7
:103420002093620DC9010E94BE835524539499C014
:103430008091670D882309F494C0411092C08CE1FB
:1034400090E00E94B4AF9C01FC011183008382E0F4
:1034500090E09383828315821482F782E682D1867C
:10346000C086108EC9012AA73BA70E944B612AA5DE
:103470003BA5D9012D923C923093660D2093650DAA
:10348000C9010E94BE83442443946BC080916A0D9D
:10349000882309F466C02DA1211163C08CE190E05E
:1034A0000E94B4AF9C01DC0111961C930E93E1E0E5
:1034B000F0E01396FC93EE93129715961C921E92D1
:1034C00014971796FC92EE9216971996DC92CE926C
:1034D000189758961C922AA73BA70E944B612AA5D1
:1034E0003BA5D9012D923C923093690D2093680D34
:1034F000C9010E94BE8321E02DA333C080916D0DD0
:10350000882379F181102DC08CE190E00E94B4AF46
:103510009C01DC0111961C930E9313961C921E9233
:10352000129715961C921E9214971796FC92EE9283
:1035300016971996DC92CE92189758961C922AA745
:103540003BA70E944B612AA53BA5F901318220824D
:1035500030936C0D20936B0DC9010E94BE838824AB
:103560008394F3E0AF0EB11C28E7A216B10409F072
:1035700007CDE8CC82E00E94CE8F882311F01FA2F5
:1035800016C081E00E94CE8F882329F082E00E943D
:10359000B28F81118EC78CE30E94F04C892B09F009
:1035A00079C78CE30E94F04C892B09F079C786E03B
:1035B000E8E2F0E1DE01549601900D928A95E1F780
:1035C000B0902110009131101091221070912310B1
:1035D00060912410509125104091261030912710B1
:1035E00020912E1080912F1090913010E091910633
:1035F000F0919206FEA3EDA3A0916C12B0916D1212
:10360000B9A7A8A79090541060904F10E090481070
:10361000F09049108090521070905110C090B90FE6
:10362000D090BA0F5090BC0F4090B70F3090B80FA9
:10363000BFA1BB8BBA8E0B8F1C8F7D8F6E8F5F8F60
:1036400048A339A32AA39CA38BA3F2E1AF2EFE01CA
:103650007396DE01119601900D92AA94E1F7E0EFC6
:10366000FAE0F093FE05E093FD05EFA1E983B8864B
:1036700009871A877B876C875D874E873F87288BF2
:103680009A8B898B82E1FE013196AEE0B6E0019023
:103690000D928A95E1F73092430E4092440E50927B
:1036A000420ED0928A0EC092890E60926E12709273
:1036B0008E0E80928D0EF0928C0EE0928B0E909278
:1036C0003F0E88A599A59093410E8093400E8DA141
:1036D0009EA1909300068093FF0587E08093ED09FB
:1036E0001092EE0961E00E94474D0E940677109209
:1036F000EF091092F00980911906811102C0109211
:103700001A0690911506911105C0811103C01092FF
:10371000C60AA3C081E08093C60A0091C10A109135
:10372000C20A8091510A60E00E94474DD801ED9194
:10373000FC910190F081E02DC801199580910E0651
:10374000882359F1813071F08330C1F488E293E22B
:103750009093100680930F0689E08093130680E112
:1037600097E217C088EB9BE09093100680930F06BA
:1037700083E08093130688E99AE30BC088E893E11D
:103780009093100680930F0686E08093130680EED8
:103790009EE290931206809311068091150688236D
:1037A000E9F1809119066091130670E08823C9F051
:1037B00080911B068823A9F080E090E00E94B8B2B7
:1037C0009B01AC0160E070E088EC92E40E9413AFD2
:1037D000609301067093020680930306909304069B
:1037E00025C080E090E00E94B8B29B01AC0160E08F
:1037F00070E088EC92E40E9413AF6093010670932E
:10380000020680930306909304061092F805109226
:10381000F9051092FA051092FB051FC010920106DF
:10382000109202061092030610920406609114068C
:1038300070E080E090E00E94B8B29B01AC0160E0D3
:1038400070E088EC92E40E9413AF6093F8057093E7
:10385000F9058093FA059093FB0510920B061092E0
:1038600005061092FC0510920606109207061092AB
:103870000806109209060E942B6B6E98769AEE98B5
:1038800080916A008F7C80936A008091440E882327
:1038900021F080916A00806203C080916A00806399
:1038A00080936A00EE980E94CB6D80E090E040E04B
:1038B0009C012157314FF901ED55FF4F50815523A0
:1038C00031F0329720813181232B09F04F5F03962D
:1038D0008837910569F740932206A1E3B6E020E01E
:1038E00030E083E2282E80E4382E90EA492E9EE3D1
:1038F000592E46EC642E4EE3742E56E8852E5EE378
:10390000952E63E9A62E6EE3B62E4BE850E40AE24C
:1039100010E47CE2E72E70E4F72EEEEBCE2EE0E42E
:10392000DE2EC9018157914FFC01ED55FF4F60819B
:10393000662309F45CC38F559F4FFC018081918100
:10394000892B09F454C370E0FB013197EF38F1057E
:1039500008F04DC38827E355FF4F8F4F0C949AAE64
:1039600084E996E811969C938E9341C382E996E888
:1039700011969C938E933BC386E492E811969C9398
:103980008E9335C38FE392E811969C938E932FC349
:103990008DE392E811969C938E9329C388EC91E86D
:1039A00011969C938E9323C38AEC91E811969C9375
:1039B0008E931DC38BEA91E811969C938E9317C347
:1039C00087E991E811969C938E9311C388E891E85A
:1039D00011969C938E930BC38CE291E811969C9365
:1039E0008E9305C381E090E811969C938E93FFC25D
:1039F0008FE191E811969C938E93F9C281EE90E845
:103A000011969C938E93F3C284E191E811969C9356
:103A10008E93EDC28DE191E811969C938E93E7C24F
:103A200086E191E811969C938E93E1C284E091E83F
:103A300011969C938E93DBC282E091E811969C9341
:103A40008E93D5C280E091E811969C938E93CFC25D
:103A500080EF90E811969C938E93C9C28EEE90E809
:103A600011969C938E93C3C28FED90E811969C9310
:103A70008E93BDC28FEC90E811969C938E93B7C243
:103A80008DEC90E811969C938E93B1C28BEC90E8EC
:103A900011969C938E93ABC281E89FE711969C93FD
:103AA0008E93A5C28FE79FE711969C938E939FC23A
:103AB0008DE79FE711969C938E9399C28BE891E4D2
:103AC00011969C938E9393C289EC90E811969C93E7
:103AD0008E938DC289EB90E811969C938E9387C24A
:103AE0008AE990E811969C938E9381C28BE790E8C7
:103AF00011969C938E937BC289E790E811969C93D4
:103B00008E9375C28AE490E811969C938E936FC24F
:103B10008BEC9FE711969C938E9369C281ED9FE792
:103B200011969C938E9363C285EA96E811969C93B6
:103B30008E935DC28AEC9FE711969C938E9357C239
:103B400089EC9FE711969C938E9351C283EA9FE77D
:103B500011969C938E934BC287EC9FE711969C9392
:103B60008E9345C285EB9FE711969C938E933FC23F
:103B700081EA9FE711969C938E9339C285EC9FE76B
:103B800011969C938E9333C283EB9FE711969C937F
:103B90008E932DC28FE99FE711969C938E9327C237
:103BA00083EC9FE711969C938E9321C281EB9FE754
:103BB00011969C938E931BC28DE99FE711969C935F
:103BC0008E9315C281EC9FE711969C938E930FC242
:103BD0008FEA9FE711969C938E9309C28BE99FE72A
:103BE00011969C938E9303C28FEB9FE711969C9343
:103BF0008E93FDC18DEA9FE711969C938E93F7C13A
:103C000089E99FE711969C938E93F1C18DEB9FE715
:103C100011969C938E93EBC18BEA9FE711969C9330
:103C20008E93E5C187E99FE711969C938E93DFC140
:103C30008BEB9FE711969C938E93D9C189EA9FE7FE
:103C400011969C938E93D3C185E99FE711969C931F
:103C50008E93CDC189EB9FE711969C938E93C7C13C
:103C600087EA9FE711969C938E93C1C183E99FE7F2
:103C700011969C938E93BBC187EB9FE711969C9303
:103C80008E93B5C185EA9FE711969C938E93AFC141
:103C900081E99FE711969C938E93A9C18CE690E4ED
:103CA00011969C938E93A3C183E690E411969C9306
:103CB0008E939DC182E790E411969C938E9397C159
:103CC00089E690E411969C938E9391C180E690E4EE
:103CD00011969C938E938BC18FE690E411969C93E2
:103CE0008E9385C186E690E411969C938E937FC156
:103CF0008DE590E411969C938E9379C187E69EE3BF
:103D000011969C938E9373C186E69EE311969C93C5
:103D10008E936DC185E69EE311969C938E9367C149
:103D20008AE490E411969C938E9361C187E59EE3AB
:103D300011969C938E935BC186E59EE311969C93AE
:103D40008E9355C185E59EE311969C938E934FC14A
:103D500087E390E411969C938E9349C18BE89FE38F
:103D600011969C938E9343C180E49FE311969C939C
:103D70008E933DC18AEB92E411969C938E9337C14A
:103D800086EA92E411969C938E9331C182E992E483
:103D900011969C938E932BC18AE696E811969C937C
:103DA0008E9325C183E49EE311969C938E931FC14D
:103DB00081E39EE311969C938E9319C18AE79DE35C
:103DC00011969C938E9313C180E39DE311969C936F
:103DD0008E930DC182E59DE311969C938E9307C14E
:103DE00082E49DE311969C938E9301C184E69DE34A
:103DF00011969C938E93FBC088E09DE311969C9353
:103E00008E93F5C088EF9CE311969C938E93EFC040
:103E10008AE19DE311969C938E93E9C084E39FE32E
:103E200011969C938E93E3C088E29FE311969C9336
:103E30008E93DDC08CE19FE311969C938E93D7C047
:103E400080E19FE311969C938E93D1C084E09FE321
:103E500011969C938E93CBC088EF9EE311969C9312
:103E60008E93C5C08CEE9EE311969C938E93BFC03B
:103E700088EF9DE311969C938E93B9C086EE9DE3E7
:103E800011969C938E93B3C084ED9DE311969C9301
:103E90008E93ADC082EC9DE311969C938E93A7C048
:103EA00080EB9DE311969C938E93A1C08EE99DE3D8
:103EB00011969C938E939BC08CE89DE311969C93E6
:103EC0008E9395C085E390E411969C938E938FC05A
:103ED00083E390E411969C938E9389C08EE290E4E4
:103EE00011969C938E9383C01196DC92CE927FC0E4
:103EF0001196FC92EE927BC011961C930E9377C0A4
:103F000085E290E411969C938E9371C011965C9318
:103F10004E936DC01196BC92AE9269C011969C9260
:103F20008E9265C011967C926E9261C011965C92E1
:103F30004E925DC011963C922E9259C0E0E7F2E499
:103F40001196FC93EE9353C08DE592E411969C93E9
:103F50008E934DC0E8E8F2E41196FC93EE9347C0CF
:103F600080E290E411969C938E9341C0EDE1F0E4E1
:103F70001196FC93EE933BC084E190E411969C93E0
:103F80008E9335C0E9E0F0E41196FC93EE932FC0D8
:103F900082E190E411969C938E9329C0EBE0F0E4CB
:103FA0001196FC93EE9323C084E29EE311969C93BA
:103FB0008E931DC0E7E1FEE31196FC93EE9317C0CC
:103FC0008AE09EE311969C938E9311C0E8EFFFE385
:103FD0001196FC93EE930BC087EE9FE311969C9392
:103FE0008E9305C0E6EDFFE31196FC93EE932D5FF3
:103FF0003F4F12962837310509F093CC10922306D3
:1040000080912806811114C080E090E0FC01E05D01
:10401000F04F20813181245631092436310528F0B2
:1040200003968837910591F703C081E080932306BA
:1040300010922A0680912F06811114C080E090E032
:10404000FC01E05DF04F20813181285C310924368C
:10405000310528F003968837910591F703C081E078
:1040600080932A068091910690919206DC01ED9151
:10407000FC91E65BFF4F2091FD0F3091FE0F4091C8
:10408000FB0F5091FC0F0190F081E02D61E019953C
:104090008091910690919206DC01ED91FC91E65B96
:1040A000FF4F20910110309102104091FF0F50916D
:1040B00000100190F081E02D62E019958091910649
:1040C00090919206DC01ED91FC91E65BFF4F20910F
:1040D000051030910610409103105091041001908A
:1040E000F081E02D63E01995809191069091920600
:1040F000DC01ED91FC91E65BFF4F209110103091B7
:10410000111040910E1050910F100190F081E02D90
:1041100064E019958091910690919206DC01ED91F1
:10412000FC91E65BFF4F20911410309115104091E7
:104130001210509113100190F081E02D65E0199557
:104140008091910690919206DC01ED91FC91E65BE5
:10415000FF4F209118103091191040911610509176
:1041600017100190F081E02D66E01995809191067D
:1041700090919206DC01ED91FC91E45BFF4F019080
:10418000F081E02D4091071061E019958091910632
:1041900090919206DC01ED91FC91E45BFF4F019060
:1041A000F081E02D4091081062E019958091910610
:1041B00090919206DC01ED91FC91E45BFF4F019040
:1041C000F081E02D4091091063E0199580919106EE
:1041D00090919206DC01ED91FC91E45BFF4F019020
:1041E000F081E02D40911A1064E0199580919106BC
:1041F00090919206DC01ED91FC91E45BFF4F019000
:10420000F081E02D40911B1065E019958091910699
:1042100090919206DC01ED91FC91E45BFF4F0190DF
:10422000F081E02D40911C1066E019958091910677
:1042300090919206DC01ED91FC9100ACF1ADE02D86
:1042400060910B1019958091910690919206DC0176
:10425000ED91FC9104ACF5ADE02D60912010199525
:104260008091910690919206DC01ED91FC9106A45B
:10427000F7A5E02D60910C10199580919106909111
:104280009206DC01ED91FC9104A8F5A9E02D609166
:104290000D10199580E090E09C012157314FF901F4
:1042A000ED55FF4F4081423731F432972081318103
:1042B000232B09F004C103968837910569F70E9402
:1042C00094878091910690919206DC01ED91FC918A
:1042D000E45AFF4F0190F081E02D40E060911D1005
:1042E00019958091910690919206DC01ED91FC91D7
:1042F000E45AFF4F0190F081E02D41E060911F10E2
:1043000019958091910690919206DC01ED91FC91B6
:10431000E45AFF4F0190F081E02D42E060911E10C1
:1043200019958091F40F882331F08091AA0F8D3078
:1043300011F01092F40F1092F40610927C0D8091FF
:10434000F50F8093F2058091F70F8093F10520918E
:10435000461030E0AFEFB0E00E944BB424E630E00E
:1043600040E050E00E94FDB320937D0D8091451008
:1043700081110E94BA430E94F0370E941A6E6B01AD
:104380007C0110E011110FC080919806882359F02C
:1043900025E73EE340ED57E060E070E080EF9AE013
:1043A0000E94905E11E00E94D785882351F00E9400
:1043B00049370E94F1450E948E430E9464850E9405
:1043C000B7370E948D63029711F00E94CD510E9471
:1043D00063880E948D630297A9F60E941A6EDC0121
:1043E000CB018C199D09AE09BF098C3B9240A105F8
:1043F000B10540F267C02C3011F40C9415158CE116
:1044000090E00E94B4AF8C012EE9622E25E0722E5E
:10441000FC017182608234E0832E912C938282822F
:10442000AA24A394BB24BA94B582A482CC24CA94AF
:10443000D12CD782C68211861086108E0E944B61C5
:1044400062E9E62E65E0F62ED801ED92FC9210931B
:104450009406009393068CE190E00E94B4AF8C0127
:10446000FC017182608293828282B582A482D782AB
:10447000C68211861086108E0E944B61D801ED9283
:10448000FC921093410D0093400DC8010E94BE8321
:104490000C943A1582E00E94CE8F81110DC081C824
:1044A00082E00E94B28F882309F481C8A3E0AFA301
:1044B0007EC881E08FA37BC892E09FA378C80E944A
:1044C0008887FFCE0E9465370E948E438091DA0A6A
:1044D000811102C00E943F780E94626386E30E94BD
:1044E0004A4EBC01990F880B990B61157105810526
:1044F000910511F00E943FB223EF3CE348EE53E0F8
:1045000060E070E080EF9AE0AB960FB6F894DEBF03
:104510000FBECDBFDF91CF911F910F91FF90EF9014
:10452000DF90CF90BF90AF909F908F907F906F90D3
:104530005F904F903F902F900C94905E2F923F92FF
:104540004F925F926F927F928F929F92AF92BF92A3
:10455000CF92DF92EF92FF920F931F93CF93DF934F
:10456000CDB7DEB7E6970FB6F894DEBF0FBECDBF6E
:1045700080919506909196060E94FE4A0E942A41DB
:104580006BE175E080919506909196060E94A04996
:104590006EEC75E0CE0101960E946149009195068E
:1045A00010919606D801ED91FC914D815E81698153
:1045B0007A810280F381E02DC8011995C8010E941B
:1045C000FE4ACE0101960E9431490E946388809183
:1045D000950690919606DC01ED91FC910284F3859D
:1045E000E02D199580919506909196060E94FE4ABD
:1045F0000E942A4160EB75E08091950690919606A5
:104600000E94A049E091DB0AE4300CF0E0E08CE38A
:1046100095E09A83898388E395E09C838B8383E389
:1046200095E09E838D838EE295E098878F83EE0FD1
:10463000FF0B81E090E08C0F9D1FE80FF91F608158
:10464000718180919506909196060E94114B0E946F
:104650002A416AE775E080919506909196060E943E
:10466000114B0E942A416EE675E08091950690916B
:1046700096060E94A049E0915B11F0915C11818146
:104680009281883E934014F40E941A41E0915B119C
:10469000F0915C11618172818091950690919606EE
:1046A0000E94BA7784E00E94277FE0915B11F0912D
:1046B0005C116581768180919506909196060E94A5
:1046C000BA7785E00E94277FE0915B11F0915C1141
:1046D0006381748180919506909196060E94BA77C5
:1046E00084E00E94277FE0915B11F0915C1167816B
:1046F00080919506909196060E94A07788E00E948E
:10470000277FE0915B11F0915C1180850E9406414A
:1047100062E675E080919506909196060E94A04908
:10472000E0916511F091661181819281883E9340FC
:1047300014F40E941A41E0916511F09166116181B3
:10474000728180919506909196060E94BA7784E0D6
:104750000E94277FE0916511F09166116581768155
:1047600080919506909196060E94BA7785E00E9406
:10477000277FE0916511F0916611638174818091CA
:104780009506909196060E94BA7784E00E94277F52
:10479000E0916511F0916611678180919506909185
:1047A00096060E94A07788E00E94277FE09165111D
:1047B000F091661180850E94064166E575E0809162
:1047C0009506909196060E94A049E0916F11F09194
:1047D000701181819281883E934014F40E941A41A5
:1047E000E0916F11F0917011618172818091950655
:1047F000909196060E94BA7784E00E94277FE0910C
:104800006F11F0917011658176818091950690917C
:1048100096060E94BA7785E00E94277FE0916F118B
:10482000F091701163817481809195069091960644
:104830000E94BA7784E00E94277FE0916F11F09187
:104840007011678180919506909196060E94A077DD
:1048500088E00E94277FE0916F11F09170118085B0
:104860000E9406416AE475E0809195069091960653
:104870000E94A049E0917911F0917A118181928191
:10488000883E934014F40E941A41E0917911F0910E
:104890007A116181728180919506909196060E94AD
:1048A000BA7784E00E94277FE0917911F0917A1124
:1048B0006581768180919506909196060E94BA77DF
:1048C00085E00E94277FE0917911F0917A11638150
:1048D000748180919506909196060E94BA7784E043
:1048E0000E94277FE0917911F0917A116781809180
:1048F0009506909196060E94A07788E00E94277FF7
:10490000E0917911F0917A1180850E9406418091A1
:104910009506909196060E94FE4A0E946263C82EF8
:1049200062EE75E080919506909196060E94114B7B
:104930000E942A410AEF10E1E12CF12CD12C570101
:104940002FEFA21AB20AB5018091950690919606B2
:104950000E94BA7749E0E416F10410F48BE001C03C
:104960008AE00E94277FD8012C9180919506909132
:1049700096062223C9F11596ED91FC911697618157
:1049800072810E94BA77D8011596ED91FC91169725
:1049900081819281883E934014F40E941A4184E000
:1049A0000E94277FD8011596ED91FC91169763819F
:1049B000748180919506909196060E94BA7784E062
:1049C0000E94277FD8011596ED91FC9116972781BB
:1049D0008091950690919606222319F06AED75E074
:1049E0000BC063ED75E008C0EC14FD041CF46BEC27
:1049F00075E002C06EEB75E00E94114B095F1F4F1E
:104A00007501BCE0AB16B10409F099CF0E942A41B0
:104A100067E176E080919506909196060E94A04904
:104A20000E946263682F80919506909196060E947D
:104A30004B7663E076E080919506909196060E9411
:104A4000A0496091D80A7091D90A809195069091F9
:104A500096060E94F0770E94638880919506909157
:104A60009606DC01ED91FC910284F385E02D199509
:104A700080919506909196060E94FE4A0E942A41D6
:104A80006EEC76E080919506909196060E94114B0F
:104A90000E942A416AEB76E08091950690919606F5
:104AA0000E94A0498091A80F0E944A5ABC0180919F
:104AB0009506909196060E94114B66EA76E08091E9
:104AC0009506909196060E94A0498091A90F0E9498
:104AD0004A5ABC0180919506909196060E94A04981
:104AE0002091A90F80919506909196062B303CF469
:104AF000293054F4283069F465E976E007C02B309A
:104B000041F461EA76E002C06BE976E00E94114B65
:104B100002C00E94FE4A61E876E08091950690917D
:104B200096060E94A0498091AA0F0E944A5ABC0191
:104B300080919506909196060E94A0492091AA0F17
:104B400080919506909196062B303CF4293054F4D0
:104B5000283069F460E776E007C02B3041F46CE759
:104B600076E002C066E776E00E94114B02C00E9428
:104B7000FE4A6CE576E080919506909196060E943B
:104B8000A0492091B70F8091950690919606222317
:104B900019F064E576E002C062E476E00E94A04984
:104BA0002091430E8091950690919606222319F04C
:104BB00067E376E002C06BE276E00E94A049809154
:104BC0009506909196060E94FE4A0E946388809105
:104BD000950690919606DC01ED91FC910284F38597
:104BE000E02D199580910002823011F40C94C32EAF
:104BF000F090CE0F0091D10F11E080919506909129
:104C000096060E94FE4A0E942A4167E979E0809157
:104C10009506909196060E94114B0E942A416EE7DC
:104C200079E080919506909196060E94A049E091C6
:104C3000E40FE6300CF0E0E083E197E09A838983AB
:104C40008EE097E09C838B8384E097E09E838D8346
:104C500080E097E098878F838CEE96E09A8789872B
:104C60008AED96E09C878B87EE0FFF0B81E090E04A
:104C70008C0F9D1FE80FF91F60817181809195064F
:104C8000909196060E94114B65E679E08091950619
:104C9000909196060E94A04960910002809195062D
:104CA000909196060E944B766CE479E0809195068F
:104CB000909196060E94A0498F2D0E94F140FF20FE
:104CC00009F44BC062E479E08091950690919606D4
:104CD0000E94A0498091950690919606112339F083
:104CE0006091CF0F0E94A0779091CF0F06C0609186
:104CF000D50F0E94A0779091D50F8091D81298136C
:104D00000C94CA2E66E279E0809195069091960601
:104D10000E94A0498091950690919606112339F042
:104D20006091D00F61110CC061E279E006C0609122
:104D3000D60F611105C06CE179E00E94A04905C061
:104D4000062E000C770B0E94BA776AE179E0809119
:104D50009506909196060E94A049809195069091A3
:104D600096060E94FE4A61E079E080919506909156
:104D700096060E94A049802F0E94F140002309F46A
:104D80004BC067EF78E080919506909196060E945F
:104D9000A0498091950690919606112339F0609173
:104DA000D20F0E94A0779091D20F06C06091D80FC9
:104DB0000E94A0779091D80F8091DA1298130C94EA
:104DC000E42E6BED78E080919506909196060E9416
:104DD000A0498091950690919606112339F0609133
:104DE000D30F61110CC066ED78E006C06091D90F59
:104DF000611105C061ED78E00E94A04905C0062E52
:104E0000000C770B0E94BA776FEC78E080919506E2
:104E1000909196060E94A0498091950690919606E1
:104E20000E94FE4A66EB78E0809195069091960686
:104E30000E94A0498091ED0F811103C00E94FF40A4
:104E400035C06BE177E080919506909196060E94BF
:104E5000A04963EB78E080919506909196060E94B8
:104E6000A0496091ED0F80919506909196060E9461
:104E7000A07763EA78E080919506909196060E946B
:104E8000A0494091EE0F5091EF0F60E070E02AE0F2
:104E900080919506909196060E94D9496EE978E036
:104EA00080919506909196060E94114B65E878E0F6
:104EB00080919506909196060E94A0498091E50FF9
:104EC0008436C8F46EE778E0809195069091960656
:104ED0000E94A0496091E50F8091950690919606F9
:104EE0000E94A0776CE778E08091950690919606F5
:104EF0000E94114B03C080E00E94FF4063E678E00F
:104F000080919506909196060E94A0498091E60FA7
:104F10008436C8F46CE578E0809195069091960609
:104F20000E94A0496091E60F8091950690919606A7
:104F30000E94A0776AE578E08091950690919606A8
:104F40000E94114B03C080E00E94FF4061E478E0C2
:104F500080919506909196060E94A04920918E0618
:104F60008091950690919606222319F06AE378E0E5
:104F700002C060E378E00E94114B67E178E0809125
:104F80009506909196060E94A0496091DB0F709162
:104F9000DC0F072E000C880B990B0E94BAB220E0A0
:104FA00030E04AE754E40E9413AFAB01BC0121E0BA
:104FB00080919506909196060E94214A62E178E0E0
:104FC00080919506909196060E94114B69EF77E0CB
:104FD00080919506909196060E94A0496091DD0F00
:104FE0007091DE0F072E000C880B990B0E94BAB24D
:104FF00020E030E04AE754E40E9413AFAB01BC016B
:1050000021E080919506909196060E94214A64EFD6
:1050100077E080919506909196060E94114B6BED7A
:1050200077E080919506909196060E94A049609144
:10503000DF0F7091E00F072E000C880B990B0E9478
:10504000BAB220E030E04AE754E40E9413AFAB016B
:10505000BC0121E080919506909196060E94214A1C
:1050600066ED77E080919506909196060E94114B2F
:105070006DEB77E080919506909196060E94A0498D
:105080009091E40F913011F09430F9F48091E10F98
:105090000E94F1408091E10F882329F169EB77E0CC
:1050A00080919506909196060E94A0496091E20F2A
:1050B00080919506909196060E94A07767EB77E025
:1050C00080919506909196060CC02091950630919E
:1050D0009606953019F46AEA77E002C065E977E050
:1050E000C9010E94A04980919506909196060E9460
:1050F000FE4A6CE777E080919506909196060E94B3
:10510000A0499091E40F2FEF290F8091950690917F
:105110009606223028F46091F3050E944B7604C075
:1051200067E677E00E94114B6EE477E08091950688
:10513000909196060E94A0498091F10F0E94F14043
:105140008091F10F882341F16CE377E0809195061F
:10515000909196060E94A0496091F20F8091950669
:10516000909196060E94A07764E277E08091950680
:10517000909196060E94A0496091F30F8091950648
:10518000909196060E94A07762E277E08091950662
:10519000909196060E94A04980919506909196065E
:1051A0000E94FE4A0E94638880919506909196061F
:1051B000DC01ED91FC910284F385E02D199580913D
:1051C0009506909196060E94FE4A0E942A4160E24E
:1051D0007AE080919506909196060E94114B0E946C
:1051E0002A416FEF79E080919506909196060E9492
:1051F000A0498091B10F8436C8F468EF79E08091BE
:105200009506909196060E94A0496091B10F8091F9
:105210009506909196060E94A07766EF79E08091BE
:105220009506909196060E94114B03C080E00E9463
:10523000FF4065ED79E080919506909196060E9479
:10524000A0498091B00F8436C8F46EEC79E080916B
:105250009506909196060E94A0496091B00F8091AA
:105260009506909196060E94A0776CEC79E080916B
:105270009506909196060E94114B03C080E00E9413
:10528000FF406BEA79E080919506909196060E9426
:10529000A0496091B90F7091BA0F1616170614F550
:1052A0000091950610919606072E000C880B990B1D
:1052B0000E94BAB220E030E04AE754E40E9413AF03
:1052C000AB01BC0122E0C8010E94214AC8010E9432
:1052D000FE4A66EA79E080919506909196060E94D2
:1052E000114B03C080E00E94FF400E9463888091C0
:1052F000950690919606DC01ED91FC910284F38570
:10530000E02D199580919506909196060E94FE4A8F
:105310000E942A4165E97BE080919506909196066E
:105320000E94114B0E942A412091150680919506FA
:1053300090919606222309F4C3C166E67BE00E94A1
:10534000A0490E9403710E94FF400E9403712091B6
:10535000950630919606882389F063E57BE0C901C4
:105360000E94A049809118060E942F7ABC0180916A
:105370009506909196060E94114B4FC060E47BE029
:10538000C9010E94A049809115060E942F7ABC0194
:1053900080919506909196060E94A04980911606EC
:1053A0008823A9F168E37BE08091950690919606A9
:1053B0000E94A049E0911606E4300CF0E0E08DE296
:1053C00093E09A8389838BE293E09C838B8389E2C9
:1053D00093E09E838D8387E293E098878F83EE0F1F
:1053E000FF0B81E090E08C0F9D1FE80FF91F60819B
:1053F000718180919506909196060E94A04966E37E
:105400007BE080919506909196060E94A04980913C
:105410009506909196060E94FE4A63E27BE0809199
:105420009506909196060E94A049809117060091DA
:10543000950610919606882321F00E942F7ABC01D0
:1054400002C06FE17BE0C8010E94114B6CE07BE081
:1054500080919506909196060E94A0498091180629
:105460000091950610919606882321F00E942F7ACC
:10547000BC0102C068E07BE0C8010E94114B65EFEF
:105480007AE080919506909196060E94A0498091BD
:105490001A068823E1F06FEE7AE0809195069091EC
:1054A00096060E94A049809119060E942F7ABC019D
:1054B00080919506909196060E94A04966ED75E050
:1054C00080919506909196060E94014B03C080E062
:1054D0000E94FF406CED7AE08091950690919606CF
:1054E0000E94A04980911B068823E1F066ED7AE0D6
:1054F00080919506909196060E94A0498091190688
:105500000E942F7ABC0180919506909196060E9488
:10551000A04966ED75E080919506909196060E94EF
:10552000014B03C080E00E94FF4063EC7AE0809171
:105530009506909196060E94A049E0911C06E330E2
:105540000CF0E3E08BE69AE09A8389838FE59AE09A
:105550009C838B838AE59AE09E838D8382E59AE023
:1055600098878F83EE0FFF0BA1E0B0E0AC0FBD1F5B
:10557000EA0FFB1F608171818091950690919606DC
:105580000E94114B60EB7AE080919506909196060F
:105590000E94A049E0910E06E4300CF0E4E08BE4B8
:1055A0009AE09A83898385E49AE09C838B838EE3D7
:1055B0009AE09E838D8388E39AE098878F8380E3C7
:1055C0009AE09A878987EE0FFF0B81E090E08C0FBD
:1055D0009D1FE80FF91F6081718180919506909160
:1055E00096060E94114B6EEA7AE0809195069091A2
:1055F00096060E94A04960911306809195069091AD
:1056000096060E94A0776FE97AE0809195069091C6
:1056100096060E94A04980910E06811110C06091EB
:10562000140680919506909196060E94A07764E9F1
:105630007AE080919506909196060E94A04960912B
:105640000F0670911006072E000C880B990B0E9414
:10565000BAB220E030E04AE754E40E9413AFAB0155
:10566000BC0121E080919506909196060E94214A06
:1056700066E87AE080919506909196060E94A0498E
:105680006091110670911206072E000C880B990B81
:105690000E94BAB220E030E04AE754E40E9413AF1F
:1056A000AB01BC0121E080919506909196060E9485
:1056B000214A67E77AE0809195069091960602C0AC
:1056C00069E77BE00E94114B0E94638880919506F8
:1056D00090919606DC01ED91FC910284F385E02D1A
:1056E000199580919506909196060E94FE4A0E9417
:1056F0002A4163E17CE080919506909196060E9494
:10570000114B0E942A4166E07CE0809195069091C1
:1057100096060E94A049E091FA0FE5300CF0E5E012
:1057200084EF9BE09A8389838DED9BE09C838B8340
:105730008BEC9BE09E838D838CEB9BE098878F8323
:1057400089EA9BE09A87898781EA9BE09C878B871F
:10575000EE0FFF0B81E090E08C0F9D1FE80FF91F0B
:105760006081718180919506909196060E94114BFF
:105770000E9463888091950690919606DC01ED91D8
:10578000FC910284F385E02D199580919506909106
:1057900096060E94FE4A0E942A4163E97CE08091BD
:1057A0009506909196060E94114B0E942A412091E5
:1057B000F40680919506909196062223C9F16CE536
:1057C0007CE00E94A04980919506909196060E94E7
:1057D000FE4A6DE37CE080919506909196060E94CA
:1057E000A0498091F40F0E94F1408091F40F811143
:1057F0000E94C59180919506909196060E94FE4A5E
:105800006EE17CE080919506909196060E94A049F9
:105810008091F60F0E94F1408091F60F81110E9455
:10582000979180919506909196060E94FE4A04C039
:105830006EE77CE00E94114B0E9463888091950680
:1058400090919606DC01ED91FC910284F385E02DA8
:10585000199584E499E6A1E0BB278BAB9CABADAB7B
:10586000BEAB80919506909196060E94FE4A0E94DA
:105870002A416EE37EE080919506909196060E9403
:10588000114B0E942A4165E27EE08091950690913D
:1058900096060E94A0492091D60A80919506909183
:1058A0009606222319F061E27EE002C06CE17EE000
:1058B0000E94114B8091D60A882349F163E07EE073
:1058C00080919506909196060E94A0496091F80FEC
:1058D0007091F90F072E000C880B990B0E94BAB239
:1058E00020E030E04AE754E40E9413AFAB01BC0172
:1058F00022E080919506909196060E94214A6EEFD3
:105900007DE080919506909196060E94114B92E35E
:10591000E92E9FE0F92E29E2222E38E1432E3CEFBA
:10592000532E4AE0A42EB12C54E6C52ED12CD7011B
:105930002C91222309F4E5C1F701329700811181EE
:105940000115110509F4DDC184EB98E6A1E0BB2740
:10595000820F911DA11DB11DABBFFC0187913324A6
:105960003394811101C0312C209195063091960617
:10597000C8010197849790F56EED7DE0C9010E9402
:10598000A04909500C3148F4E02FF0E0EE0FFF1F62
:10599000EA5FFB4F6081718102C06DEA7CE080911B
:1059A0009506909196060E94A0490C3130F4E02FA4
:1059B000F0E0E25CFB4F808101C080E090E08C521F
:1059C000924F092E000CAA0BBB0BABBFFC018791B9
:1059D0009EE0981B892F09F036C137C1C801845653
:1059E00091098438934008F03FC064EC7DE0C90120
:1059F0000E94A049C801B6010E9473AE61307105D2
:105A000031F06230710559F460EC7DE002C062EC67
:105A10007DE080919506909196060E94A0490E9493
:105A2000224180909506909096063320B1F0C801EF
:105A30000E94E886811107C06CEB7DE0C4010E94E2
:105A4000A04987E000C1813009F0FFC069EB7DE02B
:105A5000C4010E94A04988E0F6C060EB7DE0C4016B
:105A60000E94A04982E0EFC0C801885E9340803563
:105A7000964408F05AC0C80168EE73E00E9473AE05
:105A80004B0163EA7DE0C9010E94A049FAE08F164C
:105A9000910410F40E941A41B401809195069091EE
:105AA00096060E94BA770E942241609095067090F7
:105AB00096063320A1F1C8010E94E886382E6EE9CF
:105AC0007DE0C3010E94A049632D809195069091CD
:105AD00096060E94A07768E97DE0809195069091F6
:105AE00096060E94A049849CC001859C900D949CC0
:105AF000900D1124800F911FB5010E9487AE77276A
:105B000080919506909196060E94BA7766E97DE0AD
:105B100080919506909196060E94A04996C06DE8E6
:105B20007DE0C3010E94A04946C0C80188539A4441
:105B3000883E934068F509338AE41807D9F058F491
:105B400008331A4409F081C06EE77DE0C9010E9464
:105B5000A0498FE078C00A33BAE41B0791F00B33F9
:105B60001A4409F072C061E57DE0C9010E94A049B4
:105B70008EE069C063E77DE0C9010E94A04983E12E
:105B800062C061E67DE0C9010E94A0498CE05BC073
:105B9000C80180529E44883E934078F400526AE3E4
:105BA0007DE0C9010E94A0490A3010F40E941A4108
:105BB000802F0E94754084E046C0C80188509245FD
:105BC000883E934020F4085063E27DE0EACF013F35
:105BD00085E5180719F462E17DE01CC0023F95E5F8
:105BE000190739F465E07DE0C9010E94A04981E10F
:105BF0002AC0033FA5E51A0739F467EF7CE0C90125
:105C00000E94A04980E11FC0043FB5E51B0739F49D
:105C100066EE7CE0C9010E94A0498DE014C0053FFA
:105C2000E5E51E0739F46EEC7CE0C9010E94A0494D
:105C300086E009C0063F154541F465EB7CE0C901EB
:105C40000E94A04985E00E94277F69EF7DE0809156
:105C50009506909196060E94A0496EEE7DE0809197
:105C60009506909196060E94A049D7016C9170E02C
:105C700080919506909196060E94BA77F7018081EF
:105C80008A3020F482E00E94277F04C0843610F41A
:105C90000E941A410E942241D7014C91249EA001EA
:105CA0001124052E000C660B770B8BA99CA9ADA9BE
:105CB000BEA9480F591F6A1F7B1FDE0111968A017A
:105CC0009B010F5F1F4F2F4F3F4F6BBFFA01879113
:105CD0008D93B901A8018111F2CFBE016F5F7F4F93
:105CE00080919506909196060E94014B80919506B1
:105CF00090919606DC01ED91FC910284F385E02DF4
:105D00001995B3E0EB0EF11CEAEAEE16EFE0FE06A1
:105D100009F00DCE0E9463888091950690919606B9
:105D2000DC01ED91FC910284F385E02D19958091C1
:105D30009506909196060E94FE4A0E942A416FE9BC
:105D40007EE080919506909196060E94114B0E94EC
:105D50002A416CE87EE080919506909196060E941B
:105D6000A0490E94704420E030E040E050E40E94EE
:105D7000B4B2209195063091960687FF3FC069E83E
:105D80007EE0C90159C0F090D40F0091D70F10E008
:105D90000C94FD2563E379E0809195069091960639
:105DA0000E94A0496091D812809195069091960624
:105DB0000E94A07761E379E0809195069091960624
:105DC0000E94A0490C94822668EE78E080919506A6
:105DD000909196060E94A0496091DA1280919506F2
:105DE000909196060E94A07766EE78E080919506E5
:105DF000909196060E94A0490C94E12665E87EE009
:105E0000C9010E94114B62E77EE080919506909156
:105E100096060E94A0490E947044AB01BC0122E09A
:105E200080919506909196060E94214A60E77EE057
:105E300080919506909196060E94114B6DE57EE04B
:105E400080919506909196060E94A04980914210FB
:105E50000E94F14020914210809195069091960603
:105E6000222379F06AE57EE00E94A0490E94667FC5
:105E700060E57EE080919506909196060E94114B18
:105E800002C00E94FE4A0E9463888091950690910C
:105E90009606DC01ED91FC910284F385E02D1995C5
:105EA00080919506909196060E94FE4A0E942A4192
:105EB00067EF7EE080919506909196060E94114BC7
:105EC0000E942A4163EE7EE08091950690919606AD
:105ED0000E94A049409132105091331060913410CB
:105EE0007091351080919506909196060E94A77743
:105EF0006FEC7EE080919506909196060E94A049F5
:105F000040913A1050913B1060913C1070913D10BF
:105F100080919506909196060E94A7776BEB7EE0A4
:105F200080919506909196060E94A0494091361066
:105F3000509137106091381070913910809195060A
:105F4000909196060E94A77767EA7EE08091950679
:105F5000909196060E94A04940913E1050913F10AA
:105F60006091401070914110809195069091960635
:105F70000E94A7770E94638880919506909196066B
:105F8000DC01ED91FC910284F385E02D199580915F
:105F90009506909196060E94FE4A0E942A41E69636
:105FA0000FB6F894DEBF0FBECDBFDF91CF911F912A
:105FB0000F91FF90EF90DF90CF90BF90AF909F90A8
:105FC0008F907F906F905F904F903F902F900895AB
:105FD0002F923F924F925F926F927F928F929F92F9
:105FE000AF92BF92CF92DF92EF92FF920F931F93E7
:105FF000CF93DF93CDB7DEB7C65AD1090FB6F89469
:10600000DEBF0FBECDBFCDB6DEB6CC55DF4F18829A
:10601000C45AD040CD55DF4F1882C35AD04080912A
:10602000340D8A3709F447C0C0F4873709F4D9C260
:1060300038F48F3109F430C5863709F4E2C1F2C56E
:10604000883709F4DDC2893709F0ECC50E944B633B
:106050000E941A6E2B013C0129C08E3709F42EC311
:1060600038F48B3709F4CAC18C3709F4D8C2DAC5C1
:10607000813809F402C5823809F4EDC4803809F08A
:10608000D1C565C40E941A6EDC01CB018419950943
:10609000A609B70980329340A105B10508F007C5EC
:1060A0000E94CD510E944B630E945A580E948D63FA
:1060B000029741F7FCC40E948D63029729F060E0CB
:1060C00084E80E9418918BC18091DB0A823031F004
:1060D000833039F482E080938F0D03C081E0809398
:1060E0000C0E81E080933E0D8E010C551F4F2BE06E
:1060F000AE0144575F4F68E871E90E9495900E9495
:106100006263893058F0015011092BE0AE014F57FE
:106110005F4F68E872E981E00E94959010923D0D12
:10612000772473940E947863882309F43DC119820F
:1061300022961FAE229780913D0D81110EC0BE01A7
:1061400064577F4FCE018F5B9F4F0E94D2B1CC55D9
:10615000DF4F0881C45AD0400FC070923D0DBE0180
:106160006F577F4FCE018F5B9F4F0E94D2B1CD55AD
:10617000DF4F0881C35AD04010913D0DADB6BEB679
:106180008091D70AEDB7FEB722E0829FE019F109AE
:1061900011240FB6F894FEBF0FBEEDBF8DB79EB7AA
:1061A00001967C0166EE75E0CE0183569F4F0E94FA
:1061B00061498091DB0A823089F0833061F181305E
:1061C00009F0A1C04091D70A50E0B7018091E50DD8
:1061D0009091E60D0E94935410E039C02091D70AA7
:1061E00030E05FB7F89440E0842F90E08217930787
:1061F00074F4880F991FF701E80FF91FDC01A5510E
:10620000B24F8D919C91918380834F5FEDCF5FBFA3
:1062100010920B0E1CC02091D70A30E05FB7F894A3
:1062200040E0842F90E08217930774F4880F991F41
:10623000F701E80FF91FDC01AB56B24F8D919C912D
:10624000918380834F5FEDCF5FBF1092E20D6DE2CF
:1062500070E0CE0183569F4F0E9490482091D70A4C
:10626000293048F0112321F0113021F418E004C046
:1062700028E001C020E010E0121758F5F701E10F07
:10628000F11DE10FF11D608171814AE0CE01895657
:106290009F4FCB55DF4F2883C55AD0400E943649C7
:1062A000BE0169567F4FCE0183569F4F0E94B7486B
:1062B000CE0189569F4F0E943149CE0183569F4F90
:1062C0000E945C891F5FCB55DF4F2881C55AD040A3
:1062D000D3CF40E450E0BE016F5F7F4FCE018356C5
:1062E0009F4F0E945389CF55DF4F1881C15AD0402C
:1062F000CE0183569F4F0E9431490FB6F894BEBE1F
:106300000FBEADBE0BC0CE0183569F4F0E943149D8
:106310000FB6F894BEBE0FBEADBE10E0BE016F5FFB
:106320007F4FCE018F5B9F4F0E94D2B1010F10E0D3
:10633000E1E4F0E0EC0FFD1FE00FF11F1082BE0161
:106340006F5B7F4F80910713909108130E94C4499F
:10635000B801CE018F5B9F4F0E947758BC0180919E
:106360000713909108130E94BA776AE0809107138F
:10637000909108130E9499498091071390910813F6
:10638000DC01ED91FC910284F385E02D19950E94CA
:106390006263893048F080913D0D811103C0709295
:1063A0003D0D02C010923D0D0E944B630E945A5851
:1063B0000E94658481110CDE8091330D81110FC024
:1063C00080913E0D882359F080918A0D811107C07C
:1063D0008091310D9091320D0A970CF4A3CE8091EB
:1063E000DB0A823039F0833009F01CC481E08093ED
:1063F0008F0D18C481E080930C0E14C410923E0DD2
:1064000048C31091370D8FEF810F853028F060E081
:1064100089E80E94189106C4133079F018F41230FC
:10642000F9F004C0143079F0153099F040E6442EAC
:1064300049E0542E612C712C19C0412C3BE4532EA1
:10644000612C712C13C0412C26E9522E612C712C29
:106450000DC0412C92EC592E66246394712C06C019
:1064600080E8482E85E2582E612C712C00E0E12E48
:10647000F12C5701BFE8AB0EB11C1501E89427F8C9
:106480003324E6E9EE0EF11CE894E7F8FF2402302D
:1064900091F018F4013051F004C0033089F0043059
:1064A000A1F040E659E060E070E013C040E855E23A
:1064B00060E070E00EC040E05BE460E070E009C0C6
:1064C00040E056E960E070E004C040E052EC61E07A
:1064D00070E082E997E00E94E56682E997E00E9419
:1064E000B5470E941A6E4B015C01F2E38F0E911CBE
:1064F000A11CB11C0E941A580E941A6E68157905D9
:106500008A059B05B8F360E870E082E997E00E9495
:1065100056866FE070E082E997E00E945686612F10
:1065200082E997E00E946F47B10182E997E00E94FB
:1065300056860E941A6E4B015C012AE0820E911C65
:10654000A11CB11C0E941A580E941A6E6815790588
:106550008A059B05B8F367E870E082E997E00E943E
:1065600056866FE070E082E997E00E945686612FC0
:1065700082E997E00E946F47B70182E997E00E94A5
:10658000568682E997E00E94B5470E941A6E4B0139
:106590005C013EE5830E31E0931EA11CB11C0E94FC
:1065A0001A580E941A6E681579058A059B05B8F37A
:1065B0000F5F053009F06BCFB301A20182E997E0CC
:1065C0000E94E56640923A1050923B1060923C1057
:1065D00070923D10B301A2018BEA91E00E948F8975
:1065E00058C283E090E00E94B4AF2AE0DC012C9313
:1065F00022E937E012963C932E9311976AE00CC083
:1066000083E090E00E94B4AF2DE0FC01208322E9FA
:1066100037E0328321836DE00E94F1533AC240910A
:10662000370D5091380D0091390D10913A0D609150
:10663000350D7091360DCE010196CB55DF4F488355
:10664000C55AD040CA55DF4F5883C65AD0400E9421
:10665000DD7DCB55DF4F4881C55AD040CA55DF4F4D
:106660005881C65AD040892BE9F08D81873050F48B
:10667000853080F48130B0F0642F8B819C810E9442
:1066800025780DC0893070F4B8018B819C810E94FF
:106690008F8905C0BA018B819C810E9497760E94E8
:1066A000949104C061E085E80E9418918091300DBA
:1066B0008111B8C281E08093300DB4C2B090350D25
:1066C000E090360DC956DF4F1882C759D04066EEAC
:1066D00075E0CE018F579F4F0E9461496B2D7E2D33
:1066E000CE0184579F4F0E94DD7D892B09F4C9C0DC
:1066F000C057DF4FE881C059D0404E2F50E0FA011B
:106700003197E830F10508F0BCC08827E45CFE4F03
:106710008F4F0C949AAEC257DF4F88819981CE5823
:10672000D0400E94DDB323961FAE1EAE2397259660
:106730001FAE1EAE259727961FAE1EAE27974AE0C6
:10674000BE016F5F7F4F90E03EC0C257DF4F888130
:106750009981CE58D0400E94DDB3682F880F770B07
:106760004AE00AC0C257DF4F88819981CE58D04095
:106770000E94EAB34AE0BC01CE0101960E9436496C
:10678000BE016F5F7F4FCE018F579F4F0E945748CA
:10679000CE01019663C0C257DF4F88819981CE58E0
:1067A000D0400E94EAB323961FAE1EAE23972596D3
:1067B0001FAE1EAE259727961FAE1EAE27974AE046
:1067C000BE016F5F7F4F0E948BB235C0C257DF4F53
:1067D00088819981CE58D0400E94E5B323961FAEA0
:1067E0001EAE239725961FAE1EAE259727961FAE89
:1067F0001EAE27972AE0AE014F5F5F4F0E945CB24A
:106800001AC0C257DF4F88819981CE58D0400E946C
:10681000E5B323961FAE1EAE239725961FAE1EAE80
:10682000259727961FAE1EAE27972AE0AE014F5F31
:106830005F4F0E946AB2BE016F5F7F4FCE018F5BD8
:106840009F4F0E941149BE016F5B7F4FCE018F5752
:106850009F4F0E945748CE018F5B9F4F0E94314946
:106860004BE050E0BE016F5B7F4FCE018F579F4FD3
:106870000E945389CB57DF4FF880C558D04011E0B4
:1068800002C0F12C10E0CE018F579F4F0E9431497A
:10689000112309F4BCCD8E0109561F4F20E4AE012F
:1068A0004F5F5F4F68E87B2D8E2D0E949590BE0153
:1068B0006F5B7F4FCE0101960E94D2B1C956DF4F68
:1068C0008881C759D040F80E81E08F0DC956DF4F3F
:1068D0008883C759D040E1E0F0E0EC0FFD1FEF0DD9
:1068E000F11D9CE79083E1E0F0E0EC0FFD1FE80F65
:1068F000F11D1082BE016F5F7F4F80910713909151
:1069000008130E94C449C956DF4F6881C759D04057
:1069100070E0CE0101960E947758BC018091071368
:10692000909108130E94BA776AE0809107139091C2
:1069300008130E9499498091071390910813DC0174
:10694000ED91FC910284F385E02D19956BC1809146
:10695000350D9091360D8038910509F063C18E0197
:1069600004571F4F20E4AE014F5F5F4F68E870E8A7
:1069700080E00E9495906EEC75E0CE018F579F4F9E
:106980000E946149CE018F579F4F0E945C89C45776
:10699000DF4F2881CC58D040CB57DF4F8881998179
:1069A000C558D040820F911DC457DF4F8883CC5803
:1069B000D04022961FAE22974BE050E0BE016F5BA5
:1069C0007F4FCE018F579F4F0E94C379BE016F5BEF
:1069D0007F4FCE0101960E94D2B1C457DF4F88810C
:1069E000CC58D040E1E0F0E0EC0FFD1FE80FF11DC6
:1069F0001082BE016F5F7F4F809107139091081343
:106A00000E94C449C457DF4F6881CC58D04070E021
:106A1000CE0101960E947758BC0180910713909196
:106A200008130E94BA776AE08091071390910813C7
:106A30000E9499498091071390910813DC01ED9110
:106A4000FC910284F385E02D1995CE018F579F4F5D
:106A50000E943149E7C08091350D9091360D823802
:106A6000910509F0DFC08E0104571F4F20E4AE01ED
:106A70004F5F5F4F68E872E87BCF8091350D909152
:106A8000360D8138910509F0CDC080913E0D811100
:106A9000C9C00E949491C6C08091350D9091360D69
:106AA0004F9709F0BFC081E08093330DBBC00E94B7
:106AB0008D63029719F060E084E8ABCC8091DA0A2C
:106AC000811102C00E943F780E946263F82E66EE38
:106AD00075E0CE0184579F4F0E946149C956DF4F30
:106AE0001882C759D0408E0109561F4F20E4AE01CD
:106AF0004F5F5F4F68E879E780E00E949590CF573D
:106B0000DF4F19821882C158D040CD57DF4F19820C
:106B10001882C358D040CB57DF4F19821882C5580E
:106B2000D0406F2D70E080E090E02AE0AE014F5B36
:106B30005F4F0E945CB2BE016F5B7F4FCE018F57EB
:106B40009F4F0E941149BE016F577F4FCE0184575E
:106B50009F4F0E945748CE018F579F4F0E94314947
:106B60004BE050E0BE016F5B7F4FCE0184579F4FDB
:106B70000E94C379C057DF4F1881C059D040BE0171
:106B80006F5B7F4FCE0101960E94D2B1C956DF4F95
:106B90008881C759D040810F91E0980FC956DF4FC7
:106BA0009883C759D040E1E0F0E0EC0FFD1FE80FFB
:106BB000F11D8CE78083E1E0F0E0EC0FFD1FE90FB1
:106BC000F11D1082BE016F5F7F4F8091071390917E
:106BD00008130E94C449C956DF4F6881C759D04085
:106BE00070E0CE0101960E947758BC018091071396
:106BF000909108130E94BA776AE0809107139091F0
:106C000008130E9499498091071390910813DC01A1
:106C1000ED91FC910284F385E02D1995CE01845706
:106C20009F4F16CF0FB6F894DEBE0FBECDBECA552D
:106C3000DF4F0FB6F894DEBF0FBECDBFDF91CF910F
:106C40001F910F91FF90EF90DF90CF90BF90AF908A
:106C50009F908F907F906F905F904F903F902F907C
:106C600008950F931F93CF93DF938C01C1E0D0E081
:106C70000C171D07ACF00E948E4364E670E080E0C4
:106C800090E00E94694E0E948A43C017D10734F4F5
:106C90006AE570E080E090E00E94694E2196E8CFBE
:106CA000DF91CF911F910F91089583E090E0D9CFAC
:106CB00082E090E0D6CF81E090E0D3CF60E089E33E
:106CC0000E94184D60E08AE30E94184D60E085E361
:106CD0000E94184D60E085E00E94184D60E084E05D
:106CE0000E94184D60E087E00E94184D7298089548
:106CF000CF93C0910B026C2F89E30E94184D81E065
:106D0000C8276C2F8AE30E94184DC0930B02CF91C5
:106D10000895CF93DF93C0910A026C2F89E30E94FC
:106D2000184DD1E0DC276D2F8AE30E94184D6C2F9F
:106D300085E30E94184D6D2F85E00E94184D6D2F40
:106D400084E00E94184D6C2F87E00E94184DCC23E0
:106D500011F0729801C0729A90910A0281E089271D
:106D600080930A02DF91CF910895CF93DF938091B2
:106D70004A0D81110DC01092490D1092480D81E00D
:106D800090E09093470D8093460D80934A0D36C056
:106D90008091480D9091490D863191057CF18F3895
:106DA000910534F48091460D9091470D019609C0EC
:106DB0008D3521E0920754F48091460D9091470D56
:106DC00002969093470D8093460D18C0863222E0BC
:106DD000920734F48091460D9091470D0496F1CFBF
:106DE000883E93403CF48091460D9091470D8A5B1C
:106DF0009F4FE7CF1092470D1092460D8ADFC0914A
:106E0000480DD091490DC93E83E0D80754F0109247
:106E10004A0D54DF2DE237E348EE53E060E070E0C6
:106E200007C025EB36E3AE010D2E000C660B770B89
:106E300080EF9AE00E94905E9093450D8093440D00
:106E40008091460D9091470D8C0F9D1F9093490D99
:106E50008093480DDF91CF910895CF93DF93809178
:106E60009A06882319F0DF91CF917FCFC091440D0E
:106E7000D091450DBE0180EF9AE00E94295E8823E3
:106E800029F0BE0180EF9AE00E94415EDF91CF9130
:106E900015CFCF93DF93C091420DD091430DBE012A
:106EA00080EF9AE00E94295E882361F0BE0180EFA6
:106EB0009AE00E94415E1092430D1092420DDF91C4
:106EC000CF91FCCEDF91CF910895CF93DF93CDB7D3
:106ED000DEB728970FB6F894DEBF0FBECDBF809106
:106EE0003F0D8823D9F110923F0DD3DF81E08093CD
:106EF000030280919806882389F161E17FE0809107
:106F00009506909196060E94A049E091DB0AE43034
:106F10000CF0E0E08CE395E09A83898388E395E0C8
:106F20009C838B8383E395E09E838D838EE295E043
:106F300098878F83EE0FFF0BEC0FFD1F618172812D
:106F4000809195069091960628960FB6F894DEBF2C
:106F50000FBECDBFDF91CF910C94114B28960FB689
:106F6000F894DEBF0FBECDBFDF91CF910895609141
:106F7000420D7091430D80EF9AE00E94295E8111CD
:106F80002EC060E089E30E94184D60E08AE30E9411
:106F9000184D60E085E30E94184D60E085E00E9496
:106FA000184D60E084E00E94184D60E087E00E9488
:106FB000184D729880915010882319F029E836E313
:106FC00002C028E736E342E350E060E070E080EF83
:106FD0009AE00E94985E9093430D8093420D08952D
:106FE00080913F0D811112C00E94F14581E0809394
:106FF0003F0DBDDF80919706882341F062E07FE07E
:1070000080919506909196060C94114B089560E03E
:107010008AE30C94184D61E08AE30C94184D0F93A9
:107020001F93CF93DF938C01C1E0D0E00C171D07B5
:107030009CF0F1DF64E670E080E090E00E94694E31
:10704000E6DFC017D10734F46AE570E080E090E035
:107050000E94694E2196EACFDF91CF911F910F9147
:1070600008952F923F924F925F926F927F928F92EC
:107070009F92AF92BF92CF92DF92EF92FF920F93C7
:107080001F93CF93DF9300D0CDB7DEB75C010E9492
:10709000F145BDDF0E948E43809195069091960642
:1070A0000E94FE4A0E942A4124E0A216B10409F47B
:1070B00048C085E0A816B10409F479C0A3E0AA1677
:1070C000B10409F0B1C08CE190E00E94B4AF9B83A1
:1070D0008A838EE995E0EA81FB8191838083B38284
:1070E000A28281E09FEF958384838FEF90E0978366
:1070F000868311861086108ECF010E944B6182E933
:1071000095E0AA81BB818D939C93E0916C12F091E4
:107110006D12D08C0091BF111091C011169507957A
:10712000E090BD11F090BE11F694E79464E070E138
:1071300080919506909196060E94114B22242394EB
:1071400090C08CE190E00E94B4AF9B838A838EE96B
:1071500095E0EA81FB8191838083B382A28281E002
:107160009FEF958384838FEF90E0978386831186CA
:107170001086108ECF010E944B6182E995E0AA81B2
:10718000BB818D939C93E0919306F0919406D08CF3
:107190000091D4111091D51116950795E090D21158
:1071A000F090D311F694E79467E370E135C08CE179
:1071B00090E00E94B4AF9B838A838EE995E0EA81D8
:1071C000FB8191838083B382A28281E09FEF9583CC
:1071D00084838FEF90E09783868311861086108ECC
:1071E000CF010E944B6182E995E0AA81BB818D931A
:1071F0009C93E0918F06F0919006D08C0091E9115C
:107200001091EA1116950795E090E711F090E811BA
:10721000F694E79467E170E1809195069091960667
:107220000E94114B212C1DC06BEE7FE080919506D2
:10723000909196060F900F900F90DF91CF911F9134
:107240000F91FF90EF90DF90CF90BF90AF909F9005
:107250008F907F906F905F904F903F902F900C9405
:10726000114BF8D76EED7FE08091950690919606D0
:107270000E94114B62ED7FE08091950690919606F9
:107280000E94A049B80180919506909196060E94AF
:10729000F07766EC7FE080919506909196060E94CB
:1072A000A049B70180919506909196060E94F077CB
:1072B0006AEB7FE080919506909196060E94A04926
:1072C0008D2DA4D780919506909196060E94FE4A36
:1072D000AA81BB81ED91FC9111970280F381E02D91
:1072E000CD011995CA2C8A2D0E9468608D3D95406C
:1072F000A8F464E378E08A2D0E946060EA81FB8153
:10730000F78AE68AB70182810E9478606CED75E0A9
:107310008A2D0E946460DD20C1F01AC064E873E029
:107320008A2D0E946460AA81BB8157961C930E939C
:107330005697B80112968C910E9478606CED75E0BA
:107340008A2D0E946060DD2019F09924939401C079
:10735000912C33243394812C21E029830E94B25450
:1073600080916811882359F1AA81BB81ED91FC912C
:10737000119760916D1170916E110190F081E02D67
:10738000CD0119958C2D0E9468608D3DB5E09B075D
:107390005CF48438E3E09E0784F08C018D3D9540D9
:1073A00074F00CED15E00BC07C01853398403CF087
:1073B00064E3E62E68E0F62E02C004E813E02981BB
:1073C00021111FC080915E118823C9F1E0916511E0
:1073D000F091661185819681409161115091621101
:1073E0009C0121533109421753074CF1C196841770
:1073F00095072CF10E941A6E641575058605970590
:10740000F0F080915E118823C1F04091611150919C
:107410006211E0916511F0916611858196819C0160
:10742000285C3109421753072CF088539F4F84176B
:1074300095071CF481E0982605C021E02983882067
:1074400009F47CC0992009F445C0DD20F9F064E816
:1074500073E08C2D0E946460222009F458C0609172
:10746000BF0F7091C00F41E08C2D0E941F600E94E1
:107470006388AA81BB8112968C910E94686008176C
:107480001907ACF38C2D0E94F15F41C064E378E0F2
:107490008C2D0E9460602220B1F06091BF0F70912E
:1074A000C00F40E08C2D0E941F600E946388AA815B
:1074B000BB8112968C910E9468608E159F05ACF37B
:1074C0008C2D0E94F15FEA81FB81F78AE68AB70181
:1074D000828110C0DD20B1F064E378E08C2D0E9441
:1074E0006060AA81BB815796FC92EE925697B701D5
:1074F00012968C910E9478606CED75E08C2D0E9444
:10750000646012C064E873E08C2D0E946460EA81BC
:10751000FB81178B068BB80182810E9478606CED2D
:1075200075E08C2D0E9460600E941A6E2B013C0158
:10753000F8EC4F0E511C611C711C19823320D1F1E3
:10754000809154118823A1F1409157115091581105
:10755000E0915B11F0915C11858196819C01285C22
:107560003109421753072CF088539F4F8417950712
:10757000FCF481E0D8268091950690919606DD2056
:1075800039F06BEA7FE00E94114B82E090E006C088
:1075900069E97FE00E94114B81E090E040DD0E94AC
:1075A0001A6EAA81BB815896DC928824839403C00A
:1075B000812C1EC0812C80915411882309F405C2AE
:1075C000E0915B11F0915C1185819681409157119A
:1075D000509158119C0121533109421753070CF463
:1075E000F4C1C19633243394841795070CF4EDC18C
:1075F0000E944B630E94317780EF9AE00E94A05E68
:107600008091DF0A882309F4A9CE8091E10A8823BA
:1076100009F4A4CE0E9431770E941C8A8823D1F3FA
:10762000B4E0AB16B10459F0E5E0AE16B10409F4CC
:1076300065C0F3E0AF16B10409F059C1CBC0109397
:10764000AC0F0093AB0FF092AE0FE092AD0FD09263
:10765000AF0FB8018CE191E00E949776B7018EE1FF
:1076600091E00E9497766D2D80E291E00E9425784E
:10767000B80184E00E94965FB70184E00E947B5FBE
:10768000E0919306F0919406D08E8091AA0F8D30F0
:1076900029F4E091400DF091410DD08E6CED75E034
:1076A00084E00E94786066E970E080E090E00E94EB
:1076B000694E8091AA0F8D30E1F484E00E946860E9
:1076C000A0919306B0919406ED91FC9111970190D1
:1076D000F081E02D8D3D95401CF06FEF7FEF02C0F3
:1076E00061E070E0CD011995809193069091940628
:1076F0005BC0809193069091940664C01093B30F81
:107700000093B20FF092B50FE092B40FD092B60F83
:10771000B80183E291E00E949776B70185E291E09B
:107720000E9497766D2D87E291E00E942578B8013E
:1077300085E00E94965FB70185E00E947B5FE09143
:107740008F06F0919006D08E6CED75E085E00E947A
:10775000786066E970E080E090E00E94694E809178
:10776000A90F8D3059F585E00E946860A0918F06C1
:10777000B09190068D3D95404CF0ED91FC911197A4
:107780000190F081E02D6FEF7FEF08C0ED91FC914B
:1077900011970190F081E02D61E070E0CD01199525
:1077A00080918F0690919006DC01ED91FC91019003
:1077B000F081E02D60E070E0199599C080918F060E
:1077C00090919006DC01ED91FC910480F581E02D13
:1077D00019958DC01093C20F0093C10FF092C40F82
:1077E000E092C30FD092BB0FB80182E391E00E94F8
:1077F0009776B70184E391E00E9497766D2D8CE235
:1078000091E00E942578B80183E00E94965FB7015D
:1078100083E00E947B5F8091BB0FE0916C12F0913E
:107820006D12808F8091BB0F0E94627683E00E9470
:1078300068602091BB0F222369F1B9E0BC1538F0D4
:107840002091BF113091C0113695279502C02EEEC0
:1078500032E08217930709F44AC06091BF0F70911C
:10786000C00F41E083E00E941F600E946388EA81AC
:10787000FB8182810E94686008171907B4F383E0D6
:107880000E94F15FAA81BB8157961C930E93569775
:10789000B80129C029E02C1508F499C02091BD1128
:1078A0003091BE11369527958217930701F16091AB
:1078B000BF0F7091C00F40E083E00E941F600E94E4
:1078C0006388EA81FB8182810E9468608E159F0532
:1078D000B4F383E00E94F15FAA81BB815796FC92CA
:1078E000EE925697B70112968C910E947860809123
:1078F0009506909196060E94FE4AACD4B4E0AB1671
:10790000B10459F0E5E0AE16B10451F0F3E0AF1662
:10791000B10471F46FE47FE005C06FE77FE002C05F
:1079200066E67FE080919506909196060E94114B45
:1079300091D464E47FE080919506909196060E9430
:10794000114B68E37FE080919506909196060E9426
:10795000A049B80180919506909196060E94F07713
:107960006CE27FE080919506909196060E94A04976
:10797000B70180919506909196060E94F07760E29B
:107980007FE080919506909196060E94A0498D2DEA
:107990003DD480919506909196060E94FE4A0F90E4
:1079A0000F900F90DF91CF911F910F91FF90EF906B
:1079B000DF90CF90BF90AF909F908F907F906F900F
:1079C0005F904F903F902F90A5C6312C11CE2AEC9E
:1079D00038E06ACF83E090E022CB82E090E01FCBDA
:1079E00081E090E01CCB80919806809397060895E3
:1079F0008091730D882359F08091710D9091720DD3
:107A0000DC01ED91FC910480F581E02D199408953D
:107A10008091730D882369F08091710D9091720DA2
:107A2000DC01ED91FC910190F081E02D6FEF73E0AE
:107A3000199408958091730D882389F08091770DB2
:107A4000882321F080E090E0D3DF03C080E090E065
:107A5000DFDF9091770D81E089278093770D08957E
:107A60002091730D222369F0A091710DB091720DD8
:107A7000ED91FC9111970190F081E02DBC01CD01B9
:107A8000199408958091700D882359F080916E0D9E
:107A900090916F0DDC01ED91FC910480F581E02D5A
:107AA000199408958091700D882369F080916E0D6E
:107AB00090916F0DDC01ED91FC910190F081E02D32
:107AC0006FEF73E0199408958091700D882389F009
:107AD0008091760D882321F080E090E0D3DF03C011
:107AE00080E090E0DFDF9091760D81E08927809340
:107AF000760D08952091700D222369F0A0916E0DEE
:107B0000B0916F0DED91FC9111970190F081E02DF6
:107B1000BC01CD011994089520916D0D222369F0C7
:107B2000A0916B0DB0916C0DED91FC9111970190AE
:107B3000F081E02DBC01CD011994089520916A0DCA
:107B4000222369F0A091680DB091690DED91FC912F
:107B500011970190F081E02DBC01CD011994089599
:107B60002091670D222369F0A091650DB091660DFB
:107B7000ED91FC9111970190F081E02DBC01CD01B8
:107B8000199408952091640D222369F0A091620D4B
:107B9000B091630DED91FC9111970190F081E02D72
:107BA000BC01CD01199408952091610D222369F043
:107BB000A0915F0DB091600DED91FC911197019036
:107BC000F081E02DBC01CD011994089520915E0D46
:107BD000222369F0A0915C0DB0915D0DED91FC91B7
:107BE00011970190F081E02DBC01CD011994089509
:107BF00020915B0D222369F0A091590DB0915A0D8F
:107C0000ED91FC9111970190F081E02DBC01CD0127
:107C1000199408958091910690919206DC01ED915E
:107C2000FC91E65AFF4F0190F081E02D199480916C
:107C3000910690919206DC01ED91FC91E85AFF4F7C
:107C40000190F081E02D1994809191069091920617
:107C5000DC01ED91FC91EA5AFF4F0190F081E02D9B
:107C600019948091C50F81110DC080910C069091DF
:107C70000D06DC01ED91FC910190F081E02D60E0BA
:107C800070E0199408958091C50F81110DC0809105
:107C90000C0690910D06DC01ED91FC910190F081B4
:107CA000E02D6FEF70E019940895A9C3BFC38091D0
:107CB000750D882311F0A3D301C0B8D39091750D31
:107CC00081E089278093750D0895C8C3DEC3809134
:107CD000740D882311F0C2D301C0D7D39091740DD5
:107CE00081E089278093740D0895809198068823F8
:107CF00061F00E948D63029741F066E471E180912A
:107D00009506909196060C94114B089580919706D4
:107D1000882341F068E670E180919506909196067F
:107D20000C94114B089580919706882341F068E5E3
:107D300070E180919506909196060C94114B0895F0
:107D4000CF93DF9320917A0D30917B0D281739075F
:107D5000D1F090937B0D80937A0D2091970622238A
:107D600091F0EC0167E171E18091950690919606A2
:107D70000E94A049BE018091950690919606DF91E0
:107D8000CF910C94D873DF91CF910895CF93DF9367
:107D90002091780D3091790D28173907D1F0909303
:107DA000790D8093780D20919706222391F0EC01B4
:107DB0006DEF70E180919506909196060E94A04922
:107DC000BE018091950690919606DF91CF910C941B
:107DD000D873DF91CF91089520916D0D222339F052
:107DE000BC018091570D9091580D0C945D860895BB
:107DF00020916A0D222339F0BC018091550D90919C
:107E0000560D0C945D8608952091670D222339F05C
:107E1000BC018091530D9091540D0C945D86089592
:107E20002091640D222339F0BC018091510D909175
:107E3000520D0C945D8608952091610D222339F036
:107E4000BC0180914F0D9091500D0C945D8608956A
:107E500020915E0D222339F0BC0180914D0D90914F
:107E60004E0D0C945D86089520915B0D222339F010
:107E7000BC0180914B0D90914C0D0C945D86089542
:107E8000CF92DF92EF92FF9220910002213019F4FD
:107E90002091D10F04C02230C9F52091D70F2223A1
:107EA000A9F19C01211584E0380710F02FEF33E091
:107EB000ADE0B0E00E944BB42FEF33E040E050E083
:107EC0000E94FDB369017A018FEFC81AD80AE80A47
:107ED000F80A8091DA128C15C9F0C092DA128091FA
:107EE0009706882399F066EB70E180919506909152
:107EF00096060E94A0496C2D809195069091960659
:107F0000FF90EF90DF90CF900C944B76FF90EF9026
:107F1000DF90CF900895CF92DF92EF92FF92209161
:107F20000002213019F42091CE0F04C02230C9F58F
:107F30002091D40F2223A9F19C01211584E0380758
:107F400010F02FEF33E0ADE0B0E00E944BB42FEF24
:107F500033E040E050E00E94FDB369017A018FEF09
:107F6000C81AD80AE80AF80A8091D8128C15C9F004
:107F7000C092D81280919706882399F06FE970E13A
:107F800080919506909196060E94A0496C2D809153
:107F9000950690919606FF90EF90DF90CF900C940D
:107FA0004B76FF90EF90DF90CF90089581E0809323
:107FB0008E06AFD680919706882341F065E870E180
:107FC00080919506909196060C94114B089583E04C
:107FD00080938E066DD380919706882341F062E9E5
:107FE00070E180919506909196060C94114B08953E
:107FF00082E080938E065CD380919706882341F0BF
:1080000068E770E180919506909196060C94114B6B
:1080100008950C9444888091010281110C94288861
:108020000C9444880C94288880910002813011F4CB
:1080300082E001C081E00C946D8F82E00C946D8F22
:1080400081E00C946D8F0C949E229091F60F81E04C
:10805000892714C580E012C581E010C59091F40F06
:1080600081E089273AC580E038C581E036C5809136
:108070003006882321F0C3D126E132E403C0D6D1F3
:108080002FEF31E44CE251E060E070E080EF9AE0E5
:108090000C94905E80912906882321F0DFD125E49D
:1080A00032E403C0F2D12EE232E44CE251E060E06F
:1080B00070E080EF9AE00C94905E8CE00C941D8749
:1080C0008BE00C941D878AE00C941D878CE00C9447
:1080D00044878BE00C9444878AE00C9444878CE0BE
:1080E0000C946B878BE00C946B87682F80919506BE
:1080F000909196060E94A07764E471E180919506C4
:10810000909196060C94A049F0DF8091950690918D
:1081100096060C94FE4ACF92DF92EF92FF929C015A
:10812000A3E6B0E00E944BB42FEF33E040E050E014
:108130000E94FDB369017A018FEFC81AD80AE80AD4
:10814000F80A8091F1058C15A1F0C092F10580919B
:108150009706882371F066EE70E180919506909104
:1081600096060E94A0498C2DFF90EF90DF90CF9053
:10817000CBCFFF90EF90DF90CF900895CF92DF921A
:10818000EF92FF929C01A3E6B0E00E944BB42FEF68
:1081900033E040E050E00E94FDB369017A018FEFC7
:1081A000C81AD80AE80AF80A8091F2058C15A1F0DD
:1081B000C092F20580919706882371F06DEC70E112
:1081C00080919506909196060E94A0498C2DFF9073
:1081D000EF90DF90CF9098CFFF90EF90DF90CF900F
:1081E00008952091950630919606882319F06BE149
:1081F00077E002C06FE177E0C9010C94A049F1DF9C
:1082000080919506909196060C94FE4A20919506D1
:1082100030919606882319F069E371E102C06EE39C
:1082200071E1C9010E94A04980919506909196063E
:108230000C94FE4A67E371E1809195069091960651
:108240000C94A04963E371E18091950690919606A4
:108250000C94A049CF93CDE261E371E18091950642
:10826000909196060E94A049C150B1F78091950661
:10827000909196060E94FE4A8091950690919606EE
:10828000DC01ED91FC910284F385E02DCF911994EE
:10829000CF93C091890D6C2F70E088E00E94834DD0
:1082A00089E18093880D90910E02992311F0CD5FA2
:1082B00001C0C350C093890D8091890D873970F03A
:1082C000992321F08FEF8093890D08C08D3D30F008
:1082D00086E98093890D88E78093880D8091890DC8
:1082E0008F3F19F410920E0205C08A3118F481E014
:1082F00080930E024091880D50E060E070E028E429
:1083000031E480EF9AE00E94905E90933F12809358
:108310003E12CF910895CF92DF92EF92FF92CF93CA
:10832000DF93EC019C01AFEFB0E00E944BB4CC2492
:10833000CA9423E0D22EE12CF12CA70196010E94D1
:10834000FDB3B90188E00E94834D9E01A4E6B0E030
:108350000E944BB4A70196010E94FDB380914E107C
:10836000821320934E10DF91CF91FF90EF90DF901A
:10837000CF90089561E088E00E94184D80919706A3
:10838000882361F080914012811108C06AE673E190
:1083900080919506909196060C94114B0895CF9379
:1083A0008091850D81110FC081E08093850D8091B2
:1083B0009706882341F068E373E1809195069091D8
:1083C00096060E94114BC091840D6C2F85E00E948F
:1083D000184D4091531050E060E070E02FEC31E414
:1083E00080EF9AE00E94905E9093830D8093820DBF
:1083F00081E06C2F68276093840DCF910895809160
:10840000070180FF12C060E08EE30E94184D1092B9
:108410002E0680919706882341F06FEA72E18091E1
:108420009506909196060C94114B08958091070142
:1084300080FF13C061E08EE30E94184D81E08093BD
:108440002E0680919706882341F069E972E18091B8
:108450009506909196060C94114B08958091070112
:1084600081FF12C060E08FE30E94184D1092270632
:1084700080919706882341F062E872E18091950629
:10848000909196060C94114B08958091070181FFFD
:1084900013C061E08FE30E94184D81E080932706AE
:1084A00080919706882341F06CE672E180919506F1
:1084B000909196060C94114B08958091F4058823B1
:1084C00071F01092F40580919706882341F064EED4
:1084D00071E180919506909196060C94114B089548
:1084E0008091E40F833099F08091F40581110FC0E1
:1084F00081E08093F40580919706882341F06FEC2A
:1085000071E180919506909196060C94114B089517
:108510008091F405882319F080E090E0CECF80E0D0
:1085200090E0DECF8091F305833079F083E0809393
:10853000F30580919706882341F06EEB71E18091FD
:108540009506909196060C94114B08958091F30531
:10855000823079F082E08093F3058091970688233A
:1085600041F06DEA71E180919506909196060C9428
:10857000114B08958091F305813079F081E080936B
:10858000F30580919706882341F06CE971E18091B1
:108590009506909196060C94114B0895CF93DF9316
:1085A000C0913E12D0913F12BE0180EF9AE00E942E
:1085B000295E882329F0BE0180EF9AE00E94415E87
:1085C00060E088E00E94184D809197068823D1F0E2
:1085D00080914012882319F060EA73E10DC0809108
:1085E0003D12882319F067E873E106C080913F0DC2
:1085F000811108C068E773E1809195069091960615
:108600000E94114B1092401210923D12DF91CF91B7
:1086100008958091401281110FC0C0DF81E08093E6
:10862000401280919706882339F06FEC73E18091B6
:10863000950690919606F5D78091870D882329F0AD
:1086400060E088E00E94184D01C094DE9091870D93
:1086500081E089278093870D882329F040914A1073
:1086600050914B1004C040914C1050914D1060E05F
:1086700070E029E033E480EF9AE00E94905E9093EE
:108680003F1280933E1208950E948D7E8091F505E1
:10869000882369F00E94CE8E80919706882339F056
:1086A0006CE571E18091950690919606BAC70895A0
:1086B0000E948D7E8091F505882359F18091C50A2D
:1086C000811127C080918D06811123C081E08093A4
:1086D0008D060E94D28780912006882319F010927F
:1086E00020060CC08091910690919206DC01ED91DC
:1086F000FC910088F189E02D61E019958091970641
:10870000882339F061E771E1809195069091960692
:1087100088C7089560E089E30C94184D61E089E30F
:108720000C94184D60914E1070E088E00E94834DCB
:1087300080919706882339F069EB73E18091950663
:10874000909196066EC708951092860D80918306CB
:10875000811104C060E084E00E94184D809197066A
:10876000882339F067E573E180919506909196062C
:1087700058C7089581E08093860D8091830681110A
:1087800006C060917D0D70E084E00E94834D809171
:108790009706882339F065E473E1809195069091FE
:1087A00096063FC70895109283068091860D811129
:1087B00004C060E084E00C94184D60917D0D70E081
:1087C00084E00C94834DCF93DF9360E085E00E94BA
:1087D000184D8091850D81110BC08091910690916B
:1087E0009206DC01ED91FC9102ACF3ADE02D199500
:1087F000C091820DD091830DBE0180EF9AE00E945E
:10880000295E882329F0BE0180EF9AE00E94415E34
:1088100080919706882371F02091850D80919506AF
:1088200090919606222319F06CE273E102C060E297
:1088300073E1F7D61092850DDF91CF91089561E035
:1088400085E00E94184D8091910690919206DC017E
:10885000ED91FC9102ACF3ADE02D19958091970656
:10886000882339F065E173E1809195069091960631
:10887000D8C6089560E085E30E94184D8091910666
:1088800090919206DC01ED91FC9106A8F7A9E02DEC
:10889000199580919706882339F069E073E18091FA
:1088A000950690919606BDC6089561E085E30E9405
:1088B000184D8091910690919206DC01ED91FC910A
:1088C00006A8F7A9E02D199580919706882339F01D
:1088D0006EEF72E18091950690919606A2C608957A
:1088E0008F929F92AF92BF92CF92DF92EF92FF92C0
:1088F00085E40E944A4EBC01990F880B990B0E9497
:10890000BAB220E030E040E85AE30E9419B320E018
:1089100030E040EA50E40E9419B36B017C01809181
:108920000D02882351F0C0927E0DD0927F0DE0920F
:10893000800DF092810D10920D0226E636E646E695
:108940005FE360917E0D70917F0D8091800D90911D
:10895000810D0E9419B34B015C0120ED3CEC4CEC05
:108960005DE3C701B6010E9419B39B01AC01C501CB
:10897000B4010E94AFAE60937E0D70937F0D809323
:10898000800D9093810D2DE33CE248E450E40E9479
:1089900019B32AE939E949E95EE30E94AFAEFF90D5
:1089A000EF90DF90CF90BF90AF909F908F90089501
:1089B000CF93DF938091070180FD2AC0C0912B06E1
:1089C000D0912C0680913006882371F08EE30E94AE
:1089D0004A4E813092402CF010922C0610922B06B9
:1089E0000AC081E090E003C08EE30E944A4E90935B
:1089F0002C0680932B0680912B0690912C068C17C9
:108A00009D0719F410922D0603C081E080932D0676
:108A1000DF91CF910895CF93DF938091070181FD7E
:108A20002AC0C0912406D09125068091290688236A
:108A300071F08FE30E944A4E813092402CF01092E8
:108A40002506109224060AC081E090E003C08FE35F
:108A50000E944A4E90932506809324068091240616
:108A6000909125068C179D0719F41092260603C0D5
:108A700081E080932606DF91CF910895909197062B
:108A80008823C9F08091F4068823A9F081E08093BF
:108A9000F60F80937C0D9923F9F06BE372E18091DE
:108AA0009506909196064CD40E94979180919506D8
:108AB00090919606A3C51092F60F992339F063E5BD
:108AC00072E18091950690919606ABD58091F40F56
:108AD000811102C010927C0D089590919706882311
:108AE000E9F08091F4068823C9F08091AA0F8D30B7
:108AF000A9F481E08093F40F80937C0D9923F9F021
:108B00006AEF71E1809195069091960619D40E94C2
:108B1000C591809195069091960670C51092F40FBC
:108B2000992339F06AE172E1809195069091960659
:108B300078D58091F60F811102C010927C0D0895B6
:108B40008091E40F833041F12CF48130A9F0823020
:108B500099F02DC086305CF580918606909187064D
:108B6000DC01ED91FC910480F581E02D1995809157
:108B700084069091850614C080918A0690918B0698
:108B8000DC01ED91FC910480F581E02D1995809137
:108B900088069091890604C0809186069091870688
:108BA000DC01ED91FC910480F581E02D1995809117
:108BB000910690919206DC01ED91FC91EA5BFF4FEA
:108BC0000190F081E02D1995809191069091920687
:108BD000DC01ED91FC910284F385E02D60E070E012
:108BE0001994AEDF0E9430700E948D7E8091F50551
:108BF00081110E94CE8E8091930690919406DC01A3
:108C0000ED91FC910480F581E02D199580918F06FE
:108C100090919006DC01ED91FC910480F581E02DAE
:108C200019958091C50F882359F080910C06909179
:108C30000D06DC01ED91FC910480F581E02D199485
:108C4000089580910C02882351F04ADE20E030E044
:108C500040E050E40E94B4B287FF38C0089540DE7F
:108C600020E030E04AE754E40E9419B30E9480AF4C
:108C7000209143103091441040919A066217730777
:108C800010F4442349F1442309F442C029DE20E0D2
:108C900030E04AE754E40E9419B30E9480AF20916B
:108CA0004310309144106217730790F110929A06A6
:108CB00081E08093990680919706882349F166ECBC
:108CC00072E18091950690919606ABC410920C02C9
:108CD00081E080939906089581E080939A0610922E
:108CE000990680919706882381F065EE72E1809164
:108CF00095069091960624D30E94667F62EE72E1FB
:108D000080919506909196068CD46BDF0C942D374C
:108D100008950E948D7E8091F505882339F1809118
:108D20008D06811101C0089510928D060E94A087C2
:108D300080912006882319F0109220060CC08091A3
:108D4000910690919206DC01ED91FC910088F189E9
:108D5000E02D60E0199580919706882339F065E849
:108D600071E180919506909196065BC408950895EF
:108D7000CF92DF92EF92FF920F931F93CF93DF93E7
:108D80006C017A018B01C0E0D0E0CE15DF0589F0DF
:108D9000D8016D918D01D601ED91FC910190F0818A
:108DA000E02DC6011995892B11F47E0102C0219690
:108DB000ECCFC701DF91CF911F910F91FF90EF9002
:108DC000DF90CF900895FC01A089B1898C91A6898C
:108DD000B78982FD0FC09C91818D8F5F8F73228D2B
:108DE000821749F0218DDF01A20FB11D5D969C9382
:108DF000818F08958C910895FC01918D828D981733
:108E000061F0828DDF01A80FB11D5D968C91928D6E
:108E10009F5F9F73928F90E008958FEF9FEF08956B
:108E2000FC01918D828D981731F0828DE80FF11D34
:108E3000858D90E008958FEF9FEF0895FC01918D4F
:108E4000228D892F90E0805C9F4F821B91098F7348
:108E50009927089585EF96E0F1DF21E0892B09F449
:108E600020E0822F089582E997E0E8DF21E0892B56
:108E700009F420E0822F08958FE298E0DFDF21E0FF
:108E8000892B09F420E0822F08958CEC98E0D6DF3E
:108E900021E0892B09F420E0822F0895FC01848DC4
:108EA000DF01A80FB11DA35ABF4F2C91848D90E014
:108EB00001968F739927848FA689B7892C93A089EF
:108EC000B1898C9180648C93938D848D981306C0A6
:108ED0000288F389E02D80818F7D80830895EF9251
:108EE000FF920F931F93CF93DF93EC0181E0888F64
:108EF0009B8D8C8D981305C0E889F989808185FD4B
:108F000023C0F62E0B8D10E00F5F1F4F0F7311273C
:108F1000E02E8C8DE8120BC00FB607FCFACFE88963
:108F2000F989808185FFF5CFCE01B8DFF2CF8B8D37
:108F3000FE01E80FF11DE35AFF4FF0820B8FEA8923
:108F4000FB898081806207C0EE89FF896083E889A0
:108F5000F98980818064808381E090E0DF91CF9106
:108F60001F910F91FF90EF900895CF93DF93EC0145
:108F7000888D8823C1F0EA89FB89808185FD05C041
:108F8000A889B9898C9186FD0EC00FB607FCF5CF74
:108F9000808185FFF2CFA889B9898C9185FFEDCFBB
:108FA000CE017CDFE8CFDF91CF91089580E090E0A3
:108FB000892B19F06ADF811116C080E090E0892BBF
:108FC00019F05ADF811112C080E090E0892B19F06E
:108FD0004ADF81110EC080E090E0892B79F03ADF02
:108FE00081110AC008950E940000E7CF0E9400008E
:108FF000EBCF0E940000EFCF0C940000089590E0AA
:10900000FC013197E231F10508F04EC08827EC5B96
:10901000FE4F8F4F0C949AAE809180008F7703C0E3
:10902000809180008F7D80938000089580918000E2
:10903000877FF9CF84B58F7702C084B58F7D84BDDB
:1090400008958091B0008F7703C08091B0008F7D2C
:109050008093B0000895809190008F7707C0809131
:1090600090008F7D03C080919000877F8093900057
:1090700008958091A0008F7707C08091A0008F7D18
:1090800003C08091A000877F8093A0000895809105
:1090900020018F7707C0809120018F7D03C08091D0
:1090A0002001877F8093200108950E94C5B10F930E
:1090B0001F93CF93DF938C01EB01FC0180819181A1
:1090C0000097B1F0688179816115710579F042816D
:1090D00053812C813D814217530740F00E94DDB13E
:1090E0008C819D81F8019583848313C00E9449B0CF
:1090F00088819981F801918380838A819B81938300
:1091000082838C819D8195838483198218821B823E
:109110001A821D821C82DF91CF911F910F910895B9
:109120000F931F93CF93DF93EC0188819981009770
:1091300029F02A813B812617370788F48B016F5F5E
:109140007F4F0E94E1B0009761F0998388831B8371
:109150000A832C813D81232B11F4FC01108281E0D4
:1091600001C080E0DF91CF911F910F910895EF92A0
:10917000FF920F931F93CF93DF93FB0124813581DF
:10918000E080F180FC0104811581E114F10411F407
:1091900080E016C02115310591F0EC01020F131F7C
:1091A000B801BEDF8823A1F3288139818C819D819C
:1091B000B701820F931F0E94DDB11D830C8381E0F4
:1091C000DF91CF911F910F91FF90EF900895EF9253
:1091D000FF920F931F93CF93DF93EC017B018A01E2
:1091E000BA019EDF2881398181110DC02115310519
:1091F00019F0C9010E9449B0198218821D821C828F
:109200001B821A8206C01D830C83B701C9010E940C
:10921000DDB1CE01DF91CF911F910F91FF90EF90C3
:109220000895CF93DF93EC016115710551F0FB01B7
:1092300001900020E9F73197AF01461B570BC7DFBC
:109240000CC088819981009711F00E9449B0198261
:1092500018821D821C821B821A82CE01DF91CF915F
:109260000895FC01808191810C9449B00F931F9364
:10927000CF93DF93CDB7DEB762970FB6F894DEBF1A
:109280000FBECDBF8C01CB01F80111821082138279
:1092900012821582148250E0BE016F5F7F4F0E94E0
:1092A00048B2BE016F5F7F4FC801BBDF62960FB649
:1092B000F894DEBF0FBECDBFDF91CF911F910F910C
:1092C0000895FC0111821082138212821582148289
:1092D0006115710549F0FB0101900020E9F7319714
:1092E000AF01461B570B73CF0895CF93DF9300D088
:1092F0001F92CDB7DEB7611571058105910579F033
:109300009B01AC0169833A834B835C830E943CB22E
:1093100029813A814B815C810E94FDB303C060E0EA
:1093200070E0CB010F900F900F900F90DF91CF91D5
:109330000895DC01ED91FC910190F081E02D1994EC
:10934000EF92FF920F931F93CF93DF938C017B01DA
:10935000C0E0D0E0F701EC0FFD1F6491662361F0DF
:10936000D801ED91FC910190F081E02DC801199593
:10937000892B11F02196EECFCE01DF91CF911F9175
:109380000F91FF90EF9008956115710579F0FB0141
:1093900001900020E9F73197AF01461B570BDC0124
:1093A000ED91FC910280F381E02D199480E090E032
:1093B00008954F925F926F927F92EF92FF920F9378
:1093C0001F93CF93DF93CDB7DEB7A1970FB6F89475
:1093D000DEBF0FBECDBF7C01FA01CB0119A2223046
:1093E00008F42AE08E010F5D1F4F422E512C612C94
:1093F000712CBF01A30192010E9429B4F901CA0195
:10940000015011096A3014F4605D01C0695CD80133
:109410006C93232B242B252B61F7B801C701B4DFF4
:10942000A1960FB6F894DEBF0FBECDBFDF91CF91EE
:109430001F910F91FF90EF907F906F905F904F90F2
:1094400008954F925F926F927F928F929F92AF9208
:10945000BF92CF92DF92EF92FF92CF93DF93EC0116
:109460006A017B01B22E9A01AB01C701B6010E94CD
:10947000B0AF882319F068ED75E027C026013701E9
:10948000E89477F82FEF3FEF4FE75FE7C301B201B2
:109490000E94B0AF81110DC02FEF3FEF4FE75FE7A4
:1094A000C301B2010E94B4B218161CF46CED75E051
:1094B0000CC02FEF3FEF4FE75FE4C701B6010E94FA
:1094C000ACAF181694F460EE75E0CE01DF91CF9149
:1094D000FF90EF90DF90CF90BF90AF909F908F90D4
:1094E0007F906F905F904F904FCF2FEF3FEF4FE700
:1094F0005FECC701B6010E94B4B287FDE4CF20E063
:1095000030E0A901C701B6010E94B4B287FF09C0CB
:109510006DE2CE010EDF4C01F7FAF094F7F8F0940B
:1095200002C0812C912CA12C60E070E080E09FE3D0
:10953000AB1441F020E030E040E251E40E9413AF70
:10954000A394F6CF9B01AC01C701B6010E94AFAE58
:109550002B013C010E9480AF6B017C010E94B8B2DC
:109560009B01AC01C301B2010E94AEAE2B013C01D4
:109570002AE0B701A601CE011CDF7C01E80CF91C32
:10958000BB2029F06EE2CE01D4DEE80EF91EDB2C02
:10959000DD2021F120E030E040E251E4C301B201DE
:1095A0000E9419B32B013C010E9480AF4B01A12CFA
:1095B000B12C2AE0B501A401CE01FBDEE80EF91EB4
:1095C000C501B4010E94B8B29B01AC01C301B20154
:1095D0000E94AEAE2B013C01DA94DACFC701DF91D5
:1095E000CF91FF90EF90DF90CF90BF90AF909F9082
:1095F0008F907F906F905F904F90089564EE75E02C
:10960000C3CE0F931F93CF93DF93EC01BDDE8C018C
:10961000CE01F4DF800F911FDF91CF911F910F9149
:1096200008950F931F93CF93DF93EC0189DE8C0194
:10963000CE01E4DF800F911FDF91CF911F910F9139
:1096400008951F920F920FB60F9211240BB60F922E
:109650002F933F934F935F936F937F938F939F933A
:10966000AF93BF93EF93FF9385EF96E017DCFF91E5
:10967000EF91BF91AF919F918F917F916F915F918A
:109680004F913F912F910F900BBE0F900FBE0F90F7
:109690001F9018951F920F920FB60F9211240BB6C0
:1096A0000F922F933F934F935F936F937F938F937B
:1096B0009F93AF93BF93EF93FF9385EF96E083DB88
:1096C000FF91EF91BF91AF919F918F917F916F919A
:1096D0005F914F913F912F910F900BBE0F900FBE56
:1096E0000F901F9018951F920F920FB60F92112492
:1096F0000BB60F922F933F934F935F936F937F938C
:109700008F939F93AF93BF93EF93FF9382E997E07B
:10971000C5DBFF91EF91BF91AF919F918F917F91A9
:109720006F915F914F913F912F910F900BBE0F90D2
:109730000FBE0F901F9018951F920F920FB60F92A9
:1097400011240BB60F922F933F934F935F936F9318
:109750007F938F939F93AF93BF93EF93FF9382E990
:1097600097E031DBFF91EF91BF91AF919F918F9186
:109770007F916F915F914F913F912F910F900BBE11
:109780000F900FBE0F901F9018951F920F920FB65B
:109790000F9211240BB60F922F933F934F935F9329
:1097A0006F937F938F939F93AF93BF93EF93FF93A9
:1097B0008FE298E073DBFF91EF91BF91AF919F91A2
:1097C0008F917F916F915F914F913F912F910F906A
:1097D0000BBE0F900FBE0F901F9018951F920F9207
:1097E0000FB60F9211240BB60F922F933F934F9306
:1097F0005F936F937F938F939F93AF93BF93EF93F9
:10980000FF938FE298E0DFDAFF91EF91BF91AF9184
:109810009F918F917F916F915F914F913F912F9188
:109820000F900BBE0F900FBE0F901F9018951F92B8
:109830000F920FB60F9211240BB60F922F933F93F6
:109840004F935F936F937F938F939F93AF93BF9348
:10985000EF93FF938CEC98E021DBFF91EF91BF91A8
:10986000AF919F918F917F916F915F914F913F91B8
:109870002F910F900BBE0F900FBE0F901F90189559
:109880001F920F920FB60F9211240BB60F922F93C7
:109890003F934F935F936F937F938F939F93AF9378
:1098A000BF93EF93FF938CEC98E08DDAFF91EF91EB
:1098B000BF91AF919F918F917F916F915F914F91E8
:1098C0003F912F910F900BBE0F900FBE0F901F90E6
:1098D0001895CF93DF93EC01E881F9810284F38539
:1098E000E02D1995EA89FB8980818F7E8083EA8942
:1098F000FB898081877F8083EA89FB8980818F77DC
:109900008083EA89FB8980818F7D80838A8D898F1E
:10991000DF91CF910895CF92DF92EF92FF921F9344
:10992000CF93DF93EC016A017B01122FE889F9895B
:1099300082E080834115514E61057105B1F060E010
:1099400079E08DE390E0A70196010E9429B4DA0145
:10995000C9010197A109B109B695A7959795879572
:10996000AC01411580E15807A8F0E889F989108217
:1099700060E874E88EE190E0A70196010E9429B4A6
:10998000BA01A9014150510961097109769567959C
:1099900057954795EC85FD855083EE85FF8540837F
:1099A000188EEC89FD891083EA89FB8980818061AA
:1099B0008083EA89FB89808188608083EA89FB89CA
:1099C000808180688083EA89FB8980818F7D8083A4
:1099D000DF91CF911F91FF90EF90DF90CF9008958E
:1099E000CF93DF93282F30E0F901ED53FB4E8491A4
:1099F000F901E358FB4ED491F901E95CFB4EC491A7
:109A0000CC2389F08111FBDAEC2FF0E0EE0FFF1F81
:109A1000E35EFB4EA591B491EC91ED2381E090E0E3
:109A200021F480E002C080E090E0DF91CF910895C2
:109A30001F93CF93DF93282F30E0F901ED53FB4EB6
:109A40008491F901E358FB4ED491F901E95CFB4E96
:109A5000C491CC23C1F0162F8111D1DAEC2FF0E0A4
:109A6000EE0FFF1FED5FFB4EA591B4918FB7F894F9
:109A7000111105C09C91ED2FE095E92302C0EC91F6
:109A8000ED2BEC938FBFDF91CF911F910895CF9372
:109A9000DF9390E0FC01E358FB4E2491FC01E95C6C
:109AA000FB4E8491882361F190E0880F991FFC019F
:109AB000E751FC4EC591D491FC01ED5FFB4EA591A1
:109AC000B491611109C09FB7F894888120958223D1
:109AD0008883EC912E230BC0623061F49FB7F89419
:109AE0003881822F809583238883EC912E2B2C93B1
:109AF0009FBF06C08FB7F894E8812E2B28838FBFB5
:109B0000DF91CF9108951F93CF93DF93182FEB012F
:109B100061E0BDDF209711F460E004C0CF3FD105C4
:109B200031F461E0812FDF91CF911F9181CFE12F3F
:109B3000F0E0ED53FB4EE4914E2F50E0FA013197E7
:109B4000E231F10508F09DC08827EA5AFE4F8F4F99
:109B50000C949AAE84B5806884BDC7BD97C084B5A7
:109B6000806284BDC8BD92C080918000806880936F
:109B70008000D0938900C093880088C080918000C5
:109B8000806280938000D0938B00C0938A007EC057
:109B900080918000886080938000D0938D00C09376
:109BA0008C0074C08091B00080688093B000C09336
:109BB000B3006CC08091B00080628093B000C0930D
:109BC000B40064C080919000806880939000D0932E
:109BD0009900C09398005AC0809190008062809351
:109BE0009000D0939B00C0939A0050C08091900049
:109BF000886080939000D0939D00C0939C0046C0E5
:109C00008091A00080688093A0008091A0008F7B4D
:109C10008093A000D093A900C093A80037C0809182
:109C2000A00080628093A000D093AB00C093AA00F4
:109C30002DC08091A00088608093A000D093AD00DB
:109C4000C093AC0023C080912001806880932001E4
:109C5000D0932901C093280119C08091200180620E
:109C600080932001D0932B01C0932A010FC08091D3
:109C70002001886080932001D0932D01C0932C0196
:109C800005C0C038D1050CF04CCF46CFDF91CF9145
:109C90001F910895863308F0865390917B00282FFA
:109CA0002870977F922B90937B00877080648093BD
:109CB0007C0080917A00806480937A0080917A00A1
:109CC00086FDFCCF809178002091790090E0922B66
:109CD00008958F929F92AF92BF92CF92DF92EF92B0
:109CE000FF926B017C010E94F56D4B015C01C11478
:109CF000D104E104F104F1F00E94F56DDC01CB0127
:109D000088199909AA09BB09883E9340A105B105A4
:109D100070F321E0C21AD108E108F10888EE880E3C
:109D200083E0981EA11CB11CC114D104E104F1040C
:109D300019F7DDCFFF90EF90DF90CF90BF90AF90FD
:109D40009F908F9008951092BF0A0895CF93DF934C
:109D5000C1E5DAE081E090E09A8389831092BF0A3E
:109D60000E94F56D6C837D838E839F83E49AEC9AC9
:109D7000DF91CF910895CF93DF93EC0161E089E00B
:109D800086DE60E089E054DE1092D60980E195E03D
:109D900099838883DF91CF910895CF92DF92EF92DC
:109DA000FF928091D709833009F061C08091D80972
:109DB0008130D1F488EE93E0A0E0B0E080936909AF
:109DC00090936A09A0936B09B0936C0980E797E1BF
:109DD000A0E0B0E080936D0990936E09A0936F09A5
:109DE000B093700932E001C030E0E091D809F0E0B2
:109DF000E752F64F2081A0E1A30F48EE53E060E068
:109E000070E088EBC82E8BE0D82EE12CF12C832F4C
:109E100090E0FC01EE0FFF1FEE0FFF1FE759F64F1A
:109E200027FF10C0C082D182E282F382880F991F7F
:109E3000880F991FFC01E359F64F408351836283D9
:109E400073830FC04083518362837383880F991F8C
:109E5000880F991FFC01E359F64FC082D182E2823C
:109E6000F3823E5F220F3A13D2CF3093D209FF9094
:109E7000EF90DF90CF900895CF93DF938091D60934
:109E8000811151C01092D4091092D109C1E0C09340
:109E9000D609D091D50961E089E0F9DD60E089E07B
:109EA000C7DD2D2F30E040E050E060E47FE180E04E
:109EB00090E00E94FDB3C093B00089E08093B100B0
:109EC0002093B3008BEA289F212D112426952093FF
:109ED000B40080916F008B7F80936F008091B00001
:109EE00080628093B0002091840030918500E091E1
:109EF000D10981E08E0F8093D10984E0E89FF001C1
:109F00001124E759F64F80819181A281B381820F9C
:109F1000931F90938B0080938A00B29A80916F0078
:109F2000846080936F00DF91CF9108954F925F928C
:109F30006F927F928F929F92AF92BF92CF92DF9259
:109F4000EF92FF928AE18093D2092093D30988E2AD
:109F50008093D50981E08093D8098093D9098EE058
:109F60008093D70980EC92E1A0E0B0E0809369098A
:109F700090936A09A0936B09B0936C0980EB94E00D
:109F8000A0E0B0E080936D0990936E09A0936F09F3
:109F9000B0937009A4E1440F551F661F771FAA955F
:109FA000D1F722E030E0B0EBCB2EB4E0DB2EE12C99
:109FB000F12C80E6482E89E0582E612C712C90E41B
:109FC000892E9CE9992EA12CB12CC901880F991FCB
:109FD000880F991FFC01E759F64F77FF05C04082B3
:109FE00051826282738204C0C082D182E282F38293
:109FF000C9010196880F991F880F991FFC01E75925
:10A00000F64F283129F0C082D182E282F38204C067
:10A0100080829182A282B382440F551F661F771FF0
:10A020002E5F3F4F2A31310581F6FF90EF90DF9090
:10A03000CF90BF90AF909F908F907F906F905F90E8
:10A040004F901ACF8F929F92AF92BF92CF92DF9292
:10A05000EF92FF9282E18093D20986E08093D30948
:10A0600096E29093D50991E09093D8099093D909FD
:10A070008093D70988ED90E4A0E0B0E0809369096F
:10A0800090936A09A0936B09B0936C098CE19CE0F2
:10A09000A0E0B0E080936D0990936E09A0936F09E2
:10A0A000B0937009742F66275527442722E030E0CB
:10A0B000ACE1CA2EACE0DA2EE12CF12CB8E38B2E09
:10A0C000B8E19B2EA12CB12CC901880F991F880FD4
:10A0D000991FFC01E759F64F77FF05C080829182F6
:10A0E000A282B38204C0C082D182E282F382F901EB
:10A0F000EE0FFF1FEE0FFF1FE359F64FC082D18214
:10A10000E282F382440F551F661F771F2E5F3F4F79
:10A1100022313105C9F68CE199E8A0E0B0E08093E6
:10A12000AD099093AE09A093AF09B093B009FF9029
:10A13000EF90DF90CF90BF90AF909F908F909CCE8C
:10A140001F920F920FB60F9211240BB60F922F93FE
:10A150003F934F935F936F937F938F939F93AF93AF
:10A16000BF93EF93FF939091D1098091D2099813F7
:10A1700016C01092D1098091D8098F5F8093D809B9
:10A180009091D8098091D909891740F481E0809392
:10A19000D8098091D4098F5F8093D409FEDD909116
:10A1A000D4098091D30998130DC08091B0008F7DA0
:10A1B0008093B00080916F008B7F80936F0010922E
:10A1C000D60927C08091B00085FF04C08091B000FF
:10A1D0008F7D03C08091B00080628093B000209199
:10A1E000840030918500E091D10981E08E0F809349
:10A1F000D10984E0E89FF0011124E759F64F8081EE
:10A200009181A281B381820F931F90938B008093E1
:10A210008A00FF91EF91BF91AF919F918F917F91B4
:10A220006F915F914F913F912F910F900BBE0F90C7
:10A230000FBE0F901F9018951F920F920FB60F929E
:10A2400011240BB60F921F932F933F934F935F935D
:10A250006F937F938F939F93AF93BF93EF93FF93EE
:10A26000CF93DF9300D01F92CDB7DEB78091510A14
:10A27000B7DB11E0892B09F010E00E94F56D6983CE
:10A280007A838B839C8389819A81AB81BC81409145
:10A29000550A5091560A6091570A7091580A841BCA
:10A2A000950BA60BB70B2091520A3091530A24301C
:10A2B000310509F44CC02530310521F0213031053C
:10A2C000E9F414C02091540A222339F02091BF0AE6
:10A2D00020FF02C0289A01C02898112379F0813EFE
:10A2E0002EE29207A105B10548F02BC0112379F1A8
:10A2F00025E030E03093530A2093520A2091520A0D
:10A300003091530A2530310511F5E091BF0AF0E094
:10A31000EE0FFF1FE75AF54F9183808389819A8161
:10A32000AB81BC818093550A9093560AA093570A3B
:10A33000B093580A8091BF0A8F5F8093BF0A83331E
:10A3400030F084E090E09093530A8093520A0F908B
:10A350000F900F900F90DF91CF91FF91EF91BF91F0
:10A36000AF919F918F917F916F915F914F913F91AD
:10A370002F911F910F900BBE0F900FBE0F901F904B
:10A38000189581E08093D20A089581E08093D30AE2
:10A39000089581E08093D40A0895CF938091D30DDE
:10A3A000C0910F028111FEC0C23009F44FC0C3300A
:10A3B00009F49BC0C13009F025C18091D40A8111F4
:10A3C00021C181E090E00E94B4AF9093E60D8093AC
:10A3D000E50D62E083E05BDB1092D20D1092DF0DA1
:10A3E0001092DE0D1092E30D80E090E0FC01EE0F84
:10A3F000FF1FE054F24F11821082019688309105C0
:10A40000A9F71092D10D1092D00D80916A008C6046
:10A4100080936A00ED9A8FB7F89420918400309170
:10A4200085003093BF0D2093BE0D8FBF29EC31E521
:10A430004AEF50E060E070E08091DA0D9091DB0D22
:10A440000E94905E81E08093D30DDCC08091D30A9E
:10A450008111D8C081E090E00E94B4AF9093E80DE4
:10A460008093E70D809104018E7F80930401809199
:10A47000050181608093050185EF96E09093120EAF
:10A480008093110E2EE240EA56E861E070E043DA74
:10A49000809165008B7F809365001092350189E083
:10A4A000809334018EE2809332018CEF80933001EF
:10A4B00080E9809331011092100E10920F0E1092CD
:10A4C0000E0E10920D0E10920B0EEBEEFDE08CEDC9
:10A4D00095E0819391932EE0EB30F207D1F7C1E044
:10A4E000C0930C0E25EC31E550C08091D20A811149
:10A4F00089C081E090E00E94B4AF9093EA0D809310
:10A50000E90D809104018E7F809304018091050103
:10A5100081608093050185EF96E09093940D809380
:10A52000930D26E040E052EC61E070E0F4D98091B8
:10A5300065008B7F809365001092350180E18093E8
:10A54000340186E0809332018EEF8093300180E900
:10A55000809331011092E10D1092E00D1092920D56
:10A560001092910D1092E20DE5E9FDE08CED95E081
:10A57000819391932DE0E13BF207D1F71092900D7A
:10A58000C1E0C0938F0D21EC31E54AEF50E060E06F
:10A5900070E08091DA0D9091DB0D0E94905EC09387
:10A5A000D30D30C0C23069F0C330D1F0C13051F5A5
:10A5B0008091D40A811126C08091DE0D9091DF0D2B
:10A5C0001DC08091D30A81111DC08091E70D90912B
:10A5D000E80D0E94436280910F0E9091100E0EC004
:10A5E0008091D20A81110EC08091E90D9091EA0DFF
:10A5F0000E94887A8091E00D9091E10D029711F40C
:10A60000C093DB0A80910F028230A1F1833009F4FC
:10A6100053C0813009F072C08091D40A882309F4B4
:10A620006DC0ED98E59A1092D20D1092E40D109243
:10A63000DF0D1092DE0D1092E30D80E090E0FC0142
:10A64000EE0FFF1FE054F24F118210820196883006
:10A650009105A9F71092D10D1092D00D8091E50DC2
:10A660009091E60D0E9449B01092D30D1092D30A3A
:10A6700082E042C08091D30A882309F43FC08091D0
:10A68000110E9091120E25D9809131018F77809310
:10A690003101809131018F7E809331011092300120
:10A6A0008091E70D9091E80D0E9449B01092D30D72
:10A6B0001092D20A83E020C08091D20A8823F1F060
:10A6C0008091930D9091940D04D9809131018F77F1
:10A6D00080933101809131018F7E809331011092FE
:10A6E00030018091E90D9091EA0D0E9449B01092DD
:10A6F000D30D1092D40A81E080930F028091DA0D7D
:10A700009091DB0DCF910C94A05EAF92BF92CF924F
:10A71000DF92EF92FF920F931F93CF93DF937C0111
:10A720006B015A01D0E0C0E08D2F90E0F701A181CC
:10A73000B2818A159B05D0F4F601E80FF91F6081FC
:10A7400004E510E821E03327C6270C0F111D211D59
:10A75000311D2BBFF801C791ED91FC91119701902C
:10A76000F081E02DCD011995DF5FDECFED91FC91F9
:10A7700011970190F081E02D6C2FCD01DF91CF91E9
:10A780001F910F91FF90EF90DF90CF90BF90AF900F
:10A790001994CF93DF9300D01F921F92CDB7DEB7ED
:10A7A000FE01319625E0DF011D922A95E9F724E8A4
:10A7B000298325E52C832AE22D836A834B8345E098
:10A7C00050E0BF01A2DF65E070E080E090E081DA58
:10A7D00080E00F900F900F900F900F90DF91CF912E
:10A7E0000895EF92FF921F93CF93DF931F92CDB7FF
:10A7F000DEB77C01162FFC01618172810E94D57643
:10A8000065E070E080E090E064DA42E462E4C70171
:10A81000C0DF412F60E0C701BCDF811162C040E0B2
:10A8200061E0C701B6DF81115CC040E062E0C701B2
:10A83000B0DF811156C046E062E0C701AADF811196
:10A8400050C040E063E0C701A4DF81114AC040E08E
:10A8500064E0C7019EDF11E0811110E040E065E097
:10A86000C70197DF811101C01F5F40E066E0C701AB
:10A8700090DF811101C01F5F40E067E0C70189DF01
:10A88000811101C01F5F40E068E0C70182DF8111D4
:10A8900001C01F5F40E069E0C7017BDF811101C09B
:10A8A0001F5F44E06AE0C70174DF811101C01F5FD0
:10A8B00044E06AE0C7016DDF811101C01F5F62E300
:10A8C00070E080E090E005DA82E8898341E050E0C2
:10A8D000BE016F5F7F4FC70118DF81E0183011F0B4
:10A8E000111180E00F90DF91CF911F91FF90EF90B9
:10A8F0000895CF93DF9300D01F92CDB7DEB72AEA39
:10A900002983FC0120812A836B834C8344E050E03F
:10A91000BE016F5F7F4FF9DE0F900F900F900F9089
:10A92000DF91CF9108953FB7F89420E0822F90E017
:10A93000841795079CF4FC01EE0FFF1FEE53F24FB6
:10A94000A081B181880F991FFB01E80FF91FCD018C
:10A9500096958795918380832F5FE8CF3FBF1092B4
:10A96000E30D08952F923F925F926F927F928F92A4
:10A970009F92AF92CF92DF92EF92FF920F931F932D
:10A98000CF93DF931F921F92CDB7DEB76DB67EB621
:10A990000E9441630E9436630E948D63029709F012
:10A9A00025C20E947863882309F41AC2C090DC0D86
:10A9B000D090DD0DE090DA0DF090DB0DB601C7010F
:10A9C0000E94295E8823F1F0F701E250FE4F00E07B
:10A9D00010E0819191918C159D0571F40E941A6E81
:10A9E000000F111F000F111FF701E00FF11F60830F
:10A9F00071838283938308C00F5F1F4F0E3111054F
:10AA000041F702C00E9461641092D50AEDB6FEB60D
:10AA10004091D80A5091D90ACA01880F991F2DB7C1
:10AA20003EB7281B390B0FB6F8943EBF0FBE2DBFA3
:10AA30000DB71EB70F5F1F4F8091DB0A823061F0A8
:10AA4000833021F1813009F070C0B8018091E50DAB
:10AA50009091E60D68DF33C03FB7F89420E0822F75
:10AA600090E08417950774F4880F991FF801E80F98
:10AA7000F91FDC01A551B24F8D919C919183808388
:10AA80002F5FEDCF3FBF10920B0E19C03FB7F89468
:10AA900020E0822F90E08417950774F4880F991FA7
:10AAA000F801E80FF91FDC01AB56B24F8D919C9174
:10AAB000918380832F5FEDCF3FBF1092E20D20E0A6
:10AAC0006AE071E0822F90E04091D80A5091D90A53
:10AAD0008417950754F5689FF001699FF00D1124C4
:10AAE000E65AFF4EA085B1858C918823E1F0A081C4
:10AAF000B1813C91C801830F911D830F911DDC0131
:10AB000012978D919C91A281B3814D915C91119787
:10AB10000480F581E02D4817590711F4108203C015
:10AB200070838D939C932F5FCDCF0FB6F894FEBEAC
:10AB30000FBEEDBE80915411882321F083E591E191
:10AB40000E94A96380915E11882321F08DE591E137
:10AB50000E94A96380916811882321F087E691E122
:10AB60000E94A96380917211882321F081E791E10D
:10AB70000E94A9638091D60A882309F465C0809158
:10AB80006811811105C080917211882309F450C0A9
:10AB900080916B1190916C11E0916F11F091701197
:10ABA000238134812817390724F48085811109C055
:10ABB0000EC0218132818217930734F48085811180
:10ABC00006C088E090E005C080E190E002C080E22D
:10ABD00090E02091751130917611E0917911F0910A
:10ABE0007A11438154814217530724F4208522238C
:10ABF00049F00AC041815281241735073CF4208571
:10AC0000222311F0816003C0846001C08260209122
:10AC10004E1130914F112817390719F41092501125
:10AC200007C090934F1180934E1181E08093501193
:10AC300080914E1190914F11429709F4DBC081E051
:10AC40008093741180936A11EBEFF0E18EEF90E145
:10AC50009A83898398EE892E93E0992E55245394F4
:10AC6000CF010197DC018C91882309F4ACC0E4800A
:10AC7000F580D70117968C911797882309F4A3C004
:10AC80008081882309F49FC04181528118966C917C
:10AC90008401041B150B101611061CF08A01085EB6
:10ACA000134020E030E022242394312C8FE097E2FF
:10ACB000A12CC62ED12C2C143D04ACF56430A9F087
:10ACC00040F4623071F0633019F5C9018C539A4F2A
:10ACD00013C0653071F06630D9F4C9018A559A4FB6
:10ACE0000BC0C90186539A4F07C0C90184549A4FBB
:10ACF00003C0C9018E549A4FDC0112968D919C912C
:10AD00001397841B950B97FF03C09195819591092B
:10AD10008017910714F4A22C8C01BFEF2B1A3B0A69
:10AD20002E5F3F4FC8CF81E08A0DD70119969C91C5
:10AD30009923F1F1643099F028F4623041F06330E6
:10AD400049F036C06530A1F06630D9F031C08130AD
:10AD500021F52DC0813049F1833051F51EC081307D
:10AD600011F1823011F1833011F1843009F515C0F1
:10AD70008130B9F08230B9F08430C9F08530C1F447
:10AD80000CC0813061F0823061F0833061F084303A
:10AD900061F0853061F0863059F481E009C086E0C9
:10ADA00007C085E005C084E003C083E001C082E005
:10ADB000A981BA819C91981302C0108204C050826C
:10ADC000A981BA818C93379629813A81295F3F4FB7
:10ADD0003A83298331E1EF34F30709F041CF04C00E
:10ADE0000E944D630E94616481E060C00E944D63D7
:10ADF00080E05CC0E0905111F09052111E141F04CD
:10AE00000CF04FC0809169110091DA0D1091DB0DAB
:10AE10006091D60D7091D70D8823A1F081E08093C9
:10AE20006A11C80116D7811113C0A701FF0C660B68
:10AE3000770B2BE83DE5C80173D79093D70D80932E
:10AE4000D60D06C0C80105D7811102C010926A1143
:10AE5000809173110091DA0D1091DB0D6091D40D8A
:10AE60007091D50D8823C1F081E080937411C801E1
:10AE7000F0D68111E9CE4091511150915211052E19
:10AE8000000C660B770B28E83DE5C80149D7909385
:10AE9000D50D8093D40DD8CEC801DBD68111D4CE88
:10AEA00002C010926A1110927411CECE0FB6F894AF
:10AEB0007EBE0FBE6DBE0F900F90DF91CF911F91A0
:10AEC0000F91FF90EF90DF90CF90AF909F908F9079
:10AED0007F906F905F903F902F9008951F920F92F8
:10AEE0000FB60F9211240BB60F922F933F934F93EF
:10AEF0008F939F93EF93FF938091840090918500AF
:10AF00002091BE0D3091BF0D821B930B20918400C8
:10AF1000309185003093BF0D2093BE0D803727E11F
:10AF2000920770F19093C10D8093C00D8091DE0D5A
:10AF30009091DF0D029751F49091D20D8091E40D24
:10AF400098133CC081E08093E30D3EC08091DE0DFC
:10AF50009091DF0D892B49F481E090E09093DF0D13
:10AF60008093DE0D1092BD0D2FC08091DE0D90916B
:10AF7000DF0D019761F58091D20D8430D8F527C09F
:10AF80002091D20D283008F047C09C012C5D35403F
:10AF9000293B3B4068F4E091D20DEF5FE093D20D86
:10AFA000F0E0EE0FFF1FE054F24F9183808334C036
:10AFB0008091DE0D9091DF0D029771F583E090E0B6
:10AFC0009093DF0D8093DE0D1092D20D25C08091FD
:10AFD000DE0D9091DF0D0397B9F79091D20D80911E
:10AFE000E40D9813F1CF8091E40D843068F382E092
:10AFF00090E0E6CF8091BD0D8F5F8093BD0D8630D0
:10B0000018F382E090E09093DF0D8093DE0D809145
:10B01000D20D8093E40DD8CFFF91EF919F918F9146
:10B020004F913F912F910F900BBE0F900FBE0F903D
:10B030001F9018950F931F938091B50D81110DC02E
:10B040000E941A6E6093B10D7093B20D8093B30D90
:10B050009093B40D81E08093B50D0E941A6E00911B
:10B06000B10D1091B20D2091B30D3091B40DDC01F2
:10B07000CB01801B910BA20BB30B893E9340A10522
:10B08000B105A8F08AE30E94F04C892B11F060E032
:10B0900001C061E08AE30E94184D0E941A6E60931D
:10B0A000B10D7093B20D8093B30D9093B40D1F91B9
:10B0B0000F9108950F931F930E941A6E00918B0DAC
:10B0C00010918C0D20918D0D30918E0DDC01CB01F6
:10B0D000801B910BA20BB30B85339142A105B105E7
:10B0E00018F081E080938A0D1F910F91A3CFFC018E
:10B0F00080E090E06150710977FD18C02191022E27
:10B10000000C330B322F22278227932728E0AC0133
:10B11000440F551F97FF06C0CA0131E2832730E173
:10B12000932701C0CA01215091F7E4CF08950895F3
:10B13000089508950895CF93DF93EC0121E03FEF48
:10B140003B872A878FEF90E09D878C871F861E861E
:10B15000398B288B9B8B8A8B1D8A1C8A61E08AE045
:10B160000E94474D61E086E00E94474D61E08DE21C
:10B170000E94474D61E08DE00E94474D61E08BE009
:10B180000E94474D61E08EE20E94474D8A819B817B
:10B190008830910529F410922B0110922A0106C0E3
:10B1A000099721F41092290110922801DF91CF9183
:10B1B00008950F931F93CF93DF938C01FC01178A9F
:10B1C000168AEC01699640E068E0CE0192DB4FE719
:10B1D00066E0CE018EDB40E06CE0CE018ADB4FE71B
:10B1E00067E0CE0186DB0E941A6EF801648F758FCE
:10B1F000868F978FDF91CF911F910F910895CF93F5
:10B20000DF93EC018091D90D811109C06A8D7B8D8E
:10B21000CE0149960E94D57681E08093D90D21E830
:10B220003FEF3B872A878FE790E09D878C871F86BB
:10B230001E86398B288B9B8B8A8B1D8A1C8ADF91FB
:10B24000CF9108950F931F93CF93DF93EC011F8A43
:10B250001E8A8C01075E1F4F40E060E0C8010E941B
:10B26000066240E064E0C8010E9406620E941A6E15
:10B270006C8F7D8F8E8F9F8FDF91CF911F910F915C
:10B2800008950F931F93CF93DF93EC018091D80D16
:10B29000811112C00A8D1B8D6AEA70E0C8010E94FC
:10B2A0005686D801ED91FC910284F385E02DC8010A
:10B2B000199581E08093D80D4AE06EE0CE01499661
:10B2C0000E94066221E83FEF3B872A878FE790E0E4
:10B2D0009D878C871F861E86398B288B9B8B8A8B3C
:10B2E0001D8A1C8ADF91CF911F910F9108950F93B2
:10B2F0001F93CF93DF93EC011F8A1E8A8C01075E98
:10B300001F4F40E060E0C8010E94C96140E064E076
:10B31000C8010E94C9610E941A6E6C8F7D8F8E8F4A
:10B320009F8FDF91CF911F910F9108950F931F93DE
:10B33000CF93DF93EC01E8A1F9A180819181A281F3
:10B34000B3818E01075E1F4F81159649A105B10596
:10B3500009F451C040E056E960E070E082E997E00E
:10B360000E94E56664E170E080E090E00E94694E32
:10B37000E8A1F9A180819181A281B38181152BE49B
:10B380009207A105B105E9F068F4803629E092073B
:10B39000A105B105A1F080389542A105B105B9F428
:10B3A00042E012C0811521EE9207A105B10559F0C6
:10B3B0008115924CA140B10551F445E005C041E032
:10B3C00003C043E001C046E06FE0C801E2D782E974
:10B3D00097E00E94B547E8A1F9A1408151816281BF
:10B3E000738182E997E00E94E56664E170E080E0A5
:10B3F00090E00E94694E4AE06EE0C801CAD741E081
:10B4000067E1C801C6D74AA168E1C801C2D721E8EF
:10B410003FEF3B872A878FE790E09D878C871F86C9
:10B420001E86398B288B9B8B8A8B1D8A1C8ADF9109
:10B43000CF911F910F9108950C945D86EF92FF922A
:10B440000F931F93CF93DF93EC016623E1F0262F38
:10B45000653608F024E60A891B89E888F988D8014E
:10B46000AE19BF0930E00E94A8AE28EC30E040E001
:10B4700050E00E9429B4E20EF31EFB86EA86021B0E
:10B48000130B1D870C87DF91CF911F910F91FF90B8
:10B49000EF900895CF93DF93CDB7DEB7A2970FB6A5
:10B4A000F894DEBF0FBECDBF80310CF080E128ECF8
:10B4B00035E13A83298320EC35E13C832B8328EB6B
:10B4C00035E13E832D8320EB35E138872F8328EA51
:10B4D00035E13A87298720EA35E13C872B8728E93F
:10B4E00035E13E872D8720E935E1388B2F8722E82B
:10B4F00035E13A8B298B20E735E13C8B2B8B23E51B
:10B5000035E13E8B2D8B2EE335E1388F2F8B24E3F5
:10B5100035E13A8F298F2AE235E13C8F2B8F2DE1DF
:10B5200035E13E8F2D8F21E135E138A32F8F29E0C2
:10B5300035E13AA329A3E82FEE0FFF0BEC0FFD1F17
:10B5400081819281A2960FB6F894DEBF0FBECDBF67
:10B55000DF91CF9108958F929F92AF92BF92CF9239
:10B56000DF92EF92FF920F931F93DC0118968D915B
:10B570009C9119971E96CD90DC901F9768177907BC
:10B5800009F456C05896FC9058974C01092E000CAF
:10B59000AA08BB088B01072E000C220B330B861761
:10B5A00097073CF41696ED91FC911797FF2039F020
:10B5B00015C01496ED91FC911597FF2079F00D2C94
:10B5C000000CEE08FF08A9019801281939094A0959
:10B5D0005B091C966D917C911D970EC00D2C000C83
:10B5E000EE08FF08A9019801281939094A095B09E1
:10B5F0001A966D917C911B97CB01770FAA0BBB0B11
:10B60000BC01CD016C197D098E099F090E9464AEB1
:10B610008F01FF0F220B330BA9019801281939095B
:10B620004A095B090E94FDB3C20ED31EE41EF51E3B
:10B63000C6011F910F91FF90EF90DF90CF90BF90C8
:10B64000AF909F908F9008950F931F93CF93DF93A8
:10B650008C01FC01778B668B7EDFEC01F801828127
:10B66000938188309105D1F4D7FF06C060E08AE06D
:10B670000E94184D61E005C061E08AE00E94184D0B
:10B6800060E086E00E94184DD7FF03C0D195C195B8
:10B69000D109D0932B01C0932A011BC00997C9F48B
:10B6A000D7FF06C060E08DE00E94184D61E005C044
:10B6B00061E08DE00E94184D60E08BE00E94184D23
:10B6C000D7FF03C0D195C195D109D0932901C0936B
:10B6D0002801DF91CF911F910F910895EF92FF9272
:10B6E0000F931F93CF93DF938C01FC01778B668BB5
:10B6F00032DFEC01F801828193818830910529F5D0
:10B700007801F9E1EF0EF11CD7FF06C06AE0C138FD
:10B710008FEFD80754F001C068E02C2F9D2FC03860
:10B72000D1052CF02FE790E002C021E89FEF422FD7
:10B73000592F57FF03C0519541955109C701D9D8D9
:10B74000CD2B59F54FE766E026C0099731F5780112
:10B75000E9E1EE0EF11CD7FF06C06EE0C138FFEF45
:10B76000DF0754F001C06CE02C2F9D2FC038D105AD
:10B770002CF02FE790E002C021E89FEF422F592FD5
:10B7800057FF03C0519541955109C701B2D8CD2B40
:10B7900021F44FE767E0C701ACD80E941A6EF801A8
:10B7A000648F758F868F978FDF91CF911F910F9147
:10B7B000FF90EF9008950F931F93CF93DF93EC01C9
:10B7C0000E941A6E0C8D1D8D2E8D3F8DDC01CB01DC
:10B7D000801B910BA20BB30B853F9140A105B105D6
:10B7E00040F06E897F89CE01DF91CF911F910F913B
:10B7F00075CFDF91CF911F910F910895CF93DF9374
:10B80000EC017F8B6E8BA7DE9C018A819B81883047
:10B810009105C1F437FF06C061E021388FEF38078A
:10B820004CF001C060E0A901203831052CF04FE751
:10B8300050E002C041E85FEF57FF1FC051954195AE
:10B8400051091BC00997E1F4922F832F203831054D
:10B8500014F09FE780E0492F582F41388FEF5807A9
:10B8600014F441E85FEF57FF03C05195419551092A
:10B87000632F661F6627661F6C5FCE014996C6D58B
:10B880000E941A6E6C8F7D8F8E8F9F8FDF91CF916C
:10B8900008950F931F93CF93DF93EC010E941A6ECC
:10B8A0000C8D1D8D2E8D3F8DDC01CB01801B910BEE
:10B8B000A20BB30B853F9140A105B10540F06E8905
:10B8C0007F89CE01DF91CF911F910F9197CFDF91AB
:10B8D000CF911F910F910895CF93DF93EC017F8B50
:10B8E0006E8B39DE9C018A819B8188309105C1F481
:10B8F00037FF06C061E021388FEF38074CF001C0F8
:10B9000060E0A901203831052CF04FE750E002C07B
:10B9100041E85FEF57FF1FC05195419551091BC08A
:10B920000997E1F4922F832F2038310514F09FE717
:10B9300080E0492F582F41388FEF580714F441E821
:10B940005FEF57FF03C0519541955109632F661F63
:10B950006627661F6C5FCE0149961BD50E941A6E42
:10B960006C8F7D8F8E8F9F8FDF91CF9108950F9376
:10B970001F93CF93DF93EC010E941A6E0C8D1D8DE7
:10B980002E8D3F8DDC01CB01801B910BA20BB30BE5
:10B99000853F9140A105B10540F06E897F89CE01B8
:10B9A000DF91CF911F910F9197CFDF91CF911F9191
:10B9B0000F910895482F50E095E1899FF0011124DF
:10B9C000E558FE4E2181328180859185280F391FEF
:10B9D000838194818217930728F0858196812817A7
:10B9E0003907E8F485E1849FF001859FF00D11246B
:10B9F000E558FE4E858196812817390728F525815F
:10BA0000368185E1849FF001859FF00D1124E55872
:10BA1000FE4E8285823019F411861086128685E1E9
:10BA2000849FF001859FF00D1124E558FE4E32836E
:10BA300021838091840090918500280F391F3093D5
:10BA40008900209388000895838194818217930749
:10BA5000C0F623813481D5CF8091D50A811157C09A
:10BA6000E0915B11F0915C11858196819093581162
:10BA70008093571110925A1110925911E09165114B
:10BA8000F091661185819681909362118093611186
:10BA90001092641110926311E0916F11F091701186
:10BAA0008581968190936C1180936B1110926E1129
:10BAB00010926D11E0917911F0917A118581968142
:10BAC00090937611809375111092781110927711DE
:10BAD00082E190E090934F1180934E1181E080932A
:10BAE000541180935E11809368118093721180933A
:10BAF000501180E090E021E0FC01E650FF4E2183F0
:10BB0000079684359105C1F781E08093D50A0895A1
:10BB100010927411089510926A11089577FF03C06E
:10BB200071956195710920E0462F6EE20C94C86909
:10BB30006DE20C94106A6CE20C94106A4F925F9262
:10BB40006F927F928F929F92AF92BF92CF92DF922D
:10BB5000EF92FF920F931F93CF93DF936C01A4ECAE
:10BB6000CA1AADEFDA0AD601ED91FC917E970CF07E
:10BB70005DC0FC01E858FF4F812C912CA191B1913F
:10BB8000AB2B21F42115310549F450C0BFEF8B1ABE
:10BB90009B0AAEE18A16910489F748C0EC01540172
:10BBA000AA0CBB1CAA0CBB1CAC0EBD1EF501EC54B0
:10BBB000FF4F40835183628373837401EE0CFF1C3B
:10BBC000EC0EFD1EF701E858FF4F31832083EC5443
:10BBD000FF4F11830083BE01680D791DFB01EC55F9
:10BBE000FE4F81E080830E941A6EF50160837183AD
:10BBF00082839383C65CDD4F88819981F701E2508F
:10BC0000FE4F91838083D6012D913C9111972F5F38
:10BC10003F4F2D933C939C012F5F3F4F121613060D
:10BC200014F021E030E03983288302C08FEF9FEFCA
:10BC3000DF91CF911F910F91FF90EF90DF90CF9008
:10BC4000BF90AF909F908F907F906F905F904F903C
:10BC50000895DC01A250BE4F20E030E04D915D918F
:10BC60004617570739F4280F391FF901EC55FE4FD5
:10BC7000808108952F5F3F4F2E31310579F780E0A5
:10BC80000895CF93DF93EC01C45CDD4FA881B981A7
:10BC9000109709F442C0FC01E250FE4F20E030E072
:10BCA000419151914617570799F5A901440F551F26
:10BCB000480F591FFA01E858FF4F60817181672BC7
:10BCC00061F111821082FC01E20FF31FEC55FE4F6F
:10BCD0001082FA01EE53FE4F11821082235D3F4F16
:10BCE000220F331F220F331FFC01E20FF31F1082BC
:10BCF000118212821382FA01E859FE4F11821082DA
:10BD0000EA56FF4F118210821197B983A88305C0AC
:10BD10002F5F3F4F2E31310519F6DF91CF910895F6
:10BD20000F931F9301E010E009DF1F910F91089519
:10BD30000F931F9300E010E001DF1F910F91089512
:10BD40002F923F924F925F926F927F928F929F922B
:10BD5000AF92BF92CF92DF92EF92FF920F931F9319
:10BD6000CF93DF9300D000D0CDB7DEB78C010E9417
:10BD70001A6E98012E533E4F3C832B831E830D83F6
:10BD8000D801AC55BE4FBA83A9831801B2E02B1A73
:10BD9000BEEF3B0AF901AA24A394B12C32E0832E12
:10BDA000912C118210829F012A543140D9012D918A
:10BDB0003C91232B09F44DC0AD81BE812D913D9165
:10BDC0004D915C9113977D01B4EBEB0EF11CD70103
:10BDD000CD90DD90ED90FC902B013C01421A530A6E
:10BDE000640A750A4C145D046E047F0490F1C20E5F
:10BDF000D31EE41EF51EAD81BE81CD92DD92ED9283
:10BE0000FC921397A981BA812C91222311F19F01F1
:10BE100026593109D9012D913C912115310519F48B
:10BE2000B182A08216C07F01BAE5EB1AF108D701F2
:10BE30004D915C911197421753075CF4B182A08237
:10BE40004F5F5F4F4D935C934217530714F09182FD
:10BE5000808232962D813E812C5F3F4F3E832D8321
:10BE6000A981BA811196BA83A983E215F30509F075
:10BE700098CFEB81FC8181919191FC83EB838130A0
:10BE8000910599F00297C9F4EB81FC81EC54F140E3
:10BE90000190F081E02D1995AB81BC81DA966D910E
:10BEA0007C91DB97C801EDDE08C0EB81FC81EC548E
:10BEB000F1400190F081E02D19952B813C812215F4
:10BEC0003305B9F626960FB6F894DEBF0FBECDBF88
:10BED000DF91CF911F910F91FF90EF90DF90CF9066
:10BEE000BF90AF909F908F907F906F905F904F909A
:10BEF0003F902F9008956E3E22E0720738F06B3C21
:10BF000098E0790728F06AEC78E002C06EEE72E003
:10BF1000660F771F9FB7F89425E1829FF0011124E7
:10BF2000E558FE4E748363839FBF08956E3E22E002
:10BF3000720738F06B3C98E0790728F06AEC78E0FB
:10BF400002C06EEE72E0660F771F9FB7F89425E18E
:10BF5000829FF0011124E558FE4E768365839FBFD2
:10BF60000895660F771F282F30E095E1899FF00133
:10BF70001124E558FE4E858196816817790718F4DB
:10BF80006581768107C0838194818617970710F4B5
:10BF9000638174818FB7F89495E1929FF001939F2C
:10BFA000F00D1124E558FE4E728361838FBF089512
:10BFB000982F8FB7F89425E1929FF0011124E5584E
:10BFC000FE4E21E027838FBF41B121E030E0B9016F
:10BFD00002C0660F771F9A95E2F7CB01842B81B9D7
:10BFE00008958A3058F49FB7F89425E1829FF001B4
:10BFF0001124E558FE4E118610869FBF08951F93A9
:10C00000CF93DF9325E1829FC0011124EC01C55835
:10C01000DE4E8A8581110FC01FB7F89481E08A87B0
:10C0200089899A899A8389830E941A6E6B877C8793
:10C030008D879E871FBFDF91CF911F910895CF936A
:10C04000DF938A30D0F56233710538F061369DE6B2
:10C05000790728F060E67DE602C062E370E0D42F45
:10C06000C82F80E090E00E94B8B220E030E04AE7BC
:10C0700054E40E9413AF20E030E04CE852E40E9408
:10C0800019B39B01AC0160E070E08AEF94E40E9478
:10C0900013AF0E947BAF9B01DD2321F022273327C2
:10C0A000261B370B8FB7F89495E1C99FF001112437
:10C0B000E558FE4E318720878FBFDF91CF910895DD
:10C0C0008A3008F418CF08958A3008F42FCF0895E5
:10C0D0008A3058F495E1899FF0011124E558FE4E0D
:10C0E0008181928196958795089580E090E00895EA
:10C0F0008A3008F436CF08951F920F920FB60F9230
:10C1000011240BB60F920F931F932F933F934F93CE
:10C110005F936F937F938F939F93AF93BF93CF93CF
:10C12000EF93FF9380912E0E893048F010922E0EDF
:10C1300080912A12882399F0809123120DC0E091FA
:10C140002E0EE15025E1E29FF0011124E558FE4E4C
:10C150008781882321F0808192B1892782B9E0917B
:10C160002E0E85E1E89FF0011124E558FE4E8781EF
:10C17000882321F0808192B1892B82B9E0912E0E23
:10C18000C5E1CE9FF0011124E558FE4E80859185D2
:10C19000892B09F04DC0E0912E0ECE9FF0011124A5
:10C1A000E558FE4E8285813009F060C00E941A6E0B
:10C1B000E0912E0ECE9FF0011124E558FE4E03852E
:10C1C000148525853685E0912E0ECE9FF001112431
:10C1D000E558FE4E0784F089E02DAB01BC01401B01
:10C1E000510B620B730BCF01A0E0B0E084179507F1
:10C1F000A607B707D8F5E0912E0EA0912E0ECA9F84
:10C20000D0011124A558BE4E53968D919C91549700
:10C21000CE9FF0011124E558FE4E91878087E09172
:10C220002E0ECE9FF0011124E558FE4E82E082874B
:10C2300080912E0EBFDB80912E0E8F5F80932E0E8D
:10C24000FF91EF91CF91BF91AF919F918F917F918E
:10C250006F915F914F913F912F911F910F910F908F
:10C260000BBE0F900FBE0F901F901895E0912E0EF1
:10C27000809184009091850025E1E29FF0011124D6
:10C28000E558FE4E21813281820F931F90938900E1
:10C2900080938800D0CF1F93CF93DF9380912D0E92
:10C2A000811173C010922E0E9FB7F89485E128EB90
:10C2B0003BE04CED55E064E971E1A1E0B0E0E091D4
:10C2C0002E0EE93008F052C0E0912E0E8E9FF00144
:10C2D0001124E558FE4E32832183E0912E0E8E9F6D
:10C2E000F0011124E558FE4E56834583E0912E0E51
:10C2F0008E9FF0011124E558FE4E74836383E09114
:10C300002E0EF0912E0EED0101C0CC0FFA95EAF73A
:10C310008E9FF0011124E558FE4EC083E0912E0E51
:10C320008E9FF0011124E558FE4E1782E0912E0EEB
:10C330008E9FF0011124E558FE4E11861086E09183
:10C340002E0E8E9FF0011124E558FE4E1286E091CC
:10C350002E0E8E9FF0011124E558FE4E148A138A8A
:10C36000E0912E0EEF5FE0932E0EA9CF9FBF8FB707
:10C37000F89420EA3FE03093251220932412109283
:10C3800023128FBF81E080932D0EDF91CF911F91FB
:10C3900008950F931F93CF93DF938C01C62FD42F53
:10C3A000DC0111968D919C911297DC01ED91FC912D
:10C3B0000190F081E02DD8016C911995F8018181EF
:10C3C0009281DC01ED91FC910190F081E02D6C2FC8
:10C3D0001995F80181819281DC01ED91FC91019028
:10C3E000F081E02D6D2F1995F80180816C2F70E0A0
:10C3F000680F711D6D0F711D6F7777278181928195
:10C40000DF91CF911F910F910C9456860F931F933C
:10C41000CF93DF938C01C62FD42FDC0111968D9121
:10C420009C911297DC01ED91FC910190F081E02D3F
:10C43000D8016C911995F80181819281DC01ED910F
:10C44000FC910190F081E02D6C2F1995F80181810C
:10C450009281DC01ED91FC910190F081E02D6D2F36
:10C460001995F80180816C2F70E0680F711D6D0FB8
:10C47000711D6F77772781819281DF91CF911F9115
:10C480000F910C9456864F925F926F927F92AF926B
:10C49000BF92CF92DF92EF92FF921F93CF93DF93E1
:10C4A000DD24D39445E0C42E52E0A52EB12CC3E088
:10C4B000D0E0EE24E394F12C8091110E9091120EB5
:10C4C000DC01ED91FC910480F581E02D1995892B1B
:10C4D00009F4BEC0109130018091110E9091120E9E
:10C4E000DC01ED91FC910680F781E02D199596B362
:10C4F000B39A20918400309185002059384E3093B2
:10C500008D0020938C00212F2C7139F010922C0E6D
:10C51000D093100EC0930F0ECFCF93FB992790F9B5
:10C52000E0912C0EE11116C0992331F28F3021F6E3
:10C53000D0922C0E8093130E80910F0E9091100EBE
:10C54000892B09F0B9CFF092100EE0920F0E1092E5
:10C550000E0EB2CF9111DACF91E09E0F90932C0E78
:10C56000F0E0ED5EF14F8083993109F0A5CF8111A4
:10C570006CC080912A0E82FF05C0D093100EC0932C
:10C580000F0E63C083FDF9CF80910F0E9091100EB6
:10C59000019739F480910E0E8F5F80930E0E8430D8
:10C5A00020F0B092100EA0920F0E80910D0E8F5FB2
:10C5B00080930D0E90910C0E981708F044C0D09205
:10C5C0000B0EABEEBDE0E4E1FEE040E050E0BA016E
:10C5D00010E0CF01FC011B3098F401964080512CF3
:10C5E000612C712C012E04C0440C551C661C771C58
:10C5F0000A94D2F74429552966297729185FEACF8A
:10C600009A013770205E3340C29EC001C39E900DD8
:10C61000112497FD079623E0959587952A95E1F7D4
:10C6200084529A4F8D939D931B503BE0769567956E
:10C63000579547953A95D1F78EE0AB30B80749F654
:10C6400010920D0E02C010920B0E10922C0E34CFD1
:10C65000DF91CF911F91FF90EF90DF90CF90BF902F
:10C66000AF907F906F905F904F9008958091DB0A1C
:10C67000833031F48091E90D9091EA0D0C94887A21
:10C6800008958091DB0A823029F48091E70D909122
:10C69000E80DF9CE0895F5DFE9CF1092541110920C
:10C6A0005E1110926811109272111092501180E078
:10C6B00090E0FC01E650FF4E11820796843591050B
:10C6C000C1F708958091DB0A823039F0833049F058
:10C6D000813049F48091E40D01C080E18093D70A54
:10C6E00004C08EE0FBCF1092D70A8091D70A08953C
:10C6F0008091DB0A823039F0833049F0813059F47F
:10C700008091E30D0895BDDF80910B0E0895AEDF9B
:10C710008091E20D089580E008958091DB0A8230D7
:10C7200049F0833069F0813089F48091DE0D909179
:10C73000DF0D0895A6DF80910F0E9091100E0895E1
:10C7400095DF8091E00D9091E10D089581E090E0FA
:10C7500008958F929F92AF92BF92CF92DF92EF9205
:10C76000FF921F93CF93DF93EC0111E08E819F81A5
:10C77000892B09F410E02C813D81E885F985C5807D
:10C78000D680878190E0A601480F591F24173507EE
:10C7900064F180850D2C000CEE08FF08A901330F11
:10C7A000660B770B0380F481E02D9A01AB012C1905
:10C7B0003D094E095F09882329F0A1E0BFEF0E94DF
:10C7C00025B404C0AFEFB0E00E9419B44F01FF0FD1
:10C7D000AA08BB08A50194012C193D094E095F095F
:10C7E0000E94FDB33F832E834BC0A601481B590B0B
:10C7F000421753070CF43FC080850D2C000CEE0847
:10C80000FF08A901330F660B770B81809280092CFA
:10C81000000CAA08BB089A01AB01281939094A097A
:10C820005B09882399F0A1E0BFEF0E9425B4A7011E
:10C830009601281939094A095B090E94FDB3DA01FA
:10C84000C90181509F4FAF4FBF4F12C0AFEFB0E053
:10C850000E9419B4A7019601281939094A095B09F0
:10C860000E94FDB3DA01C9018F5F9109A109B109E5
:10C870009F838E8305C01F821E82111101C0198201
:10C880008E819F81009789F08F3F910519F014F0F8
:10C890008FEF90E081305FEF950714F481E09FEF18
:10C8A0009F838E8381E018271A83DF91CF911F9198
:10C8B000FF90EF90DF90CF90BF90AF909F908F90C0
:10C8C0000895CF93DF93C091DA0DD091DB0D609185
:10C8D000DC0D7091DD0DCE01BCD981110CC02CE2B4
:10C8E0003DE54CE251E060E070E0CE0119DA909352
:10C8F000DD0D8093DC0DDF91CF91089508950895AB
:10C90000089508950895623039F0633041F0613040
:10C9100041F44093700E089540936F0E0895409334
:10C920006E0E0895623069F06330A1F06130D1F489
:10C930005093740E4093730E3093760E2093750EC1
:10C94000089550937B0E40937A0E30937D0E209382
:10C950007C0E08955093840E4093830E3093860E80
:10C960002093850E08950895089508952091880EC6
:10C97000211102C0FC01628308952091880E2111CB
:10C9800002C0FC01648308952091880E211102C029
:10C99000FC0163830895089508958091880E8111A4
:10C9A00002C00C94FC700895089580E008950895E5
:10C9B000089508950895089508958091880E81112D
:10C9C00004C08FE090E00C94FA7108958091880E75
:10C9D000811121C0633091F028F4613049F0623058
:10C9E00051F00895653081F060F0663081F008956F
:10C9F00089E090E00EC08AE090E00BC08BE090E010
:10CA000008C08CE090E005C08DE090E002C08EE0B0
:10CA100090E00C94FA7108952091880E211108C0BD
:10CA2000FC018481882321F082E090E00C94FA716B
:10CA300008952091880E211108C0FC01838188236C
:10CA400021F081E090E00C94FA7108958091880EB5
:10CA5000811104C08BE090E00C94FA7108958091EC
:10CA6000880E811105C060E080E190E00C9438727E
:10CA700008958091880E811105C060E08FE090E0FC
:10CA80000C94387208958091880E811127C063300C
:10CA9000A1F028F4613049F0623059F00895653012
:10CAA000A1F078F06630A9F0089560E089E090E0A8
:10CAB00013C060E08AE090E00FC060E08BE090E09F
:10CAC0000BC060E08CE090E007C060E08DE090E09B
:10CAD00003C060E08EE090E00C943872089580917D
:10CAE000880E811127C06330A1F028F4613049F02D
:10CAF000623059F008956530A1F078F06630A9F001
:10CB0000089561E089E090E013C061E08AE090E080
:10CB10000FC061E08BE090E00BC061E08CE090E042
:10CB200007C061E08DE090E003C061E08EE090E03E
:10CB30000C94387208952091880E211109C0FC01CF
:10CB40008281882329F061E088E090E00C943872BB
:10CB500008952091880E211109C0FC018481882349
:10CB600029F061E082E090E00C9438720895209101
:10CB7000880E211109C0FC018381882329F061E01E
:10CB800081E090E00C94387208958091880E8111B4
:10CB900005C061E086E090E00C94387208958091C1
:10CBA000880E811105C060E08BE090E00C94387233
:10CBB00008958091880E811105C061E087E090E0C2
:10CBC0000C94387208958091880E811105C061E03F
:10CBD00085E090E00C94387208958091880E811160
:10CBE0002BC06091710E7091720E8091810E9091A8
:10CBF000820E47D81092770E8091880E81110BC05B
:10CC00006091780E7091790E8091810E9091820ED4
:10CC100038D810927E0E8091880E81110BC06091E1
:10CC20007F0E7091800E8091810E9091820E29D896
:10CC30001092870E1092330E08958091880E811104
:10CC400016C08091330E811112C025E833E748EBFE
:10CC50005BE060E070E08091810E9091820E60D880
:10CC60009093720E8093710E81E08093330E08953D
:10CC70008091880E882321F06CED75E081E071C908
:10CC800084E090E00C94FA718091880E882321F062
:10CC900068EE73E081E065C960E084E090E00C94A8
:10CCA00038728091880E811119C08091680E882396
:10CCB000A9F068EE73E081E054D91092680E2CEF71
:10CCC00030E748E95AE360E070E08091810E90918E
:10CCD000820E26D89093670E8093660E08956CEDB1
:10CCE00075E080E03EC924EF31E0DB010E94A8AE90
:10CCF0002FEF30E040E050E00E94FDB3CA01B901DF
:10CD000064527A4F8F4F9F4F80E02BC98091880EDD
:10CD1000882331F060ED77E081E023D90C94B6737D
:10CD200061E083E090E00C9438722091880E21112C
:10CD300003C002960C94C97308952091880E222393
:10CD400081F06FE676E080E00CD921E138E642E33D
:10CD500050E060E070E08091810E9091820E0C9422
:10CD6000905E02960C94C97380E022D981E020D9AC
:10CD70008091880E811102C082E01AD96CED75E0B5
:10CD800080E0EFD86CED75E081E0EBD88091880E03
:10CD900081110CC084E591E8A1E0BB27ABBFFC0189
:10CDA0006791769182E0DDD80C94E5700895FC01DE
:10CDB00080899189938782878289938995878487DF
:10CDC0008489958997878687089526E00C948B4CF3
:10CDD00080913B0E90913C0E916090933C0E80931D
:10CDE0003B0E089580913B0E90913C0E806890938D
:10CDF0003C0E80933B0E089580913B0E90913C0E2B
:10CE0000806190933C0E80933B0E0895FC018281DB
:10CE1000882371F08381882359F0138280913B0E1F
:10CE200090913C0E24E0822790933C0E80933B0E21
:10CE30000895FC018281882371F0838181110BC0E8
:10CE400081E0838380913B0E90913C0E84609093AF
:10CE50003C0E80933B0E0895FC018481882371F081
:10CE60008581882359F0158280913B0E90913C0E6C
:10CE700028E0822790933C0E80933B0E0895FC019E
:10CE80008481882371F0858181110BC081E08583C5
:10CE900080913B0E90913C0E886090933C0E809365
:10CEA0003B0E089580913B0E90913C0E20E282272C
:10CEB00090933C0E80933B0E089580913B0E909191
:10CEC0003C0E806290933C0E80933B0E0895DC01F3
:10CED000ED91FC910680F781E02D60E070E01994FF
:10CEE00077FF03C07195619571096F3F710519F066
:10CEF00014F06FEF70E080913B0E90913C0E8C7BB4
:10CF0000917090933C0E80933B0E80913B0E9091DC
:10CF10003C0E6F30710514F480641FC067337105D7
:10CF200014F481641AC06F3571051CF4816490613A
:10CF300014C0673871051CF4816490630EC06F3AA9
:10CF400071051CF48164906408C0673D71051CF490
:10CF50008164906502C08164906690933C0E8093DA
:10CF60003B0E089580E094E090933C0E80933B0E3E
:10CF7000089580913B0E90913C0E926090933C0EF0
:10CF800080933B0E80913B0E90913C0E8064909379
:10CF90003C0E80933B0E08950895089508950895DA
:10CFA00008950895089508950895089580E00895D6
:10CFB0000895089508950895089508950895089589
:10CFC0000895089508950895089508950895089579
:10CFD000089580E0089508950895FC0164830895FC
:10CFE000FC0162830895FC0113821482158216826B
:10CFF0001782108611860895089508950895FC01FA
:10D0000083810895FC0165830895FC01648308957C
:10D01000FC0160870895FC0166830895FC0182810C
:10D0200008956CED75E080E00C94B15FFC01128214
:10D0300013821482158261E086E10E94474D61E00F
:10D0400086E10E94184DE2E7F0E0808181608083F4
:10D0500010923C0E10923B0E08950F931F93CF93A6
:10D06000DF93EC017093820E6093810E4093880EE3
:10D0700081E090E00E94B4AF8C010DD910933E0E78
:10D0800000933D0E91E09093680E9093690E10927C
:10D09000670E1092660E10926C0E10926B0E10922C
:10D0A0006D0E10926A0E24EF31E03093740E2093CF
:10D0B000730E28EB3BE03093760E2093750E20E242
:10D0C00033E030937B0E20937A0E2CEA3DE03093D0
:10D0D0007D0E20937C0E28E037E03093840E209361
:10D0E000830E24E931E13093860E2093850E109251
:10D0F000700E10926F0E10926E0E1092770E1092AC
:10D100007E0E1092870E1092720E1092710E109277
:10D11000790E1092780E1092800E10927F0E9883E6
:10D1200099839A83DF91CF911F910F9108951F9258
:10D130000F920FB60F9211240BB60F922F933F93BD
:10D140004F935F936F937F938F939F93AF93BF930F
:10D15000EF93FF9380913A0E8F5F80933A0E9091F8
:10D16000390E891708F401C110923A0E8091380ED9
:10D1700090E08730910508F0F8C0FC018827E85955
:10D18000FE4F8F4F0C949AAE60E086E10E94184DDE
:10D1900080E48093390E81E048C061E086E10E941E
:10D1A000184D88E08093390E36C060E086E10E9419
:10D1B000184D8091360E9091370E97FF05C088E18B
:10D1C0008093390E84E031C088E08093390E83E08B
:10D1D0002CC061E086E10E94184D88E18093390EF1
:10D1E0008091350E8F5F8093350E803150F0109214
:10D1F000350E85E01AC061E086E10E94184D88E096
:10D20000EDCF8091360E9091370E880F991F909335
:10D21000370E8093360E82E008C060E086E10E94FF
:10D22000184D88E08093390E86E08093380E9DC0BB
:10D2300061E086E10E94184D80EC8093390E809168
:10D240003B0E90913C0E9093370E8093360E80915A
:10D250003B0E90913C0E91FF1DC08091340E8823AF
:10D26000B1F080913B0E90913C0E22E0922790937A
:10D270003C0E80933B0E80913B0E90913C0E80645F
:10D2800090933C0E80933B0E1092340E03C081E0CD
:10D290008093340E80913B0E90913C0E92FF0EC015
:10D2A0008091340E882339F010923C0E10923B0E80
:10D2B0001092340E03C081E08093340E80913B0EB7
:10D2C00090913C0E84FF14C08091340E882369F045
:10D2D00080913B0E90913C0E20E1822790933C0E72
:10D2E00080933B0E1092340E03C081E08093340E85
:10D2F00080913B0E90913C0E87FF13C08091340EBD
:10D30000882361F080913B0E90913C0E8058909361
:10D310003C0E80933B0E1092340E03C081E080934C
:10D32000340E80913B0E90913C0E90FF14C0809182
:10D33000340E882369F080913B0E90913C0E21E0E1
:10D34000922790933C0E80933B0E1092340E03C0B4
:10D3500081E08093340E80913B0E90913C0E90932F
:10D36000370E8093360E1092380EFF91EF91BF91D9
:10D37000AF919F918F917F916F915F914F913F916D
:10D380002F910F900BBE0F900FBE0F901F9018950E
:10D39000FF920F931F93CF93DF938C01C62FF42E30
:10D3A000D22F6AED70E0DC011A968D919C911B974B
:10D3B0000E945686F80182859385DC01ED91FC91EF
:10D3C0000190F081E02D6C2F1995F80182859385ED
:10D3D000DC01ED91FC910190F081E02D6F2D19950C
:10D3E000F80182859385DC01ED91FC910190F0813B
:10D3F000E02D6D2F1995EC2FF0E0BF0166527F4FA5
:10D400006F0D711D6D0F711D6F777727F801828584
:10D410009385DF91CF911F910F91FF900C945686C9
:10D4200020E040E0B5CF65E4FBCF68E4F9CFCF93CF
:10D43000DF93FC012381222321F0EC0161E4F0DF82
:10D440001B82DF91CF910895CF93DF93FC0123815D
:10D45000211105C0EC0160E4E3DF81E08B83DF9103
:10D46000CF910895FC012581222311F060E5D8CFEA
:10D470000895FC012481222311F06CE3D1CF08959B
:10D48000FC012085222331F02185222319F0118609
:10D490006BE3C6CF0895FC012085222339F0218556
:10D4A000211104C021E021876AE3BACF0895FC016D
:10D4B0002681222331F02781222319F0178269E384
:10D4C000AFCF0895FC012681222339F02781211155
:10D4D00004C021E0278368E3A3CF089567E3A0CFCA
:10D4E0006AE49ECF69E49CCF66E39ACF65E398CF68
:10D4F0006EE496CF64E394CF63E392CF62E390CF80
:10D5000061E38ECF60E38CCF6FE28ACF242F462F6A
:10D510006CE43ECF462F20E067E43ACF462F20E070
:10D5200066E436CF262F64E433CFCF92DF92FF92AA
:10D530000F931F93CF93DF938C01F62E443F81E02E
:10D54000580738F0413187E2580728F040E157E2A8
:10D5500002C044EF51E0243F81E0380738F0E90190
:10D560002131374228F0C0E1D7E202C0C4EFD1E058
:10D57000CA01845F914022E3C22ED12CB6010E94E1
:10D5800073AE462F2F2D62E4C80102DFCE01845F07
:10D590009140B6010E9473AE462F2F2D63E4C8015F
:10D5A000DF91CF911F910F91FF90DF90CF90F0CE40
:10D5B000262F40E06FE3ECCE262F40E06EE3E8CE6E
:10D5C000262F40E06DE3E4CE462F20E06FE4E0CE6E
:10D5D000462F20E06DE4DCCEFC016283611104C0C3
:10D5E00020E040E06BE4D4CE089577FF03C071954E
:10D5F0006195710920E0462F6BE4CACE809110023C
:10D60000882311F0729801C0729A9091100281E003
:10D61000892780931002089510920B061092050638
:10D620001092FC051092060610920706109208064A
:10D630001092090681E08093C30A4091110650912F
:10D64000120660E070E02BE23BE68091FD059091D0
:10D65000FE050C94905E8091D60981111CC0109239
:10D660000E0A10920F0A1092100A1092110A1092CC
:10D67000120A1092130A1092160A8091C10A909110
:10D68000C20ADC01ED91FC910190F081E02D199529
:10D690001092C30A08952BE23BE645E050E060E0BB
:10D6A00070E08091FD059091FE050C94905E609174
:10D6B0004F0E7091500E8091FD059091FE050E94D5
:10D6C000295E882319F081E080934E0E089560E072
:10D6D00087E00E94184D1092C40A089561E087E027
:10D6E0000E94184D81E08093C40A0895CF93DF9380
:10D6F00080915C0E811110C084EF91E090935B0EDD
:10D7000080935A0E8BE290E09093590E8093580EBE
:10D7100081E080935C0E20C08091580E9091590E4C
:10D720008532910514F0049709C08331910514F0F6
:10D73000029704C0823091052CF001979093590E06
:10D740008093580E8091580E9091590E97FF04C007
:10D750001092590E1092580EC091570ECC2311F012
:10D76000B6DF01C0BBDF81E08C278093570EC091EC
:10D770005A0ED0915B0E1C161D0654F010925C0ED2
:10D78000A6DF26EE3BE64AEF50E060E070E007C01F
:10D7900026E73BE6AE010D2E000C660B770B809161
:10D7A000FD059091FE050E94905E9093560E809329
:10D7B000550E8091580E9091590EC81BD90BD093DD
:10D7C0005B0EC0935A0EDF91CF9108950F931F9374
:10D7D000CF93DF938091C50A882329F0DF91CF9101
:10D7E0001F910F9183CF0091550E1091560EC0914D
:10D7F000FD05D091FE05B801CE010E94295E882367
:10D8000021F0B801CE010E94415EDF91CF911F91BE
:10D810000F915DCFCF92DF92EF92FF921092C50AE7
:10D8200020910106309102064091030650910406B2
:10D83000609106067091070680910806909109068E
:10D840000E94AEAE6B017C0120E030E0A9010E9495
:10D85000B4B287FD09C0C0920606D0920706E092D6
:10D860000806F092090608C01092060610920706F4
:10D870001092080610920906FF90EF90DF90CF906B
:10D88000A5CF0F931F93CF93DF938091540E909168
:10D890000B0681112AC0992309F456C00091520E3B
:10D8A0001091530EC091FD05D091FE05B801CE0137
:10D8B0000E94295E882321F0B801CE010E94415EBA
:10D8C0000DDF21E43CE642EC51E060E070E0809145
:10D8D000FD059091FE050E94985E9093530E8093F3
:10D8E000520E81E08093540E5AC08091C40A99234D
:10D8F00061F0882329F0DF91CF911F910F91E7CE3E
:10D90000DF91CF911F910F91E9CE8823C9F36091E8
:10D91000520E7091530E8091FD059091FE050E946C
:10D92000415E21E43CE644E150E060E070E080913B
:10D93000FD059091FE050E94985E9093530E809392
:10D94000520E1092540E2BC0C0911102D0911202AF
:10D950002297D0931202C09311021C161D0674F474
:10D96000BE01772787E00E94834DCC2321F081E020
:10D970008093C40A14C01092C40A11C06091520E60
:10D980007091530E8091FD059091FE050E94415EBD
:10D990009EDE8FEF90E09093120280931102DF9150
:10D9A000CF911F910F9108950F931F93CF93DF9302
:10D9B00000914A0E10914B0EC0914C0ED0914D0E1D
:10D9C000C00FD11FD0934D0EC0934C0EBE017727D0
:10D9D00087E00E94834DCC2321F081E08093C40A2C
:10D9E00002C01092C40A10161106ECF58091480E80
:10D9F0009091490EC817D9070CF485C080914E0E3E
:10DA0000882371F01092490E1092480E8CEF9FEF10
:10DA100090934B0E80934A0E81E08093470E73C023
:10DA200068E770E080E090E00E947549DC01CB017E
:10DA30000A96A11DB11D9093490E8093480E68E28D
:10DA400070E080E090E00E947549DC01CB010A960D
:10DA5000A11DB11D66277727681B790B70934B0EAC
:10DA600060934A0E50C0012B09F44DC08091480EBE
:10DA70009091490E8C179D070CF445C08091470E7C
:10DA8000882311F100914F0E1091500EC091FD05A9
:10DA9000D091FE05B801CE010E94295E882399F13C
:10DAA000B801CE010E94415E12DE10924D0E10921E
:10DAB0004C0E1092470E80910B06882321F1DF91C6
:10DAC000CF911F910F91DDCE69E670E080E090E08C
:10DAD0000E947549DC01CB018A569F4FAF4FBF4F63
:10DAE0009093490E8093480E68E270E080E090E0E9
:10DAF0000E947549DC01CB010A96A11DB11D9093CE
:10DB00004B0E80934A0EDF91CF911F910F91089594
:10DB1000EF92FF921F93CF93DF9300D0CDB7DEB784
:10DB200084E689838CE38A8388E28B831091510E8B
:10DB30001330E8F4E12EF12C10FF02C0C8DD01C063
:10DB4000CDDDE1E0F0E0EC0FFD1FEE0DFF1D4081AB
:10DB500050E060E070E028E83DE68091FD0590919E
:10DB6000FE050E94905E1F5F1093510E03C0AFDD53
:10DB70001092510E0F900F900F90DF91CF911F9147
:10DB8000FF90EF90089560E088E00C94184D61E0FC
:10DB900089E20C94184D0F931F93CF93DF9360E0AD
:10DBA0008BE20E94184D0091450E1091460EC091D7
:10DBB000FD05D091FE05B801CE010E94295E8823A3
:10DBC00041F0B801CE01DF91CF911F910F910C94DC
:10DBD000415EDF91CF911F910F91089581E0809375
:10DBE000C30A80911906FAD536CD3FB7F8948091D3
:10DBF000620E9091630EA091640EB091650E26B5F1
:10DC0000A89B05C02F3F19F00196A11DB11D3FBF74
:10DC1000BA2FA92F982F8827820F911DA11DB11D02
:10DC2000BC01CD0142E0660F771F881F991F4A95FE
:10DC3000D1F708952FB7F89460915E0E70915F0E42
:10DC40008091600E9091610E2FBF08951F93CF9326
:10DC5000DF93CDB7DEB765970FB6F894DEBF0FBE82
:10DC6000CDBF11E01093C70A80913F0E882391F138
:10DC70000E941C771092F40982E390E09A838983D2
:10DC800028E230E03C832B832EE630E03E832D8378
:10DC900024EF31E038872F831D8A25E1FE0131967C
:10DCA000A5EFB9E001900D922A95E1F79093F30961
:10DCB0008093F20984E08093F1090E941177BADF22
:10DCC0006093E3097093E4098093E5099093E60972
:10DCD0001093EF0965960FB6F894DEBF0FBECDBF67
:10DCE000DF91CF911F9108951F920F920FB60F925F
:10DCF00011242F933F938F939F93AF93BF93809162
:10DD00005E0E90915F0EA091600EB091610E309109
:10DD10005D0E23E0230F2D3720F40196A11DB11DC8
:10DD200005C026E8230F0296A11DB11D20935D0EAC
:10DD300080935E0E90935F0EA093600EB093610E81
:10DD40008091620E9091630EA091640EB091650E69
:10DD50000196A11DB11D8093620E9093630EA09356
:10DD6000640EB093650EBF91AF919F918F913F91DB
:10DD70002F910F900FBE0F901F9018950F931F9328
:10DD8000CF93DF930091550E1091560EC091FD0573
:10DD9000D091FE05B801CE010E94295E8823A1F032
:10DDA000B801CE010E94415E27E53BE648EB5BE00F
:10DDB00060E070E08091FD059091FE050E94905E0C
:10DDC0009093560E8093550E60914F0E7091500EA9
:10DDD0008091FD059091FE050E94295E81114BC046
:10DDE00010924E0E8FEF90E090934D0E80934C0E5C
:10DDF00075DC68E770E080E090E00E947549DC0126
:10DE0000CB010A96A11DB11D9093490E8093480E37
:10DE100068E270E080E090E00E947549DC01CB018F
:10DE20000A96A11DB11D66277727681B790B709391
:10DE30004B0E60934A0E24ED3CE644E150E060E076
:10DE400070E08091FD059091FE050E94985E909390
:10DE5000500E80934F0E27E53BE648EB5BE060E019
:10DE600070E08091FD059091FE050E94905E909378
:10DE7000560E8093550EDF91CF911F910F9108950B
:10DE80008F929F92AF92BF92CF92EF92FF920F9399
:10DE90001F93CF93DF9320911C06223008F07AC0A5
:10DEA0007B018C018090060690900706A0900806E2
:10DEB000B090090620E030E0A901C501B4010E943C
:10DEC000B4B2181654F520E030E0A901C501B40140
:10DED0000E94ACAF181654F420E030E048E452E45D
:10DEE000C501B4010E94B4B21816D4F420E030E0A9
:10DEF00048E452E4C501B4010E94ACAF18169CF48A
:10DF000020E030E048EC52E4C501B4010E94B4B214
:10DF100087FF09C0CBE4D0E008C0C0E0D0E005C076
:10DF2000C2E3D0E002C0C4E6D0E08FEF8C0D8230B7
:10DF300070F4209739F06C2FC8010E941E5A6C2F84
:10DF4000C7010DC0C8010E94D766C70116C08DEF7A
:10DF50008C0D8330F8F4209779F06C2FC801DF9195
:10DF6000CF911F910F91FF90EF90CF90BF90AF9006
:10DF70009F908F900C941E5AC801DF91CF911F91F2
:10DF80000F91FF90EF90CF90BF90AF909F908F90A8
:10DF90000C94D766DF91CF911F910F91FF90EF9076
:10DFA000CF90BF90AF909F908F9008958F929F9247
:10DFB000AF92BF92CF92DF92EF92FF92C09006068F
:10DFC000D0900706E0900806F090090620E030E0C7
:10DFD000A901C701B6010E94ACAF20E030E040E0EB
:10DFE0005FE387FD0BC0C701B6010E94AFAE4B01D6
:10DFF0005C010E947BAF97FD27C010C0C701B6012E
:10E000000E94AEAE0E947BAF97FD1EC065367105C3
:10E0100081059105DCF424E6822F14C0C501B4010A
:10E020000E947BAF65367105810591057CF420E087
:10E0300030E040E05FE3C701B6010E94AFAE0E944E
:10E040007BAF84E6861B03C084E601C080E0FF90BE
:10E05000EF90DF90CF90BF90AF909F908F900895FA
:10E060000F931F93CF93DF930091F6051091F7055F
:10E07000C091FD05D091FE05B801CE010E94295E38
:10E08000882321F0B801CE010E94415E8091C50A2B
:10E09000882339F01092C50ADF91CF911F910F911B
:10E0A00095CBDF91CF911F910F91089560E089E2A8
:10E0B0000E94184D27EC3DE642E350E060E070E03E
:10E0C0008091FD059091FE050C94905E1F920F9239
:10E0D0000FB60F9211240BB60F922F933F934F93CD
:10E0E0005F936F937F938F939F93AF93BF93EF93C0
:10E0F000FF938091440E8823A9F0669917C0EE988B
:10E100004ADD8091430E882389F08091420E882356
:10E1100039F0E091400EF091410E82810E94FF5F44
:10E12000C6D004C0669B02C0EE9835DDFF91EF912A
:10E13000BF91AF919F918F917F916F915F914F911F
:10E140003F912F910F900BBE0F900FBE0F901F901D
:10E15000189561E08BE20E94184DEE9A2BEC3DE69B
:10E1600048E853E160E070E08091FD059091FE0584
:10E170000E94905E9093460E8093450E089561E054
:10E180008BE20E94184DEE9A2BEC3DE648E853E1F5
:10E1900060E070E08091FD059091FE050E94905E28
:10E1A0009093460E8093450E08951092C70A4091B1
:10E1B0000F065091100660E070E026E23EE6809186
:10E1C000FD059091FE050C94905E8091880E811162
:10E1D00012C084E591E8A1E0BB27ABBFFC016791C9
:10E1E000769182E00E94B15F81E08093690E109287
:10E1F0006D0E10926A0E089581E08093680E6CEDAA
:10E2000075E00C94B15F81E20E94F04C21E0892B13
:10E2100009F420E0822F089580911506882309F4DF
:10E2200045C081E08093C30AEEDF882329F0809106
:10E2300018068823D1F106C080911606811104C00A
:10E2400080911506CBD231C090911506963069F5B4
:10E25000823081F08330D1F0813039F5E091310A9C
:10E26000F091320A72978081918145E550E060E03B
:10E2700070E017C0E091310AF091320A7297808104
:10E2800091814AE550E060E070E00BC0E091310A16
:10E29000F091320A7297808191814FE550E060E001
:10E2A00070E08F5C954F0E942250D5C908958091EF
:10E2B000440E882319F081E08093C00A8091FF0505
:10E2C00090910006DC01ED91FC910688F789E02D24
:10E2D000199580918E0E8111E9DE80918D0E882333
:10E2E00091F061E088E00E94184D40918B0E5091B2
:10E2F0008C0E60E070E023EC3DE68091FD0590918E
:10E30000FE050E94905E8091440E882321F080914A
:10E31000430E811101C080DF8091430E882379F084
:10E320008091440E882359F08091420E882339F061
:10E33000E091400EF091410E82810E94FF5F35CF47
:10E340008091C50A811155C05EDF8823E9F081E024
:10E350008093C50A8091FF0590910006DC01ED9144
:10E36000FC910288F389E02D199530DA2AE03CE629
:10E3700048E95AE360E070E08091FD059091FE0568
:10E380000E94905E12DF09C08091430E882329F11C
:10E390008091440E882311F0F2DE3ECFDADE8091C8
:10E3A000420E882339F0E091400EF091410E8281B7
:10E3B0000E94FF5F4091890E50918A0E1416150637
:10E3C000BCF4052E000C660B770B27E531E7809136
:10E3D000FD059091FE050C94905E8091420E88237D
:10E3E00039F0E091400EF091410E82810E94FF5F72
:10E3F0005ECF08950F931F932091880E211135C091
:10E4000044E551E861E077279C01220F331F820F1A
:10E41000931F092E000CAA0BBB0B0296A11DB11D68
:10E42000840F951FA61FB71FABBFFC01879104E5A2
:10E4300011E821E0332740916D0E93E0499FA00140
:10E440001124052E000C660B770B4E5F5F4F6F4F4C
:10E450007F4F040F151F261F371F2BBFF801079191
:10E46000801718F01F910F91B0CE1F910F91089552
:10E470008F929F92AF92BF92CF92DF92EF92FF92D4
:10E480000F931F93CF93DF93EC01A62E8091880EFC
:10E4900081116BC044E551E861E077276E01CC0C37
:10E4A000DD1CCC0EDD1E0D2C000CEE08FF08D70184
:10E4B000C6010296A11DB11D480F591F6A1F7B1F7F
:10E4C0006BBFFA01879144E551E861E07727B0908E
:10E4D0006D0E93E0B99E80011124012E000C220BD9
:10E4E000330B0E5F1F4F2F4F3F4F400F511F621FC7
:10E4F000731F6BBFFA014791481708F036C0809030
:10E500006B0E90906C0E0091810E1091820EB401F2
:10E51000C8010E94295E882321F0B401C8010E942D
:10E52000415E84E591E8A1E0BB278C0D9D1DAE1DE9
:10E53000BF1DABBFFC016791769182E00E94B15F85
:10E54000B0926A0EC0936D0EAA2079F01092690EF7
:10E5500025EE30E742E350E060E070E0C8010E9441
:10E56000905E90936C0E80936B0EDF91CF911F9114
:10E570000F91FF90EF90DF90CF90BF90AF909F9062
:10E580008F900895CF92DF92EF92FF928091880E44
:10E59000811134C08091870E882381F161E08EE083
:10E5A00090E066DF6091850E7091860ECB01A0E051
:10E5B000B0E0C090830ED090840EE12CF12CC816F0
:10E5C000D906EA06FB0664F4BC01CD016C197D098D
:10E5D0008E099F090E947549C60ED71EE81EF91EB6
:10E5E00022EC32E7B701A6018091810E9091820E54
:10E5F0000E94905E9093800E80937F0EFF90EF902C
:10E60000DF90CF900895CF92DF92EF92FF928091AA
:10E61000880E811134C080917E0E882381F161E0E3
:10E620008DE090E025DF60917C0E70917D0ECB0136
:10E63000A0E0B0E0C0907A0ED0907B0EE12CF12CDF
:10E64000C816D906EA06FB0664F4BC01CD016C19B4
:10E650007D098E099F090E947549C60ED71EE81EC6
:10E66000F91E23E033E7B701A6018091810E909156
:10E67000820E0E94905E9093790E8093780EFF90A8
:10E68000EF90DF90CF900895CF92DF92EF92FF92BC
:10E690008091880E811134C08091770E882381F19A
:10E6A00061E08CE090E0E4DE6091750E7091760E92
:10E6B000CB01A0E0B0E0C090730ED090740EE12CBE
:10E6C000F12CC816D906EA06FB0664F4BC01CD019C
:10E6D0006C197D098E099F090E947549C60ED71EC7
:10E6E000E81EF91E24E433E7B701A6018091810EEC
:10E6F0009091820E0E94905E9093720E8093710EA4
:10E70000FF90EF90DF90CF9008958091880E811157
:10E710002CC08091700E882341F08091770E81117A
:10E7200004C081E08093770EAFDF80916F0E882365
:10E7300061F08091880E811108C080917E0E811158
:10E7400004C081E080937E0E5EDF80916E0E882390
:10E7500061F08091880E811108C08091870E81112F
:10E7600004C081E08093870E0DCF08951092680E4B
:10E770002CEF30E744EF51E060E070E08091810ED3
:10E780009091820E0E94905E9093670E8093660E29
:10E7900008958091880E81110AC08091680E8823A7
:10E7A00031F060ED77E081E00E94B15FDFCF089546
:10E7B0000F931F93CF93DF93EC01AB0160E070E008
:10E7C0002AE00E94D9498C01CE010E94FE4A800FA6
:10E7D000911FDF91CF911F910F9108958F929F927A
:10E7E000AF92BF92CF92DF92EF92FF920F931F935F
:10E7F000CF93DF931F921F92CDB7DEB7082E000C88
:10E80000990BAA0BBB0BFC013197ED30F10508F019
:10E8100033C28827E159FE4F8F4F0C949AAE84E0A3
:10E820008093D2098AE08093D30986E28093D50948
:10E8300081E08093D8098093D9098093D70948E172
:10E8400056E120E030E08091D20990E028173907A6
:10E850000CF059C1FA0185919491A0E0B0E0880FC5
:10E86000991FAA1FBB1FF901EE0FFF1FEE0FFF1F1D
:10E87000E759F64F80839183A283B3832F5F3F4F85
:10E880004E5F5F4FE0CF84E08093D2098AE08093AF
:10E89000D30986E28093D50981E08093D8098093DB
:10E8A000D90982E08093D70940E156E120E030E0C9
:10E8B0008091D20990E0281739070CF024C1FA01A1
:10E8C00085919491A0E0B0E0880F991FAA1FBB1F0B
:10E8D000F901EE0FFF1FEE0FFF1FE759F64F808380
:10E8E0009183A283B3832F5F3F4F4E5F5F4FE0CF93
:10E8F00084E08093D30985E28093D50981E08093F9
:10E90000D80988E08093D90983E08093D70980E013
:10E9100090E0FC01E85FF94EE491DC01A652B64FAD
:10E92000EC93019688309105A1F70E94CD4EEBC083
:10E9300088E08093D20986E08093D30986E28093B1
:10E94000D50981E08093D8098093D90984E0809328
:10E95000D70948EF55E120E030E08091D20990E0FE
:10E96000281739070CF0CFC0FA0185919491A0E0E7
:10E97000B0E0880F991FAA1FBB1FF901EE0FFF1F00
:10E98000EE0FFF1FE759F64F80839183A283B38375
:10E990002F5F3F4F4E5F5F4FE0CF88E08093D209FB
:10E9A00086E08093D30986E28093D50981E0809345
:10E9B000D8098093D90985E08093D70948EE55E1BD
:10E9C00020E030E08091D20990E0281739070CF060
:10E9D0009AC0FA0185919491A0E0B0E0880F991F48
:10E9E000AA1FBB1FF901EE0FFF1FEE0FFF1FE75914
:10E9F000F64F80839183A283B3832F5F3F4F4E5F97
:10EA00005F4FE0CFE091310AF091320A7297808136
:10EA1000918140E550E060E070E08F5C954F0E948E
:10EA200022502AC182E18093D20985E08093D309E4
:10EA300082E28093D50981E08093D8098093D90937
:10EA400087E08093D70980E993E3A0E0B0E080936A
:10EA5000690990936A09A0936B09B0936C09F2E07D
:10EA60008F2E912C01E010E080E090E0A0E0BBE56B
:10EA70004CE454E060E070E024EEC22E2CE0D22E94
:10EA8000E12CF12C9801220F331F220F331F540168
:10EA9000AA0CBB1CAA0CBB1C2759364FF901B7FFA7
:10EAA0000DC0C082D182E282F38295012759364F90
:10EAB000F90140835183628373830CC04083518387
:10EAC0006283738395012759364FF901C082D18241
:10EAD000E282F382880F991FAA1FBB1F0E5F1F4F90
:10EAE000F2E08F0E911C22E18216910459F688E71C
:10EAF0009FEFA0E0B0E08093AD099093AE09A093A2
:10EB0000AF09B093B0090E943C4FB6C0CE01019648
:10EB10000E94BB4E23E040E150E060E070E072C034
:10EB200084E08093D20982E38093D30986E28093C4
:10EB3000D50981E08093D8098093D9098AE0809330
:10EB4000D70940EE55E120E030E08091D20990E015
:10EB500028173907C4F6FA0185919491A0E0B0E036
:10EB6000880F991FAA1FBB1FF901EE0FFF1FEE0FA1
:10EB7000FF1FE759F64F80839183A283B3832F5FF2
:10EB80003F4F4E5F5F4FE1CF84E08093D20980E238
:10EB90008093D30986E28093D50981E08093D809D8
:10EBA0008093D9098BE08093D70948ED55E120E0A7
:10EBB00030E08091D20990E0281739070CF0A3CFFC
:10EBC000FA0185919491A0E0B0E0880F991FAA1FE7
:10EBD000BB1FF901EE0FFF1FEE0FFF1FE759F64FA6
:10EBE00080839183A283B3832F5F3F4F4E5F5F4F3C
:10EBF000E0CFCE0101960E94BB4E21E040E154E0FF
:10EC000060E070E0CE0101960E94964F35C084E02E
:10EC10008093D20983E08093D30986E28093D5095B
:10EC200081E08093D8098093D9098DE08093D7093A
:10EC300040ED55E120E030E08091D20990E02817C6
:10EC400039070CF060CFFA0185919491A0E0B0E013
:10EC5000880F991FAA1FBB1FF901EE0FFF1FEE0FB0
:10EC6000FF1FE759F64F80839183A283B3832F5F01
:10EC70003F4F4E5F5F4FE0CF0F900F90DF91CF91EE
:10EC80001F910F91FF90EF90DF90CF90BF90AF90CA
:10EC90009F908F9008950F931F93CF93DF93EC0174
:10ECA000462F50E060E070E02AE00E94D9498C01D4
:10ECB000CE010E94FE4A800F911FDF91CF911F91DC
:10ECC0000F9108952FB7F894882381F08091BD119A
:10ECD0009091BE119093CC118093CB118091CD1166
:10ECE0009091CE1118161906ACF00FC08091BF118B
:10ECF0009091C0119093CC118093CB118091CD1144
:10ED00009091CE11181619062CF48091CD11909186
:10ED1000CE1107C08091CD119091CE119195819522
:10ED200091099093CE118093CD112FBF0895AF928A
:10ED3000BF92CF92DF92EF92FF920F931F93CF93E8
:10ED4000DF931F921F92CDB7DEB78C017A83698360
:10ED5000CE0101966C01580192E0A90EB11CE12C84
:10ED6000F12CC8010E94DDB3F60161916F01861795
:10ED700031F0C8010E94EFB3FFEFEF1AFF0A0F5FF7
:10ED80001F4F0A151B0569F781E0EF2809F480E0A1
:10ED90000F900F90DF91CF911F910F91FF90EF9007
:10EDA000DF90CF90BF90AF900895EF92FF920F93B6
:10EDB0001F93CF93DF931F921F92CDB7DEB78C01C5
:10EDC0007B018AEA8A8341E050E0BE016E5F7F4F9B
:10EDD000C8010E948553D701ED91FC910284F3850F
:10EDE000E02DC701199582E8898341E050E0BE011A
:10EDF0006F5F7F4FC8010E9485530F900F90DF9186
:10EE0000CF911F910F91FF90EF9008958091EE099F
:10EE1000882311F061E001C060E08091ED090C945D
:10EE2000184D8091EE09882311F060E001C061E087
:10EE30008091ED090C94184DCF93DF93C3EED9E088
:10EE40001C861D861E86188A1F860E941A6E68837D
:10EE500079838A839B83198618861C86DF91CF91DC
:10EE60000895CF92DF92EF92FF920F931F930E942B
:10EE70001A6E6B017C016093391270933A12809381
:10EE80003B1290933C128091DC0A0E94F04C8093DC
:10EE900038129091DE0A992329F091E0811190E0D7
:10EEA000909338128091E60A9091E70AA091E80ABF
:10EEB000B091E90A97018601081B190B2A0B3B0B3D
:10EEC0004091EA0A5091EB0A6091EC0A7091ED0AC8
:10EED0009091DF0A041715072607370760F4C092E0
:10EEE000E20AD092E30AE092E40AF092E50A109274
:10EEF000E10A892F1EC09093E00A80913812809316
:10EF0000DF0AC092E20AD092E30AE092E40AF092A9
:10EF1000E50A891761F0C092E60AD092E70AE0920A
:10EF2000E80AF092E90A91E09093E10A02C0109297
:10EF3000E10A1F910F91FF90EF90DF90CF9008951D
:10EF4000462F50E060E070E02AE00C94D9490F931E
:10EF50001F93CF93DF93EC012AE00E94D9498C01E3
:10EF6000CE010E94FE4A800F911FDF91CF911F9129
:10EF70000F910895CF92DF92EF92FF920F931F931C
:10EF8000CF93DF936B01770FEE08FF08F7FE1BC0EE
:10EF9000EC016DE20E9499498C0144275527BA0182
:10EFA0004C195D096E097F092AE0CE010E94D949FA
:10EFB000800F911FDF91CF911F910F91FF90EF90E4
:10EFC000DF90CF9008952AE0B701A601DF91CF919D
:10EFD0001F910F91FF90EF90DF90CF900C94D94943
:10EFE000CF92DF92EF92FF920F931F93CF93DF9315
:10EFF0008C016B01770FEE08FF08F7FE12C06DE27F
:10F000000E949949EC0144275527BA014C195D0922
:10F010006E097F092AE0C8010E94D949C80FD91F8B
:10F0200006C02AE0B701A6010E94D949EC01C80137
:10F030000E94FE4A8C0F9D1FDF91CF911F910F916F
:10F04000FF90EF90DF90CF9008950F931F93CF9391
:10F05000DF931F92CDB7DEB78C0169830E94DDB3C9
:10F060006981861729F0C8010E94EFB381E001C0D1
:10F0700080E00F90DF91CF911F910F910895CF9372
:10F080000E94626384E090E09093D90A8093D80A4A
:10F0900080E99EE090935C1180935B111092561171
:10F0A0008091D70A9091900E891718F091E0909373
:10F0B000531129E93EE030936611209365111092B7
:10F0C00060119091990E891718F091E090935D115D
:10F0D00022EA3EE03093701120936F1110926A1172
:10F0E0009091A20E891718F091E0909367112BEA86
:10F0F0003EE030937A11209379111092741190911F
:10F10000AB0E891718F091E0909371111092D60A06
:10F1100020E030E0F901E05DF04F40815181415045
:10F1200051094432510520F491E09093D60A05C06C
:10F130002D5F3F4F2837310569F79091D60A992303
:10F1400041F12091A30E3091A40E2D5D3F4F3093DD
:10F15000A40E2093A30E2091A50E3091A60E23524B
:10F1600031093093A60E2093A50E2091AC0E30915C
:10F17000AD0E2D5D3F4F3093AD0E2093AC0E209120
:10F18000AE0E3091AF0E235231093093AF0E209363
:10F19000AE0E9091A90F9F3049F49091AA0F9F3025
:10F1A00029F4109252111092511108C02091F80FB9
:10F1B0003091F90F309352112093511122E130E038
:10F1C00030934F1120934E112091D80A3091D90AD3
:10F1D000A4EBBEE0EAEFF0E141E0B683A5839C91A9
:10F1E000992329F0891718F040832F5F3F4F1A9613
:10F1F000379691E1EE34F90781F73093D90A2093DD
:10F20000D80A2131310534F080E190E09093D90A99
:10F210008093D80A0E944D6387E591E190935D1039
:10F2200080935C1080915B1190915C1190935B10C6
:10F2300080935A1084E591E190935F1080935E1063
:10F2400085E591E1909361108093601083E591E1F1
:10F25000909363108093621081E691E19093671020
:10F26000809366108091651190916611909365105E
:10F27000809364108EE591E19093691080936810FB
:10F280008FE591E190936B1080936A108DE591E189
:10F2900090936D1080936C108BE691E190937110B8
:10F2A0008093701080916F119091701190936F10F6
:10F2B00080936E1088E691E19093731080937210A2
:10F2C00089E691E1909375108093741087E691E13F
:10F2D000909377108093761085E791E190937B105F
:10F2E00080937A108091791190917A11909379108E
:10F2F0008093781082E791E190937D1080937C1049
:10F3000083E791E190937F1080937E1081E791E1F4
:10F3100090938110809380102091D80A3091D90A5F
:10F320002450310960E07AE0C7E0462F50E04217F0
:10F33000530724F5CA010496789FF001799FF00DD8
:10F340001124E65AFF4EC49FC001C59F900D1124A1
:10F35000AC0144505F4E53834283DC01A650BF4E44
:10F3600015964D915C9116975183408385509F4E21
:10F3700095838483B187A0876F5FD7CF81E0809327
:10F38000DA0ACF9108950F931F93CF93DF93FC0177
:10F39000248135812115310519F4FB01108211C03A
:10F3A000EA0121972C173D0708F4E9018B01FC01C4
:10F3B00060817181AE01C8010E94E4B1C00FD11F0C
:10F3C0001882DF91CF911F910F910895FC01128255
:10F3D000138214821582168217821286089580E0A5
:10F3E00008950F931F93CF938C016EED76E18CEC13
:10F3F00098E00E94A049D8011896ED91FC911997C8
:10F40000608171818CEC98E0D3D9C1E0D8011A9663
:10F410008C91C81700F569ED76E18CEC98E00E94BC
:10F42000A0496C2F8CEC98E08BDD66ED76E18CECDE
:10F4300098E00E94A049F80190858185E92FF82F76
:10F44000EC0FF11DEC0FF11D608171818CEC98E0E7
:10F45000AFD9CF5FDBCFCF911F910F910895CF939D
:10F46000DF93CDB7DEB76E970FB6F894DEBF0FBE51
:10F47000CDBF8F300CF080E02EEC36E13A8329834B
:10F4800027EC36E13C832B8329EB36E13E832D8349
:10F490002DEA36E138872F8323EA36E13A87298738
:10F4A0002CE936E13C872B8728E936E13E872D871A
:10F4B00021E936E1388B2F8726E836E13A8B298B14
:10F4C00029E736E13C8B2B8B2EE636E13E8B2D8BEC
:10F4D00022E636E1388F2F8B20E536E13A8F298FEF
:10F4E0002FE336E13C8F2B8F2AE336E13E8F2D8FC1
:10F4F000E82FEE0FFF0BEC0FFD1F818192816E96BE
:10F500000FB6F894DEBF0FBECDBFDF91CF91089547
:10F51000AF92BF92CF92DF92EF92FF920F931F9321
:10F52000CF93DF938AE492E17EE1D72ED80ECC24EC
:10F53000C39402E010E0C3E0D0E0E2E0BE2EEE248F
:10F54000E394F12C8091930D9091940DDC01ED9159
:10F55000FC910480F581E02D1995892B09F4ADC04B
:10F56000A09030018091930D9091940DDC01ED916C
:10F57000FC910680F781E02D199596B3B39A2091FE
:10F58000840030918500285A344E30938D002093AA
:10F590008C002A2D2C7119F01092900D4BC093FB0A
:10F5A000992790F9E091900DE11116C0992351F23D
:10F5B000803241F6C092900D80934A128091E00D06
:10F5C0009091E10D892B09F0BDCFF092E10DE09211
:10F5D000E00D1092920DB6CF9111DECFE13041F4E3
:10F5E000803409F0AFCFB092900D80934B12E6CFEC
:10F5F00091E09E0F9093900DF0E0E65BFD4E8083CE
:10F60000903209F09FCF1092900DEAE4F2E12FEFD3
:10F610003FEF8191281B3109DE12FBCF4091681228
:10F620008091691290E0982F8827840F911D2817E8
:10F63000390729F0D093E10DC093E00D83CF80917D
:10F64000E00D9091E10D019739F48091920D8F5F5B
:10F650008093920D843020F01093E10D0093E00D23
:10F660008091910D8F5F8093910D90918F0D9817E0
:10F6700008F5C092E20D20E030E0F901E65BFD4EB6
:10F680004281838190E0982F8827840F911DAC01DF
:10F690004F5E52404B3D554028F4F901EB56F24F76
:10F6A000918380832E5F3F4F2C31310531F71092CB
:10F6B000910D48CF1092E20D45CFDF91CF911F9170
:10F6C0000F91FF90EF90DF90CF90BF90AF90089593
:10F6D000EF92FF920F931F93CF93DF9310928F0EB1
:10F6E00082E08093900E68EE73E07093920E6093C8
:10F6F000910E40ED57E05093940E4093930E2CEDF5
:10F7000035E03093960E2093950E8FE08093970E00
:10F710001092980E94E09093990E70939B0E6093C4
:10F720009A0E50939D0E40939C0E30939F0E209303
:10F730009E0E8093A00E1092A10E93E09093A20EC5
:10F740007093A40E6093A30E5093A60E4093A50E43
:10F750003093A80E2093A70E8093A90E1092AA0EA4
:10F7600091E09093AB0E7093AD0E6093AC0E5093FE
:10F77000AF0E4093AE0E3093B10E2093B00E809337
:10F78000B20E1092B30EE4EBFEE0ADEBBEE080E013
:10F7900008EE13E060ED77E04CED55E031E022E05B
:10F7A00095E0980F9083128301837483638356835B
:10F7B0004583ED01229791E03883219628831C929E
:10F7C0008F5F3A961A968C3059F710922C0F9093BF
:10F7D0002D0F10922E0F90932F0F80E090E09C0140
:10F7E0002157314FF901EF55FF4F118210823296A8
:10F7F000108203968837910591F784E290E0909308
:10F80000310F8093300F81E08093320F2CE030E095
:10F810003093340F2093330F94E09093350F21E20F
:10F8200030E03093370F2093360F27E02093380FC6
:10F8300029E030E030933A0F2093390F20E12093F4
:10F840003B0F7AE07093A80F2BE02093A90F209331
:10F85000AA0F48EE53E05093AC0F4093AB0F20ED4E
:10F8600037E03093AE0F2093AD0F1092AF0F64E6E8
:10F870006093B00F6093B10F5093B30F4093B20FEA
:10F880003093B50F2093B40F1092B60F1092B70FAC
:10F890008093B80F1092BA0F1092B90F8093BB0FDC
:10F8A0008093BC0FE8ECF0E0F093BE0FE093BD0F47
:10F8B000E0E2F3E0F093C00FE093BF0F5093C20F6C
:10F8C0004093C10F3093C40F2093C30F8093C50F93
:10F8D000E9E5F0E0F093C70FE093C60FE0E8F0E051
:10F8E000F093C90FE093C80FEFEFF0E0F093CB0F68
:10F8F000E093CA0FF093CD0FE093CC0F8093CE0F1F
:10F900009093CF0F1092D00F8093D10F9093D20F7E
:10F910001092D30F1092D40F8093D50F1092D60F60
:10F920001092D70F8093D80F1092D90F98E290932E
:10F93000DA0F5093DC0F4093DB0F5093DE0F4093B0
:10F94000DD0F3093E00F2093DF0F8093E10F92E300
:10F950009093E20FE2E0E093E30F8093E40F609373
:10F96000E50FE6E4E093E60F9093E70F1092E80FBF
:10F970001092E90F1092EA0F1092EB0F1092EC0F19
:10F980001092ED0FEAEFF0E0F093EF0FE093EE0F3F
:10F990001092F00F1092F10F6093F20F61E46093F8
:10F9A000F30F1092F40F9093F50F1092F60F9093BF
:10F9B000F70FEEE5F1E0F093F90FE093F80F1092F6
:10F9C000FA0FACEDB5E0B093FC0FA093FB0F00EA8B
:10F9D0001FE01093FE0F0093FD0F30930010209353
:10F9E000FF0FC8E8D3E1D0930210C093011068EB79
:10F9F000E62E6BE0F62EF0920410E0920310E0E4A5
:10FA0000FFE1F0930610E09305101092071010929A
:10FA100008101092091069E160930A1080930B108E
:10FA200080930C1080930D1050930F1040930E1084
:10FA30003093111020931010F0921310E0921210D6
:10FA40001093151000931410D0931710C093161034
:10FA500020E737E1309319102093181010921A10F4
:10FA600010921B1010921C1090931D1090931E105A
:10FA700090931F101092201080932110109231103B
:10FA80001092221099E0909323101092241010925B
:10FA900025101092261010922710B0932910A093D1
:10FAA0002810F0932B10E0932A1080932C10709361
:10FAB0002D1010922E1021E030E030933010209362
:10FAC0002F1040E052EC61E070E040933210509310
:10FAD0003310609334107093351040933610509368
:10FAE0003710609338107093391040E056E960E0A9
:10FAF00070E040933A1050933B1060933C10709329
:10FB00003D1040933E1050933F106093401070930F
:10FB100041101092421020E039E1309344102093BC
:10FB20004310109245109EE190934610109247109A
:10FB30002EE130E0309349102093481030934B1061
:10FB400020934A1030934D1020934C1090934E10F8
:10FB500090934F1080935010809351101092521038
:10FB600090935310809354108093551086E799E139
:10FB7000A0E0B0E08093561090935710A0935810D7
:10FB8000B09359100FE81EE0C0E0D0E0CE010E9413
:10FB9000DDB3F80161918F01861719F0CE010E9443
:10FBA000EFB32196CB3CF1E0DF0781F7DF91CF91F6
:10FBB0001F910F91FF90EF9008954F925F926F9277
:10FBC0007F928F929F92AF92BF92CF92DF92EF92ED
:10FBD000FF92CF93DF93EB01A0914812B0914912AD
:10FBE0009D012F5F3F4F45E0429F2001439F500CF6
:10FBF0001124052C000C66087708812C912C5401E7
:10FC00002C33E1E03E07ECF447E851E861E0772768
:10FC100075016401C40CD51CE61CF71C4C0D5D1D60
:10FC20006E1D7F1D6BBFFA014791569165E0860EF0
:10FC3000911CA11CB11CC417D50729F12F5F3F4FA0
:10FC4000DFCF25E0822E912CA12CB12C21E030E0D9
:10FC5000A217B30708F44CC047E851E861E07727E2
:10FC6000480D591D6A1D7B1D6BBFFA0147915691C6
:10FC7000F5E08F0E911CA11CB11CC417D50719F01B
:10FC80002F5F3F4FE5CF47E851E861E07727E5E098
:10FC9000E29F6001E39FD00C11240D2C000CEE08B4
:10FCA000FF084E5F5F4F6F4F7F4F4C0D5D1D6E1D08
:10FCB0007F1D6BBFFA0147915691FC01538342832C
:10FCC00047E851E861E077274C5F5F4F6F4F7F4F08
:10FCD000C40ED51EE61EF71EEBBEF601C790FC0152
:10FCE000C4823093491220934812C901019606C07C
:10FCF000109249121092481280E090E0DF91CF916B
:10FD0000FF90EF90DF90CF90BF90AF909F908F903B
:10FD10007F906F905F904F9008950F931F93809105
:10FD2000431281111EC00E941A6E0091441210915C
:10FD300045122091461230914712AB01BC01401B85
:10FD4000510B620B730B8091411290914212A0E013
:10FD5000B0E084179507A607B70718F481E08093F1
:10FD600043121F910F910895809141129091421278
:10FD7000892B89F080914312882381F00E941A6EAA
:10FD800060934412709345128093461290934712E9
:10FD900010924312089581E08093431208951F92B8
:10FDA0000F920FB60F9211242F938F939F9310925F
:10FDB0009500109294008091CF0A8F5F8093CF0AB4
:10FDC0009091D412891784F01092CF0A2091D10A11
:10FDD0008091DF129091E012820F911D27FD9A957C
:10FDE0009093E0128093DF128091CE0A8F5F809310
:10FDF000CE0A9091E412891784F01092CE0A2091D5
:10FE0000D00A8091E2129091E312820F911D27FD9A
:10FE10009A959093E3128093E2129F918F912F9184
:10FE20000F900FBE0F901F9018958091CD0A8111F1
:10FE300004C08091CC0A882321F0809171008260F7
:10FE400003C0809171008D7F8093710008951F938E
:10FE5000CF93DF931F92CDB7DEB710E0181731F0C4
:10FE600089830E941A411F5F8981F8CF0F90DF912B
:10FE7000CF911F910895CF93DF9360E088E00E94B7
:10FE8000184D10924012C0913E12D0913F12BE0107
:10FE900080EF9AE00E94295E882329F0BE0180EF5E
:10FEA0009AE00E94415E81E080933D128091970626
:10FEB000882341F060E276E1809195069091960664
:10FEC0000E94114BDF91CF910C94484160914310F7
:10FED0007091441080E090E00E94B8B220E030E0E1
:10FEE0004AE754E40E9413AFAB01BC0121E08091CA
:10FEF0009506909196060C94214A0C94CE420C944F
:10FF0000BA4180917612882319F00E94CE4202C035
:10FF10000E94BA419091761281E0892780937612EF
:10FF200008958AE0D8C789E0D6C788E0D4C787E0BB
:10FF3000D2C786E0D0C785E0CEC784E0CCC783E0D7
:10FF4000CAC782E0C8C781E0C6C789E076C788E033
:10FF500074C787E072C786E070C785E06EC784E02B
:10FF60006CC783E06AC782E068C781E066C789E042
:10FF70008BC788E089C787E087C786E085C785E0AB
:10FF800083C784E081C783E07FC782E07DC781E0CB
:10FF90007BC7BEC7C9C780913D12811101C06BCF1D
:10FFA0000895CF93DF9380913D12882321F1109221
:10FFB0003D1260E088E00E94184DC0913E12D09141
:10FFC0003F12BE0180EF9AE00E94295E882329F04B
:10FFD000BE0180EF9AE00E94415E809197068823DF
:10FFE00069F060EE77E18091950690919606DF9139
:10FFF000CF910C94114BDF91CF913DCFDF91CF91F9
:020000021000EC
:1000000008950F931F93CF93DF9300917112109176
:100010007212C091FD05D091FE05B801CE010E947B
:10002000295E882379F0B801CE010E94415E80915B
:10003000FF0590910006DC01ED91FC9100A0F1A17B
:10004000E02D199500916F1210917012C091FD056D
:10005000D091FE05B801CE010E94295E882321F0CF
:10006000B801CE010E94415E729880919706882364
:1000700061F061E977E18091950690919606DF91B4
:10008000CF911F910F910C94114BDF91CF911F9144
:100090000F910895CF93DF9380914012882311F13F
:1000A0000E94CE4210924012C0913E12D0913F1257
:1000B000BE0180EF9AE00E94295E882329F0BE01EC
:1000C00080EF9AE00E94415E80919706882371F04C
:1000D00067EC77E18091950690919606DF91CF913C
:1000E0000C94114BDF91CF910C940943DF91CF9188
:1000F00008950C9409430E94CE42409148105091BB
:10010000491060E070E02AEB31E480EF9AE00E9451
:10011000905E90933F1280933E12809197068823C1
:1001200041F06CEA77E180919506909196060C94E7
:10013000114B08950E94BA414091481050914910C6
:1001400060E070E02EEC32E480EF9AE00E94905E76
:1001500090933F1280933E1280919706882341F03E
:1001600069E977E180919506909196060C94114B80
:10017000089580917712882319F00E94CE4202C020
:100180000E9492439091771281E0892780937712A1
:1001900008950C9492430C94A4430C94BA43809118
:1001A0007512882319F00E94A44302C00E94BA432A
:1001B0009091751281E089278093751208950C94AF
:1001C000E3430E94E3438091910690919206DC0103
:1001D000ED91FC9104A0F5A1E02D19940C941F441D
:1001E00080917412882319F00E94E34302C00E9498
:1001F0001F449091741281E08927809374120895AE
:100200000C943A440C94554480917312882319F04D
:100210000E943A4402C00E9455449091731281E0BA
:1002200089278093731208950C947E908091430ED9
:1002300081110C9468900C947E900C9468900E94AC
:10024000CF418091910690919206DC01ED91FC9155
:1002500002A0F3A1E02D1994CF93DF93C091FD0587
:10026000D091FE056091711270917212CE010E94C0
:10027000295E811129C040916E1250E060E070E06B
:100280002EEF3AE6CE010E94985E90937212809310
:1002900071128091FF0590910006DC01ED91FC91B7
:1002A000068CF78DE02D199580911A06882361F050
:1002B00060916F12709170128091FD059091FE0512
:1002C0000E94295E882371F0809197068823E9F0C7
:1002D00068E877E18091950690919606DF91CF913D
:1002E0000C94114B0E94EE6D2EEE3DE644E650E07C
:1002F00060E070E08091FD059091FE050E94985E9F
:100300009093701280936F12DFCFDF91CF91089599
:100310000E94567080919706882341F06DE577E141
:1003200080919506909196060C94114B0895E0915A
:100330006C12F0916D1282810E94FF5F809197068E
:10034000882341F06FE377E18091950690919606BE
:100350000C94114B08958091440E882319F00E944B
:10036000BF7002C00E94A97080919706882379F01F
:100370002091B70F8091950690919606222319F04F
:1003800063E077E102C06CE177E10C94114B0895D2
:100390000C948946CF938091C70A882309F46BC0D7
:1003A0000E9403719091C50A882341F0911163C0A6
:1003B00080912106882309F446C05DC091115BC07D
:1003C00080919706882341F064EE76E1809195064E
:1003D000909196060E94114B0E94A07181E080933B
:1003E0000A0680910702813009F045C08091F10F23
:1003F000882309F440C08091B70F882379F026E262
:100400003EE842E350E060E070E080EF9AE00E9456
:10041000985E90936B1280936A122DC04091B90F31
:100420005091BA0F141615065CF4052E000C660BDD
:10043000770B2BE13EE880EF9AE0CF910C94905E31
:10044000CF910C941B8E82E08093210680919706B9
:10045000882341F060EF76E18091950690919606B1
:100460000E94114BC1E0C09320060E9489460E9461
:10047000A071C0930A06CF9108950C9458438091BF
:100480008D0681110C9489460C9458430C94CE8EA1
:1004900008950895FC01828193818830910529F4A3
:1004A00010922B0110922A010895099721F41092BD
:1004B0002901109228010895FC01178A168A6CED13
:1004C00075E082810C947860CF93DF93EC011F8AF2
:1004D0001E8A8A810E94F15F8B8D882331F08A8188
:1004E0000E9468609A8F898F1B8EDF91CF9108954B
:1004F000DF92EF92FF920F931F93CF93DF93EC0164
:100500008A81893010F40E94D85FDD8C6B8D7C8DE0
:10051000098D1A8DEA80FB8089E08E1508F466C08B
:100520000F30110538F001369DE6190728F000E676
:100530001DE602C00FE010E06F30710538F0613643
:100540008DE6780728F060E67DE602C06FE070E097
:1005500080E090E00E94B8B220E030E04AE754E446
:100560000E9413AF20E030E04CE852E40E9419B33F
:100570009B01AC0160E070E08AEF94E40E9413AF4D
:100580000E947BAFFF2425E12E9DF0012F9DF00DF1
:100590001124E558FE4EDD2071F023813481AB013A
:1005A00077FF04C044275527461B570B88279927F8
:1005B000841B950B0AC025813681AB0177FF04C0EF
:1005C00044275527461B570BCA014FB7F89455E1EE
:1005D0005E9DF0015F9DF00D1124E558FE4E108BDD
:1005E0000787328B218B948B838B4FBF9D8D6B8DB7
:1005F0007C8D8A819923F9F08A3058F495E1899F9E
:10060000F0011124E558FE4E0581168116950795D7
:1006100002C00EEE12E041E00E941F6061E070E057
:1006200080E090E00E94694E8A810E94686008170D
:100630001907A0F31EC08A3058F495E1899FF00194
:100640001124E558FE4E038114811695079502C0CA
:100650000AEC18E040E00E941F6061E070E080E07A
:1006600090E00E94694E8A810E946860801791071D
:10067000A0F38A810E94F15FB8018A81DF91CF9156
:100680001F910F91FF90EF90DF900C947860CF93C3
:10069000DF93EC018A81893010F40E94D85F48EE24
:1006A00053E05B874A8720ED37E03D872C878CED50
:1006B00095E09F878E87598B488B3B8B2A8B9D8B30
:1006C0008C8BDF91CF910895CF93DF93EC017F8BDB
:1006D0006E8B888599856817790769F48A810E94ED
:1006E000F15F8B8D882329F18A810E9468609A8F3F
:1006F000898F1B8E1EC0CE010E94AB5AEA81EA3060
:10070000B0F49C01C39714F022E330E02E3C8FEF4D
:10071000380714F42EEC3FEF8FB7F89495E1E99F7A
:10072000F0011124E558FE4E318720878FBF81E00C
:100730008B8FDF91CF910895CF93DF93EC018BA145
:100740009CA1892B11F01CA21BA29B0177FF03C067
:10075000319521953109B901CE010E94AB5A909390
:100760002D0180932C019F8B8E8B0E941A6E6F8FB0
:1007700078A389A39AA3DF91CF910895CF93DF93B4
:10078000EC018A81893010F40E94D85F2EEC3FEF93
:100790003B872A8782E390E09D878C871F861E8691
:1007A000398B288B9B8B8A8B1D8A1C8A6EEE72E09C
:1007B0008A810E9464606AEC78E08A810E946060AD
:1007C0008CED95E09A8F898F1B8EDF91CF910895E4
:1007D000CF93DF93EC018BA19CA1892B11F01CA27C
:1007E0001BA2CE010E94D76610922D0110922C01FF
:1007F0001F8A1E8A0E941A6E6F8F78A389A39AA3FC
:10080000DF91CF9108950F931F93CF93DF93FC0156
:1008100023A134A1232B91F1EC010E941A6E0F8DBC
:1008200018A129A13AA1DC01CB01801B910BA20BDD
:10083000B30B4097A105B10508F18BA19CA10197CD
:10084000E9F46E897F89615071097F8B6E8BCE01CF
:10085000161617062CF0DF91CF911F910F91B8CF8C
:100860000E94AB5A90932D0180932C019F8B8E8B0D
:100870000E941A6E6F8F78A389A39AA3DF91CF91FC
:100880001F910F910895CF93DF93EC018D8D9E8D75
:100890001B861A869D878C871F861E86198A188A52
:1008A0009B8B8A8B1D8A1C8A61E08CE20E94474DDB
:1008B0008A819B81089721F410922D0110922C01BE
:1008C0001CA21BA2DF91CF9108956F927F928F920D
:1008D0009F92AF92BF92CF92DF92EF92FF920F93CF
:1008E0001F93CF93DF938091071390910813DC013E
:1008F000ED91FC910480F581E02D1995B12C18162D
:1009000019060CF0D1C0AA24A394809107139091EA
:100910000813DC01ED91FC910480F581E02D19951F
:10092000892B09F4C1C0C091D21281E08C0F809351
:10093000D2128091071390910813DC01ED91FC9184
:100940000680F781E02D1995EC2FF0E0EE56FD4E74
:1009500080838A30D1F6E090D212F12C10923C0DB7
:1009600010923B0D1092370D1092380D1092390DE8
:1009700010923A0D1092360D1092350D1092340DE2
:1009800082E9C82E82E1D82E00E010E0D0E0C0E07D
:100990000E151F050CF06BC0F60191916F019D3093
:1009A00009F462C09C3799F19A3009F051C0CC2308
:1009B00051F16C2E712CC3010197F3D470933C0D4F
:1009C00060933B0D0E941A6E60938B0D70938C0D9B
:1009D00080938D0D90938E0D80917812882309F469
:1009E0005FC080903B0D90903C0DB801661977096F
:1009F00082E992E10E9477588816990609F450C05E
:100A0000109291124FC010929112D0E02DC08C2FF5
:100A100090E0FC01EB51FD4E1082D13089F060F086
:100A2000D23099F4BED46093370D7093380D809313
:100A3000390D90933A0D09C0B4D46093340D05C0BC
:100A4000B0D47093360D6093350DDF5FC0E00CC0FD
:100A50000F3311053CF4EC2FF0E0EB51FD4E908389
:100A6000CF5F02C0109291120F5F1F4F91CF809104
:100A7000911281110EC08091310D9091320D01962D
:100A80009093320D8093310D60E087E80E941891B9
:100A900002C0BB24B394109292121092D21235CF9E
:100AA000A0929112D1E0E0CF8B2DDF91CF911F91D9
:100AB0000F91FF90EF90DF90CF90BF90AF909F90FD
:100AC0008F907F906F900895CF931092330D109276
:100AD000300D1092320D1092310D61E089E30E94C9
:100AE000184D0E941A588091071390910813DC0149
:100AF000ED91FC910480F581E02D1995892B61F031
:100B00008091071390910813DC01ED91FC91068010
:100B1000F781E02D1995E7CF0E94949180910713FA
:100B200090910813DC01ED91FC910284F385E02D96
:100B3000199510928A0D0E941A6E60938B0D709316
:100B40008C0D80938D0D90938E0DC1E0BEDE8111D2
:100B50000E94E82F0E945A580E944B638091310DE9
:100B60009091320D0A9724F480918A0D882331F0F8
:100B700060E08AE80E941891C093330D8091330D94
:100B8000882321F38091300D882341F04BEC51E014
:100B900060E070E08FE89EE00E94CDB360E089E302
:100BA0000E94184D60E08AE3CF910C94184DEF92AB
:100BB000FF920F931F93CF93DF9300D000D0CDB758
:100BC000DEB767EE75E0CE0101960E9461490D81A6
:100BD0001E81F02EEE24E394809107139091081368
:100BE000DC01ED91FC910480F581E02D1995892BB4
:100BF00021F18091071390910813DC01ED91FC9194
:100C00000680F781E02D19958F3439F4E092901227
:100C100080938512E0928412DFCF909190129923F5
:100C2000D9F2E091841291E09E0F90938412F0E04B
:100C3000EB57FD4E80839F1578F2809184128F15BB
:100C400010F4F12C21C04BE050E069E772E1CE01D5
:100C500001960E94C379A5E8B2E1E7EEF5E0FF2432
:100C6000F3941127CF01875E95408017910734F4E4
:100C70009D9181919817B1F3F12CF4CF10928512C8
:100C80001092901210928412CE0101960E94314966
:100C90008F2D26960FB6F894DEBF0FBECDBFDF9125
:100CA000CF911F910F91FF90EF900895DC01ED918E
:100CB000FC910190F081E02D1994CF93DF93EC012A
:100CC0007F8B6E8B0E94AB5ABC018A81DF91CF91E2
:100CD0000C9478600F931F93CF93DF932091C50FEF
:100CE00021111BC0C0910C06D0910D0608811981FD
:100CF0009C01AFEFB0E00E944BB42FEF33E040E037
:100D000050E00E94FDB3D801ED91FC91B901CE01F4
:100D1000DF91CF911F910F911994DF91CF911F9186
:100D20000F9108950C94138F0E948D7E8091F5058C
:100D300081110C94CE8E0C94138F60E478E1809135
:100D40009506909196060C94A049CF939C01A4E639
:100D5000B0E00E944BB42FEF33E040E050E00E943F
:100D6000FDB3C22F30E08091D312281B310937FF29
:100D700003C0319521953109233031053CF1C33051
:100D800020F0C23618F0C4E601C0C0E080919106A0
:100D900090919206DC01ED91FC91EC5AFF4F01908D
:100DA000F081E02D6C2F1995C093D3128091970696
:100DB000882361F068E178E180919506909196062C
:100DC0000E94A0498C2FCF910C948440CF9108951C
:100DD0009C010197849710F4822F0895C9018456CD
:100DE00091098438934040F4C90164E670E00E94A0
:100DF00073AE822F94E61BC0283E43E03407D8F040
:100E0000C90168EE73E00E9473AE48E15CEF649F35
:100E1000C001659F900D749F900D1124280F391FFC
:100E2000C9016AE070E00E9487AE822F9AE0699F54
:100E300080191124089580E00895CF93C82F8091E0
:100E4000910690919206DC01ED91FC91EE5BFF4FD3
:100E50000190F081E02D6C2F1995809197068823E1
:100E600089F06BDF6C2F80919506909196060E9419
:100E7000A07768E378E18091950690919606CF91EE
:100E80000C94114BCF910895CF93C82F8091910668
:100E900090919206DC01ED91FC91E05CFF4F019096
:100EA000F081E02D6C2F199580919706882389F0A9
:100EB00044DF6C2F80919506909196060E94A07752
:100EC00065E278E18091950690919606CF910C9419
:100ED000114BCF910895CF93C82F80919106909197
:100EE0009206DC01ED91FC9106ACF7ADE02D6C2F84
:100EF000199580919706882349F01FDF6C2F809108
:100F0000950690919606CF910C944B76CF910895CB
:100F10008091910690919206DC01ED91FC91048400
:100F2000F585E02D60E019948091910690919206EC
:100F3000DC01ED91FC910484F585E02D61E01994CC
:100F4000CF93DF938091C50F882349F180910102EF
:100F5000882329F1C0910C06D0910D068BA19CA18C
:100F6000892B11F01CA21BA22D8D3E8D8B8D9C8D8B
:100F70009B878A873D872C879F878E87E881F981A9
:100F80000190F081E02D60E070E0CE0119951F8A9C
:100F90001E8A0E941A6E6F8F78A389A39AA3DF918D
:100FA000CF910895CF93DF938091C50F882349F1A6
:100FB00080910102882329F1C0910C06D0910D0681
:100FC0008BA19CA1892B11F01CA21BA22D8D3E8D03
:100FD000898D9A8D9B878A873D872C879F878E87EF
:100FE000E881F9810190F081E02D60E070E0CE01B0
:100FF00019951F8A1E8A0E941A6E6F8F78A389A383
:101000009AA3DF91CF9108951F93CF93DF9390918F
:10101000C50F9923C9F0182FC0910C06D0910D0669
:10102000CE010E94D7668E899F89892B49F41123AE
:1010300019F0898D9A8D02C08B8D9C8D9F8B8E8B24
:1010400081E090E09CA38BA3DF91CF911F91089545
:10105000809101028823B9F01092010280919706D5
:10106000882341F068E078E180919506909196069A
:101070000E94114B0E948D7E8091F505882319F006
:1010800080918D06C1CF08958091010281111AC00F
:1010900081E08093010280919706882341F069EFF7
:1010A00077E180919506909196060E94114B0E94DF
:1010B0008D7E8091F505882329F080918D06811120
:1010C00071CF3ECF08950F931F930E9431776AD757
:1010D00080EF9AE00E94A05E0E944B630E948D7E8A
:1010E0008091EB099091EC09892B01F10E941A6E15
:1010F0000091E7091091E8092091E9093091EA0986
:10110000AB01BC01401B510B620B730B8091EB09CF
:101110009091EC09A0E0B0E084179507A607B70707
:1011200028F40E9406770E941C7722C08091F20961
:101130009091F309892BE1F00E941A6E0091E30966
:101140001091E4092091E5093091E609AB01BC0159
:10115000401B510B620B730B8091F2099091F309C4
:10116000A0E0B0E084179507A607B70708F45AC0B7
:101170008091E40F833041F12CF48130A9F082306A
:1011800099F02DC086305CF5809186069091870697
:10119000DC01ED91FC910680F781E02D199580919D
:1011A00084069091850614C080918A0690918B06E2
:1011B000DC01ED91FC910680F781E02D199580917D
:1011C00088069091890604C08091860690918706D2
:1011D000DC01ED91FC910680F781E02D199580915D
:1011E0008F0690919006DC01ED91FC910680F781CD
:1011F000E02D19958091930690919406DC01ED9174
:10120000FC910680F781E02D199580910C06909154
:101210000D06DC01ED91FC910680F781E02D1F9118
:101220000F9119948091F0098F5F8093F00990914C
:10123000F1098917E0F480FF03C00E94067702C01D
:101240000E9411778091F409811122C0E091F00988
:10125000EB3008F066CFF0E0EE0FFF1FEB50F64FDB
:10126000808191819093F3098093F20911C080915C
:10127000090A882309F455CF8091F5099091F60960
:101280009093F3098093F2091092F0090E9411776C
:101290000E941A6E6093E3097093E4098093E50954
:1012A0009093E60965CF4115510529F06115710547
:1012B00011F00C94C3790895EF92FF920F931F934E
:1012C000CF93DF931F921F92CDB7DEB78C018CE7CF
:1012D00089831A82F801E480F580FFEFEF1AFF0A94
:1012E000B701C8010E949048882381F0F80120814D
:1012F000318184819581BE016F5F7F4F820F931F83
:101300000E94DDB1F801F582E48281E00F900F9038
:10131000DF91CF911F910F91FF90EF900895AF92C1
:10132000BF92CF92DF92EF92FF920F931F93CF93D2
:10133000DF9300D01F92CDB7DEB78C0149835A836B
:101340006B837C83CE0101966C01580194E0A90E59
:10135000B11CE12CF12CC8010E94DDB3F6016191B2
:101360006F01861731F0C8010E94EFB3FFEFEF1A4B
:10137000FF0A0F5F1F4F0A151B0569F781E0EF2871
:1013800009F480E00F900F900F900F90DF91CF91B4
:101390001F910F91FF90EF90DF90CF90BF90AF9093
:1013A0000895CF92DF92EF92FF920F931F93CF9306
:1013B000DF93EC010091E512E0E0F0E020E030E0A6
:1013C000A90110E0CE17DF071CF1309711F40D32A0
:1013D000E1F0DF01AB51BD4EFC9080ED8F0D8A3006
:1013E000A8F4AAE0B0E00E9419B42F2DFF0C330B33
:1013F000205331096901330FEE08FF089B01AC014E
:101400002C0D3D1D4E1D5F1D01C011E03196DACF40
:10141000CA01B901112339F09095809570956195B5
:101420007F4F8F4F9F4FDF91CF911F910F91FF9073
:10143000EF90DF90CF9008958091DF0A811105C071
:1014400081E09091E10A911101C080E00895CF936D
:10145000DF9320910A0A30910B0AE9012697A881AF
:10146000B981A65FB54F12961C92082E000C990BFD
:10147000AA0BBB0BFC013197EE30F10508F057C108
:101480008827E458FE4F8F4F0C949AAEF9013A9793
:1014900080819181865F954F0E9479AC882309F401
:1014A0004BC1E0910A0AF0910B0A36970190F08146
:1014B000E02DE65FF54F81E0A0C0F9013C97808107
:1014C0009181865F954F0E94B6AB882309F434C1A1
:1014D000E0910A0AF0910B0A36970190F081E02D15
:1014E000E65FF54F82E089C0F9013E9780819181E6
:1014F000865F954F0E94F9AA882309F41DC1E091E7
:101500000A0AF0910B0A36970190F081E02DE65F10
:10151000F54F83E072C0F901709780819181865FF9
:10152000954F0E947CAA882309F406C1E0910A0A1B
:10153000F0910B0A36970190F081E02DE65FF54FB0
:1015400084E05BC0F901729780819181865F954F3D
:101550000E9437AA882309F4EFC0E0910A0AF091AB
:101560000B0A36970190F081E02DE65FF54F85E09C
:1015700044C0F901749780819181865F954F0E94E4
:10158000BEA9882309F4D8C0E0910A0AF0910B0A99
:1015900036970190F081E02DE65FF54F86E02DC093
:1015A000F901769780819181865F954F0E9438A9D5
:1015B000882309F4C1C0E0910A0AF0910B0A36971A
:1015C0000190F081E02DE65FF54F87E016C0F9014C
:1015D000789780819181865F954F0E942AA9882300
:1015E00009F4AAC0E0910A0AF0910B0A369701901B
:1015F000F081E02DE65FF54F88E082839DC0F90120
:10160000B09780819181865F954F0E944CA6882378
:1016100009F492C0E0910A0AF0910B0A3697019002
:10162000F081E02DE65FF54F83819481A581B6813D
:101630004097A105B10509F07FC08EC0F9017A97E6
:1016400080819181865F954F0E945FA8882309F46D
:1016500073C0E0910A0AF0910B0A36970190F0816D
:10166000E02DE65FF54F8AE0C8CFF9017C978081D5
:101670009181865F954F0E9494A7882309F45CC0EE
:10168000E0910A0AF0910B0A36970190F081E02D63
:10169000E65FF54F8BE0B1CFF901B0978081918182
:1016A000865F954F0E944CA6882309F445C0E091BF
:1016B0000A0AF0910B0A36970190F081E02DE65F5F
:1016C000F54F83819481A581B68180319440A10535
:1016D000B10591F543C0F9017E9780819181865FC4
:1016E000954F0E94C5A6882339F1E0910A0AF0912E
:1016F0000B0A36970190F081E02DE65FF54F8DE003
:101700007CCFF901B09780819181865F954F0E94CF
:101710004CA6882389F0E0910A0AF0910B0A3697CB
:101720000190F081E02DE65FF54F8EE066CFE88115
:10173000F981E65FF54F1282E0910A0AF0910B0AF7
:1017400036970190F081E02DE65FF54F81E09281C0
:10175000911106C080E004C089E04FCF8CE04DCFEE
:10176000DF91CF910895EF92FF920F931F93CF9344
:10177000DF931F921F92CDB7DEB741110AC07C01E3
:1017800097FF03C0F194E194F108E616F70664F4BC
:1017900002C0E12CF12C81E08093CC0A8FEF6333FF
:1017A00071059CF425E012C06E157F0534F010928F
:1017B000CC0A81E091E021E00AC06D337105BCF3F1
:1017C00081E08093CC0A23E001C024E092E03091D4
:1017D000CC0A332379F03FB7F894899F902D1124D8
:1017E0009093D00A2093E4120091E2121091E31238
:1017F0003FBF0AC09FB7F8941092D00AF092E3124C
:10180000E092E2129FBF87014A8389830E94157F7D
:101810004A818981442319F017FF19C014C081300F
:1018200031F417FD10C0E016F1068CF40FC08F3FA5
:1018300071F40E151F0554F00F3F110541F03CF0F7
:101840000FEF10E004C000E010E001C08701C80104
:101850000F900F90DF91CF911F910F91FF90EF901C
:101860000895CF92DF92EF92FF920F931F93CF9341
:10187000DF93042FE22E433049F0453039F04430F5
:1018800041F4F92EFF1CFF24FF1C04C0FF24F39435
:1018900001C0F12CFC0197FF03C0F195E195F1091E
:1018A000EF011092CD0A013009F432C1053009F080
:1018B0006EC08091F412811118C0C091E112D0E085
:1018C000D093F312C093F21281E08093CD0A21E00D
:1018D00030E03093F1122093F0123093E012209315
:1018E000DF128093F41211E0B9C08091DF12909161
:1018F000E01281159640E8F581E08093CD0A809151
:10190000DF129091E0122091F0123091F112821BBF
:10191000930BC091F212D091F312089720F1BE01FF
:1019200080E090E00E94B8B22091DB123091DC128E
:101930004091DD125091DE120E9419B320E030E098
:1019400040E05FE30E94AFAE0E947BAFEB0170937B
:10195000F3126093F2128091DF129091E012909353
:10196000F1128093F012CF31D1050CF075C0E1E097
:1019700001C0E0E01092CD0A1092F3121092F21220
:101980001092F4128E2F11E0C0E0D0E061C0EE2082
:10199000E1F0023029F48091C80A9091C90A04C08C
:1019A0008091CA0A9091CB0AE817F9070CF0B3C0EE
:1019B00081E08093CD0A8091DA1294E0F595E79565
:1019C0009A95E1F7EE5F1FEF43C0DB0177FF03C09D
:1019D000B195A195B109AE17BF07C4F48091D91292
:1019E000882309F49CC081E08093CD0A8091D812AD
:1019F0009091D7129130A1F5EA1BFB0BFD970CF0EB
:101A0000845011E054976CF5E4E02CC0EA17FB0712
:101A10000CF085C08091D612882309F480C0043070
:101A200009F47DC081E08093CD0A8091DA12909113
:101A3000D512913009F07CC0E233F10514F48E5FC9
:101A400077C0AE1BBF0BD3970CF472C0825070C02E
:101A50001E1644F0E1E006C011E081E0E1E006C0BE
:101A600011E0E2E0181614F06E0160C06E01909172
:101A7000CD0A9923D9F02FB7F8941E9F902D1124E9
:101A80009093D10A8093D4121C161D063CF48091C9
:101A9000DF129091E012892B09F44CC0053021F03F
:101AA000C091DF12D091E0122FBF09C08FB7F89418
:101AB0001092D10AD093E012C093DF128FBF0E9420
:101AC000157FEE2019F0D7FF1DC018C0113031F47A
:101AD000D7FD14C0CC16DD06ACF413C01F3F91F443
:101AE000023011F0033071F4CC15DD0554F0CF3F16
:101AF000D10541F03CF0CFEFD0E004C0C0E0D0E031
:101B000001C0E601FF2001F1D195C195D1091CC0AA
:101B100090E080E006C090E080E01FEF03C09E2FC1
:101B20008F2F11E06F01C92FD82FE1E081E09FCF07
:101B30001FEF97CF8091D10A082E000C990B90933C
:101B4000E0128093DF12AACFCE01DF91CF911F91D7
:101B50000F91FF90EF90DF90CF900895CF92DF929A
:101B6000EF92FF9297FF26C0CC24DD24C61AD70A35
:101B70000D2C000CEE08FF08092E000CAA0BBB0B65
:101B80009C01AD0121503F4F4F4F5F4FC701B60140
:101B900060957095809590950E9464AE2EEF30E030
:101BA00040E050E00E94FDB3C20ED31EE41EF51EBD
:101BB000C60126C0009711F1092E000CAA0BBB0B21
:101BC0009C01AD012150310941095109CB01770F29
:101BD000AA0BBB0BBC01CD016150710981099109B0
:101BE0000E9464AE2EEF30E040E050E00E94FDB372
:101BF000DA01C9010196A11DB11D02C080E090E08B
:101C0000FF90EF90DF90CF90089580919106909192
